 MFCD42UD

 Timestamp is 35887318 (Wed Jun 17 18:53:28 1998)

 Preferred load address is 5f700000

 Start         Length     Name                   Class
 0001:00000000 0002ca66H .text                   CODE
 0001:0002ca70 00000242H .text$AFX_CORE2         CODE
 0001:0002ccc0 00000520H .text$AFX_INIT          CODE
 0001:0002d1e0 00000583H .text$AFX_VDEL          CODE
 0001:0002d770 00001cc0H .text$x                 CODE
 0002:00000000 00000528H .idata$5                DATA
 0002:00000530 0000889cH .rdata                  DATA
 0002:00008dd0 000007acH .rdata$r                DATA
 0002:00009580 000033d8H .xdata$x                DATA
 0002:0000c958 00000060H .didat$2                DATA
 0002:0000c9b8 00000020H .didat$3                DATA
 0002:0000c9d8 0000009cH .didat$4                DATA
 0002:0000ca74 00000036H .didat$6                DATA
 0002:0000caac 0000009cH .didat$7                DATA
 0002:0000cb48 00000064H .idata$2                DATA
 0002:0000cbac 00000014H .idata$3                DATA
 0002:0000cbc0 00000528H .idata$4                DATA
 0002:0000d0e8 0000034eH .idata$6                DATA
 0002:0000d440 00000b39H .edata                  DATA
 0003:00000000 00000004H .CRT$XCA                DATA
 0003:00000004 00000004H .CRT$XCL                DATA
 0003:00000008 00000004H .CRT$XCZ                DATA
 0003:0000000c 00000004H .CRT$XIA                DATA
 0003:00000010 00000004H .CRT$XIZ                DATA
 0003:00000020 00000540H .data                   DATA
 0003:00000560 0000009cH .didat$5                DATA
 0003:00000600 00000064H .bss                    DATA
 0004:00000000 00000100H .rsrc$01                DATA
 0004:00000100 00001030H .rsrc$02                DATA

  Address         Publics by Value              Rva+Base     Lib:Object

 0001:00000000       ?GetHead@CSimpleList@@QBEPAXXZ 5f701000 f i dlldb.obj
 0001:00000010       ?AfxThrowDBException@@YGXFPAVCDatabase@@PAX@Z 5f701010 f   dbcore.obj
 0001:00000121       ??0CDBException@@QAE@F@Z   5f701121 f   dbcore.obj
 0001:00000194       ??1CDBException@@UAE@XZ    5f701194 f   dbcore.obj
 0001:000001f7       ?BuildErrorString@CDBException@@UAEXPAVCDatabase@@PAXH@Z 5f7011f7 f   dbcore.obj
 0001:000005cf       ?GetErrorMessage@CDBException@@UAEHPAGIPAI@Z 5f7015cf f   dbcore.obj
 0001:00000651       ?TraceErrorMessage@CDBException@@QBEXPBG@Z 5f701651 f   dbcore.obj
 0001:0000075e       ?Empty@CDBException@@QAEXXZ 5f70175e f   dbcore.obj
 0001:0000077f       ?AfxGetHENV@@YGPAXXZ       5f70177f f   dbcore.obj
 0001:0000079a       ??0CDatabase@@QAE@XZ       5f70179a f   dbcore.obj
 0001:00000866       ??1CDatabase@@UAE@XZ       5f701866 f   dbcore.obj
 0001:000008e8       ?Open@CDatabase@@UAEHPBGHH0H@Z 5f7018e8 f   dbcore.obj
 0001:00000ac8       ?OpenEx@CDatabase@@UAEHPBGK@Z 5f701ac8 f   dbcore.obj
 0001:00000c3c       ?ExecuteSQL@CDatabase@@QAEXPBG@Z 5f701c3c f   dbcore.obj
 0001:00000edf       ?Cancel@CDatabase@@QAEXXZ  5f701edf f   dbcore.obj
 0001:00000f32       ?Close@CDatabase@@UAEXXZ   5f701f32 f   dbcore.obj
 0001:000010a7       ?Free@CDatabase@@IAEXXZ    5f7020a7 f   dbcore.obj
 0001:000011e2       ?OnSetOptions@CDatabase@@UAEXPAX@Z 5f7021e2 f   dbcore.obj
 0001:00001270       ?GetDatabaseName@CDatabase@@QBE?AVCString@@XZ 5f702270 f   dbcore.obj
 0001:00001314       ?BeginTrans@CDatabase@@QAEHXZ 5f702314 f   dbcore.obj
 0001:000013c1       ?CommitTrans@CDatabase@@QAEHXZ 5f7023c1 f   dbcore.obj
 0001:000014a3       ?Rollback@CDatabase@@QAEHXZ 5f7024a3 f   dbcore.obj
 0001:00001585       ?Check@CDatabase@@UBEHF@Z  5f702585 f   dbcore.obj
 0001:000015a2       ?CheckHstmt@CDatabase@@QBGHFPAX@Z 5f7025a2 f   dbcore.obj
 0001:0000165a       ?ReplaceBrackets@CDatabase@@QAEXPAG@Z 5f70265a f   dbcore.obj
 0001:000017cd       ?AllocConnect@CDatabase@@IAEXK@Z 5f7027cd f   dbcore.obj
 0001:000019f9       ?Connect@CDatabase@@IAEHK@Z 5f7029f9 f   dbcore.obj
 0001:00001c13       ?VerifyConnect@CDatabase@@IAEXXZ 5f702c13 f   dbcore.obj
 0001:00001cdd       ?GetConnectInfo@CDatabase@@IAEXXZ 5f702cdd f   dbcore.obj
 0001:00002102       ?BindParameters@CDatabase@@UAEXPAX@Z 5f703102 f   dbcore.obj
 0001:0000210f       ?AssertValid@CDatabase@@UBEXXZ 5f70310f f   dbcore.obj
 0001:00002122       ?Dump@CDatabase@@UBEXAAVCDumpContext@@@Z 5f703122 f   dbcore.obj
 0001:00002262       ??0CRecordset@@QAE@PAVCDatabase@@@Z 5f703262 f   dbcore.obj
 0001:000026ba       ??1CRecordset@@UAE@XZ      5f7036ba f   dbcore.obj
 0001:000028eb       ?Open@CRecordset@@UAEHIPBGK@Z 5f7038eb f   dbcore.obj
 0001:00002bbc       ?Close@CRecordset@@UAEXXZ  5f703bbc f   dbcore.obj
 0001:00002fb8       ?IsOpen@CRecordset@@QBEHXZ 5f703fb8 f   dbcore.obj
 0001:0000312e       ?IsFieldDirty@CRecordset@@QAEHPAX@Z 5f70412e f   dbcore.obj
 0001:00003278       ?IsFieldNull@CRecordset@@QAEHPAX@Z 5f704278 f   dbcore.obj
 0001:0000334c       ?IsFieldNullable@CRecordset@@QAEHPAX@Z 5f70434c f   dbcore.obj
 0001:000033d7       ?CanBookmark@CRecordset@@QBEHXZ 5f7043d7 f   dbcore.obj
 0001:00003462       ?Move@CRecordset@@UAEXJG@Z 5f704462 f   dbcore.obj
 0001:000035fb       ?CheckRowsetError@CRecordset@@UAEXF@Z 5f7045fb f   dbcore.obj
 0001:00003787       ?GetBookmark@CRecordset@@QAEXAAVCDBVariant@@@Z 5f704787 f   dbcore.obj
 0001:00003872       ?SetBookmark@CRecordset@@QAEXABVCDBVariant@@@Z 5f704872 f   dbcore.obj
 0001:00003911       ?SetRowsetSize@CRecordset@@UAEXK@Z 5f704911 f   dbcore.obj
 0001:00003a9e       ?AddNew@CRecordset@@UAEXXZ 5f704a9e f   dbcore.obj
 0001:00003bb8       ?Edit@CRecordset@@UAEXXZ   5f704bb8 f   dbcore.obj
 0001:00003d82       ?Update@CRecordset@@UAEHXZ 5f704d82 f   dbcore.obj
 0001:00003e44       ?Delete@CRecordset@@UAEXXZ 5f704e44 f   dbcore.obj
 0001:00003ef8       ?CancelUpdate@CRecordset@@QAEXXZ 5f704ef8 f   dbcore.obj
 0001:00003f77       ?FlushResultSet@CRecordset@@QBEHXZ 5f704f77 f   dbcore.obj
 0001:00003fef       ?GetODBCFieldInfo@CRecordset@@QAEXPBGAAUCODBCFieldInfo@@@Z 5f704fef f   dbcore.obj
 0001:000040b2       ?GetODBCFieldInfo@CRecordset@@QAEXFAAUCODBCFieldInfo@@@Z 5f7050b2 f   dbcore.obj
 0001:00004188       ?GetFieldValue@CRecordset@@QAEXPBGAAVCDBVariant@@F@Z 5f705188 f   dbcore.obj
 0001:00004258       ?GetFieldValue@CRecordset@@QAEXFAAVCDBVariant@@F@Z 5f705258 f   dbcore.obj
 0001:0000452e       ?GetFieldValue@CRecordset@@QAEXPBGAAVCString@@@Z 5f70552e f   dbcore.obj
 0001:000045f1       ?GetFieldValue@CRecordset@@QAEXFAAVCString@@@Z 5f7055f1 f   dbcore.obj
 0001:000047d1       ?SetFieldDirty@CRecordset@@QAEXPAXH@Z 5f7057d1 f   dbcore.obj
 0001:0000488a       ?SetFieldNull@CRecordset@@QAEXPAXH@Z 5f70588a f   dbcore.obj
 0001:000049bd       ?SetParamNull@CRecordset@@QAEXHH@Z 5f7059bd f   dbcore.obj
 0001:00004a3c       ?SetLockingMode@CRecordset@@QAEXI@Z 5f705a3c f   dbcore.obj
 0001:00004ab2       ?Requery@CRecordset@@UAEHXZ 5f705ab2 f   dbcore.obj
 0001:00004d45       ?Cancel@CRecordset@@QAEXXZ 5f705d45 f   dbcore.obj
 0001:00004db3       ?GetDefaultConnect@CRecordset@@UAE?AVCString@@XZ 5f705db3 f   dbcore.obj
 0001:00004df5       ?GetDefaultSQL@CRecordset@@UAE?AVCString@@XZ 5f705df5 f   dbcore.obj
 0001:00004e37       ?DoFieldExchange@CRecordset@@UAEXPAVCFieldExchange@@@Z 5f705e37 f   dbcore.obj
 0001:00004e57       ?DoBulkFieldExchange@CRecordset@@UAEXPAVCFieldExchange@@@Z 5f705e57 f   dbcore.obj
 0001:00004ea0       ?OnSetOptions@CRecordset@@UAEXPAX@Z 5f705ea0 f   dbcore.obj
 0001:00004f5c       ?Check@CRecordset@@UBEHF@Z 5f705f5c f   dbcore.obj
 0001:00005092       ?PreBindFields@CRecordset@@UAEXXZ 5f706092 f   dbcore.obj
 0001:0000509d       ?SetState@CRecordset@@IAEXHPBGK@Z 5f70609d f   dbcore.obj
 0001:000051ec       ?AllocHstmt@CRecordset@@IAEHXZ 5f7061ec f   dbcore.obj
 0001:000055f9       ?BuildSQL@CRecordset@@IAEXPBG@Z 5f7065f9 f   dbcore.obj
 0001:00005775       ?PrepareAndExecute@CRecordset@@IAEXXZ 5f706775 f   dbcore.obj
 0001:00005b76       ?VerifyDriverBehavior@CRecordset@@IAEXXZ 5f706b76 f   dbcore.obj
 0001:00005cce       ?VerifyCursorSupport@CRecordset@@IAEKXZ 5f706cce f   dbcore.obj
 0001:00005dc7       ?AllocAndCacheFieldInfo@CRecordset@@IAEXXZ 5f706dc7 f   dbcore.obj
 0001:00006087       ?AllocRowset@CRecordset@@IAEXXZ 5f707087 f   dbcore.obj
 0001:000060eb       ?FreeRowset@CRecordset@@IAEXXZ 5f7070eb f   dbcore.obj
 0001:00006175       ?EnableBookmarks@CRecordset@@IAEXXZ 5f707175 f   dbcore.obj
 0001:000061f6       ?SetUpdateMethod@CRecordset@@IAEXXZ 5f7071f6 f   dbcore.obj
 0001:00006246       ?SetConcurrencyAndCursorType@CRecordset@@IAEXPAXK@Z 5f707246 f   dbcore.obj
 0001:00006441       ?IsSQLUpdatable@CRecordset@@QAEHPBG@Z 5f707441 f   dbcore.obj
 0001:000064a8       ?IsSelectQueryUpdatable@CRecordset@@QAEHPBG@Z 5f7074a8 f   dbcore.obj
 0001:0000674a       ?IsJoin@CRecordset@@SGHPBG@Z 5f70774a f   dbcore.obj
 0001:00006785       ?FindSQLToken@CRecordset@@SGPBGPBG0@Z 5f707785 f   dbcore.obj
 0001:000069ca       ?InitRecord@CRecordset@@QAEXXZ 5f7079ca f   dbcore.obj
 0001:00006a49       ?ResetCursor@CRecordset@@QAEXXZ 5f707a49 f   dbcore.obj
 0001:00006aa2       ?CheckRowsetCurrencyStatus@CRecordset@@QAEXGJ@Z 5f707aa2 f   dbcore.obj
 0001:00006bde       ?FetchData@CRecordset@@QAEFGJPAK@Z 5f707bde f   dbcore.obj
 0001:00006ccb       ?SkipDeletedRecords@CRecordset@@QAEXGJPAKPAF@Z 5f707ccb f   dbcore.obj
 0001:00006ed8       ?SetRowsetCurrencyStatus@CRecordset@@UAEXFGJK@Z 5f707ed8 f   dbcore.obj
 0001:00007209       ?RefreshRowset@CRecordset@@QAEXGG@Z 5f708209 f   dbcore.obj
 0001:000072cc       ?SetRowsetCursorPosition@CRecordset@@QAEXGG@Z 5f7082cc f   dbcore.obj
 0001:00007356       ?BuildSelectSQL@CRecordset@@IAEXXZ 5f708356 f   dbcore.obj
 0001:000075a3       ?AppendFilterAndSortSQL@CRecordset@@IAEXXZ 5f7085a3 f   dbcore.obj
 0001:0000761c       ?IsRecordsetUpdatable@CRecordset@@IAEHXZ 5f70861c f   dbcore.obj
 0001:000076f5       ?ExecuteSetPosUpdate@CRecordset@@IAEXXZ 5f7086f5 f   dbcore.obj
 0001:00007801       ?PrepareUpdateHstmt@CRecordset@@IAEXXZ 5f708801 f   dbcore.obj
 0001:00007991       ?BuildUpdateSQL@CRecordset@@IAEXXZ 5f708991 f   dbcore.obj
 0001:00007dd3       ?ExecuteUpdateSQL@CRecordset@@IAEXXZ 5f708dd3 f   dbcore.obj
 0001:00007fb8       ?SendLongBinaryData@CRecordset@@IAEXPAX@Z 5f708fb8 f   dbcore.obj
 0001:00008215       ?AllocStatusArrays@CRecordset@@QAEXXZ 5f709215 f   dbcore.obj
 0001:0000840c       ?GetBoundFieldIndex@CRecordset@@QAEHPAX@Z 5f70940c f   dbcore.obj
 0001:0000843a       ?GetBoundParamIndex@CRecordset@@QAEHPAX@Z 5f70943a f   dbcore.obj
 0001:00008468       ?GetFieldIndexByName@CRecordset@@QAEFPBG@Z 5f709468 f   dbcore.obj
 0001:000084ef       ?GetFieldLengthBuffer@CRecordset@@QAEPAJKH@Z 5f7094ef f   dbcore.obj
 0001:00008573       ?GetFieldStatus@CRecordset@@QAEEK@Z 5f709573 f   dbcore.obj
 0001:000085ba       ?SetFieldStatus@CRecordset@@QAEXKE@Z 5f7095ba f   dbcore.obj
 0001:00008613       ?ClearFieldStatus@CRecordset@@QAEXXZ 5f709613 f   dbcore.obj
 0001:00008639       ?IsFieldStatusDirty@CRecordset@@QBEHK@Z 5f709639 f   dbcore.obj
 0001:00008685       ?SetDirtyFieldStatus@CRecordset@@QAEXK@Z 5f709685 f   dbcore.obj
 0001:000086dd       ?ClearDirtyFieldStatus@CRecordset@@QAEXK@Z 5f7096dd f   dbcore.obj
 0001:00008735       ?IsFieldStatusNull@CRecordset@@QBEHK@Z 5f709735 f   dbcore.obj
 0001:00008781       ?SetNullFieldStatus@CRecordset@@QAEXK@Z 5f709781 f   dbcore.obj
 0001:000087d9       ?ClearNullFieldStatus@CRecordset@@QAEXK@Z 5f7097d9 f   dbcore.obj
 0001:00008831       ?IsParamStatusNull@CRecordset@@QBEHK@Z 5f709831 f   dbcore.obj
 0001:0000887d       ?SetNullParamStatus@CRecordset@@QAEXK@Z 5f70987d f   dbcore.obj
 0001:000088d5       ?ClearNullParamStatus@CRecordset@@QAEXK@Z 5f7098d5 f   dbcore.obj
 0001:0000892d       ?IsFieldNullable@CRecordset@@QBEHK@Z 5f70992d f   dbcore.obj
 0001:000089a4       ?BindParams@CRecordset@@QAEIPAX@Z 5f7099a4 f   dbcore.obj
 0001:00008a17       ?RebindParams@CRecordset@@QAEXPAX@Z 5f709a17 f   dbcore.obj
 0001:00008a90       ?BindFieldsToColumns@CRecordset@@QAEIXZ 5f709a90 f   dbcore.obj
 0001:00008b79       ?BindFieldsForUpdate@CRecordset@@QAEXXZ 5f709b79 f   dbcore.obj
 0001:00008bd9       ?UnbindFieldsForUpdate@CRecordset@@QAEXXZ 5f709bd9 f   dbcore.obj
 0001:00008c39       ?Fixups@CRecordset@@QAEXXZ 5f709c39 f   dbcore.obj
 0001:00008cd0       ?AppendNames@CRecordset@@QAEIPAVCString@@PBG@Z 5f709cd0 f   dbcore.obj
 0001:00008dbe       ?AppendNamesValues@CRecordset@@QAEIPAXPAVCString@@PBG@Z 5f709dbe f   dbcore.obj
 0001:00008eb1       ?AppendValues@CRecordset@@QAEIPAXPAVCString@@PBG@Z 5f709eb1 f   dbcore.obj
 0001:00008fa4       ?StoreFields@CRecordset@@QAEXXZ 5f709fa4 f   dbcore.obj
 0001:0000900f       ?LoadFields@CRecordset@@QAEXXZ 5f70a00f f   dbcore.obj
 0001:00009082       ?MarkForUpdate@CRecordset@@QAEXXZ 5f70a082 f   dbcore.obj
 0001:000090c1       ?MarkForAddNew@CRecordset@@QAEXXZ 5f70a0c1 f   dbcore.obj
 0001:00009100       ?AllocDataCache@CRecordset@@QAEXXZ 5f70a100 f   dbcore.obj
 0001:0000913f       ?FreeDataCache@CRecordset@@QAEXXZ 5f70a13f f   dbcore.obj
 0001:0000933c       ?DumpFields@CRecordset@@QBEXAAVCDumpContext@@@Z 5f70a33c f   dbcore.obj
 0001:00009370       ?UpdateInsertDelete@CRecordset@@IAEHXZ 5f70a370 f   dbcore.obj
 0001:00009708       ?GetLBFetchSize@CRecordset@@MAEJJ@Z 5f70a708 f   dbcore.obj
 0001:0000971a       ?GetLBReallocSize@CRecordset@@MAEJJ@Z 5f70a71a f   dbcore.obj
 0001:0000972c       ?GetDefaultFieldType@CRecordset@@SGFF@Z 5f70a72c f   dbcore.obj
 0001:00009823       ?GetDataBuffer@CRecordset@@SGPAXAAVCDBVariant@@FPAHFK@Z 5f70a823 f   dbcore.obj
 0001:00009b50       ?GetTextLen@CRecordset@@SGHFK@Z 5f70ab50 f   dbcore.obj
 0001:00009bc2       ?GetData@CRecordset@@SGJPAVCDatabase@@PAXFF1HF@Z 5f70abc2 f   dbcore.obj
 0001:00009d5c       ?GetLongCharDataAndCleanup@CRecordset@@SGXPAVCDatabase@@PAXFJPAPAXHAAVCString@@F@Z 5f70ad5c f   dbcore.obj
 0001:00009ece       ?GetLongBinaryDataAndCleanup@CRecordset@@SGXPAVCDatabase@@PAXFJPAPAXHAAVCDBVariant@@F@Z 5f70aece f   dbcore.obj
 0001:0000a096       ?AssertValid@CRecordset@@UBEXXZ 5f70b096 f   dbcore.obj
 0001:0000a0c3       ?Dump@CRecordset@@UBEXAAVCDumpContext@@@Z 5f70b0c3 f   dbcore.obj
 0001:0000a344       ?AfxSetCurrentRecord@@YGXPAJJF@Z 5f70b344 f   dbcore.obj
 0001:0000a369       ?AfxSetRecordCount@@YGXPAJJJHF@Z 5f70b369 f   dbcore.obj
 0001:0000a3ac       ?AfxSetRecordCount@@YGXPAJJHF@Z 5f70b3ac f   dbcore.obj
 0001:0000a3f3       ?IsOpen@CDatabase@@QBEHXZ  5f70b3f3 f   dbcore.obj
 0001:0000a41a       ?CanUpdate@CDatabase@@QBEHXZ 5f70b41a f   dbcore.obj
 0001:0000a454       ?CanTransact@CDatabase@@QBEHXZ 5f70b454 f   dbcore.obj
 0001:0000a48e       ?SetLoginTimeout@CDatabase@@QAEXK@Z 5f70b48e f   dbcore.obj
 0001:0000a4b4       ?SetQueryTimeout@CDatabase@@QAEXK@Z 5f70b4b4 f   dbcore.obj
 0001:0000a4da       ?GetConnect@CDatabase@@QBEABVCString@@XZ 5f70b4da f   dbcore.obj
 0001:0000a4fb       ?GetBookmarkPersistence@CDatabase@@QBEKXZ 5f70b4fb f   dbcore.obj
 0001:0000a51c       ?GetCursorCommitBehavior@CDatabase@@QBEHXZ 5f70b51c f   dbcore.obj
 0001:0000a53e       ?GetCursorRollbackBehavior@CDatabase@@QBEHXZ 5f70b53e f   dbcore.obj
 0001:0000a560       ?ThrowDBException@CDatabase@@MAEXF@Z 5f70b560 f   dbcore.obj
 0001:0000a592       ?SetSynchronousMode@CDatabase@@QAEXH@Z 5f70b592 f   dbcore.obj
 0001:0000a5c1       ?GetSQL@CRecordset@@QBEABVCString@@XZ 5f70b5c1 f   dbcore.obj
 0001:0000a5fd       ?GetTableName@CRecordset@@QBEABVCString@@XZ 5f70b5fd f   dbcore.obj
 0001:0000a639       ?IsBOF@CRecordset@@QBEHXZ  5f70b639 f   dbcore.obj
 0001:0000a676       ?IsEOF@CRecordset@@QBEHXZ  5f70b676 f   dbcore.obj
 0001:0000a6b3       ?IsDeleted@CRecordset@@QBEHXZ 5f70b6b3 f   dbcore.obj
 0001:0000a6f0       ?CanUpdate@CRecordset@@QBEHXZ 5f70b6f0 f   dbcore.obj
 0001:0000a72d       ?CanScroll@CRecordset@@QBEHXZ 5f70b72d f   dbcore.obj
 0001:0000a76a       ?CanAppend@CRecordset@@QBEHXZ 5f70b76a f   dbcore.obj
 0001:0000a7a7       ?CanRestart@CRecordset@@QBEHXZ 5f70b7a7 f   dbcore.obj
 0001:0000a7eb       ?CanTransact@CRecordset@@QBEHXZ 5f70b7eb f   dbcore.obj
 0001:0000a82b       ?GetODBCFieldCount@CRecordset@@QBEFXZ 5f70b82b f   dbcore.obj
 0001:0000a866       ?GetRowsetSize@CRecordset@@QBEKXZ 5f70b866 f   dbcore.obj
 0001:0000a8a3       ?GetRowsFetched@CRecordset@@QBEKXZ 5f70b8a3 f   dbcore.obj
 0001:0000a8e0       ?GetRowStatus@CRecordset@@QBEGG@Z 5f70b8e0 f   dbcore.obj
 0001:0000a950       ?GetRecordCount@CRecordset@@QBEJXZ 5f70b950 f   dbcore.obj
 0001:0000a98d       ?GetStatus@CRecordset@@QBEXAAUCRecordsetStatus@@@Z 5f70b98d f   dbcore.obj
 0001:0000a9e0       ?ThrowDBException@CRecordset@@UAEXFPAX@Z 5f70b9e0 f   dbcore.obj
 0001:0000aa2b       ?MoveNext@CRecordset@@QAEXXZ 5f70ba2b f   dbcore.obj
 0001:0000aa6e       ?MovePrev@CRecordset@@QAEXXZ 5f70ba6e f   dbcore.obj
 0001:0000aab1       ?MoveFirst@CRecordset@@QAEXXZ 5f70bab1 f   dbcore.obj
 0001:0000aaf4       ?MoveLast@CRecordset@@QAEXXZ 5f70baf4 f   dbcore.obj
 0001:0000ab37       ?SetAbsolutePosition@CRecordset@@QAEXJ@Z 5f70bb37 f   dbcore.obj
 0001:0000ab80       ??_ECDBException@@UAEPAXI@Z 5f70bb80 f i dbcore.obj
 0001:0000ab80       ??_GCDBException@@UAEPAXI@Z 5f70bb80 f i dbcore.obj
 0001:0000abb0       ??_GCDatabase@@UAEPAXI@Z   5f70bbb0 f i dbcore.obj
 0001:0000abe0       ?AtlW2AHelper@@YGPADPADPBGH@Z 5f70bbe0 f i dbcore.obj
 0001:0000ac00       ?AtlW2AHelper@@YGPADPADPBGHI@Z 5f70bc00 f i dbcore.obj
 0001:0000ac90       __wcsinc                   5f70bc90 f i dbcore.obj
 0001:0000aca0       ??_GCRecordset@@UAEPAXI@Z  5f70bca0 f i dbcore.obj
 0001:0000aca0       ??_ECRecordset@@UAEPAXI@Z  5f70bca0 f i dbcore.obj
 0001:0000acd0       ??_ECODBCFieldInfo@@QAEPAXI@Z 5f70bcd0 f i dbcore.obj
 0001:0000ad40       ??1CODBCFieldInfo@@QAE@XZ  5f70bd40 f i dbcore.obj
 0001:0000ad60       ??_GCString@@QAEPAXI@Z     5f70bd60 f i dbcore.obj
 0001:0000ad90       ??0CODBCFieldInfo@@QAE@XZ  5f70bd90 f i dbcore.obj
 0001:0000adb0       ??_GCNoTrackObject@@UAEPAXI@Z 5f70bdb0 f i dbcore.obj
 0001:0000adb0       ??_ECNoTrackObject@@UAEPAXI@Z 5f70bdb0 f i dbcore.obj
 0001:0000ade0       ??1CNoTrackObject@@UAE@XZ  5f70bde0 f i dbcore.obj
 0001:0000ae00       ??0CFieldExchange@@QAE@IPAVCRecordset@@PAX@Z 5f70be00 f   dbrfx.obj
 0001:0000aedd       ?IsFieldType@CFieldExchange@@QAEHPAI@Z 5f70bedd f   dbrfx.obj
 0001:0000afdd       ?Default@CFieldExchange@@QAEXPBGPAXPAJHII@Z 5f70bfdd f   dbrfx.obj
 0001:0000b602       ?RFX_Text@@YGXPAVCFieldExchange@@PBGPAGHHF@Z 5f70c602 f   dbrfx.obj
 0001:0000c2e0       ?RFX_Text@@YGXPAVCFieldExchange@@PBGAAVCString@@HHF@Z 5f70d2e0 f   dbrfx.obj
 0001:0000d0cb       ?RFX_Int@@YGXPAVCFieldExchange@@PBGAAH@Z 5f70e0cb f   dbrfx.obj
 0001:0000d368       ?RFX_Long@@YGXPAVCFieldExchange@@PBGAAJ@Z 5f70e368 f   dbrfx.obj
 0001:0000d605       ?RFX_Byte@@YGXPAVCFieldExchange@@PBGAAE@Z 5f70e605 f   dbrfx.obj
 0001:0000d8a4       ?RFX_Bool@@YGXPAVCFieldExchange@@PBGAAH@Z 5f70e8a4 f   dbrfx.obj
 0001:0000db49       ?RFX_Binary@@YGXPAVCFieldExchange@@PBGAAVCByteArray@@H@Z 5f70eb49 f   dbrfx.obj
 0001:0000e024       ?RFX_Date@@YGXPAVCFieldExchange@@PBGAAVCTime@@@Z 5f70f024 f   dbrfx.obj
 0001:0000ebd4       ?RFX_Date@@YGXPAVCFieldExchange@@PBGAAUtagTIMESTAMP_STRUCT@@@Z 5f70fbd4 f   dbrfx.obj
 0001:0000f0ff       ?RFX_Date@@YGXPAVCFieldExchange@@PBGAAVCOleDateTime@@@Z 5f7100ff f   dbrfx.obj
 0001:0000fc1a       ?RFX_LongBinary@@YGXPAVCFieldExchange@@PBGAAVCLongBinary@@@Z 5f710c1a f   dbrfx.obj
 0001:000101e1       ?GetLongBinarySize@CFieldExchange@@QAEJH@Z 5f7111e1 f   dbrfx.obj
 0001:0001034d       ?GetLongBinaryData@CFieldExchange@@QAEXHAAVCLongBinary@@PAJ@Z 5f71134d f   dbrfx.obj
 0001:000105d8       ?ReallocLongBinary@CFieldExchange@@QAEPAEAAVCLongBinary@@JJ@Z 5f7115d8 f   dbrfx.obj
 0001:000106dd       ?AfxStoreField@@YGXAAVCRecordset@@IPAX@Z 5f7116dd f   dbrfx.obj
 0001:00010828       ?AfxLoadField@@YGXAAVCRecordset@@IPAXPAJ@Z 5f711828 f   dbrfx.obj
 0001:00010934       ?AfxCompareValueByRef@@YGHPAX0H@Z 5f711934 f   dbrfx.obj
 0001:00010c26       ?AfxCopyValueByRef@@YGXPAX0PAJH@Z 5f711c26 f   dbrfx.obj
 0001:00010ebb       ?RFX_Text_Bulk@@YGXPAVCFieldExchange@@PBGPAPADPAPAJH@Z 5f711ebb f   dbrfx.obj
 0001:0001104b       ?RFX_Bool_Bulk@@YGXPAVCFieldExchange@@PBGPAPAHPAPAJ@Z 5f71204b f   dbrfx.obj
 0001:000111d8       ?RFX_Int_Bulk@@YGXPAVCFieldExchange@@PBGPAPAHPAPAJ@Z 5f7121d8 f   dbrfx.obj
 0001:00011365       ?RFX_Long_Bulk@@YGXPAVCFieldExchange@@PBGPAPAJ2@Z 5f712365 f   dbrfx.obj
 0001:000114f2       ?RFX_Date_Bulk@@YGXPAVCFieldExchange@@PBGPAPAUtagTIMESTAMP_STRUCT@@PAPAJ@Z 5f7124f2 f   dbrfx.obj
 0001:0001167f       ?RFX_Byte_Bulk@@YGXPAVCFieldExchange@@PBGPAPAEPAPAJ@Z 5f71267f f   dbrfx.obj
 0001:00011809       ?RFX_Binary_Bulk@@YGXPAVCFieldExchange@@PBGPAPAEPAPAJH@Z 5f712809 f   dbrfx.obj
 0001:00011999       ?AfxRFXBulkDefault@@YGXPAVCFieldExchange@@PBGPAXPAJHI@Z 5f712999 f   dbrfx.obj
 0001:00011a96       ?SetFieldType@CFieldExchange@@QAEXI@Z 5f712a96 f   dbrfx.obj
 0001:00011af0       ?SetLength@CDBByteArray@@QAEXH@Z 5f712af0 f i dbrfx.obj
 0001:00011b30       ?_GetBaseMessageMap@CRecordView@@KGPBUAFX_MSGMAP@@XZ 5f712b30 f   dbview.obj
 0001:00011b3a       ?GetMessageMap@CRecordView@@MBEPBUAFX_MSGMAP@@XZ 5f712b3a f   dbview.obj
 0001:00011b4a       ??0CRecordView@@IAE@PBG@Z  5f712b4a f   dbview.obj
 0001:00011b6f       ??0CRecordView@@IAE@I@Z    5f712b6f f   dbview.obj
 0001:00011b94       ??1CRecordView@@UAE@XZ     5f712b94 f   dbview.obj
 0001:00011bb0       ?OnInitialUpdate@CRecordView@@UAEXXZ 5f712bb0 f   dbview.obj
 0001:00011c53       ?IsOnFirstRecord@CRecordView@@QAEHXZ 5f712c53 f   dbview.obj
 0001:00011c92       ?IsOnLastRecord@CRecordView@@QAEHXZ 5f712c92 f   dbview.obj
 0001:00011cef       ?OnMove@CRecordView@@UAEHI@Z 5f712cef f   dbview.obj
 0001:00011e19       ?OnUpdateRecordFirst@CRecordView@@IAEXPAVCCmdUI@@@Z 5f712e19 f   dbview.obj
 0001:00011e93       ?OnUpdateRecordPrev@CRecordView@@IAEXPAVCCmdUI@@@Z 5f712e93 f   dbview.obj
 0001:00011eac       ?OnUpdateRecordNext@CRecordView@@IAEXPAVCCmdUI@@@Z 5f712eac f   dbview.obj
 0001:00011f1a       ?OnUpdateRecordLast@CRecordView@@IAEXPAVCCmdUI@@@Z 5f712f1a f   dbview.obj
 0001:00011f94       ?AfxFieldText@@YGHPAVCDataExchange@@HPAXPAVCRecordset@@@Z 5f712f94 f   dbview.obj
 0001:000120c8       ?DDX_FieldText@@YGXPAVCDataExchange@@HAAHPAVCRecordset@@@Z 5f7130c8 f   dbview.obj
 0001:000120f9       ?DDX_FieldText@@YGXPAVCDataExchange@@HAAEPAVCRecordset@@@Z 5f7130f9 f   dbview.obj
 0001:0001212a       ?DDX_FieldText@@YGXPAVCDataExchange@@HAAIPAVCRecordset@@@Z 5f71312a f   dbview.obj
 0001:0001215b       ?DDX_FieldText@@YGXPAVCDataExchange@@HAAJPAVCRecordset@@@Z 5f71315b f   dbview.obj
 0001:0001218c       ?DDX_FieldText@@YGXPAVCDataExchange@@HAAKPAVCRecordset@@@Z 5f71318c f   dbview.obj
 0001:000121bd       ?DDX_FieldText@@YGXPAVCDataExchange@@HAAVCString@@PAVCRecordset@@@Z 5f7131bd f   dbview.obj
 0001:00012370       ?DDX_FieldText@@YGXPAVCDataExchange@@HPAGHPAVCRecordset@@@Z 5f713370 f   dbview.obj
 0001:00012460       ?DDX_FieldLBString@@YGXPAVCDataExchange@@HAAVCString@@PAVCRecordset@@@Z 5f713460 f   dbview.obj
 0001:000125db       ?DDX_FieldLBStringExact@@YGXPAVCDataExchange@@HAAVCString@@PAVCRecordset@@@Z 5f7135db f   dbview.obj
 0001:000126a5       ?DDX_FieldLBIndex@@YGXPAVCDataExchange@@HAAHPAVCRecordset@@@Z 5f7136a5 f   dbview.obj
 0001:00012711       ?DDX_FieldCBString@@YGXPAVCDataExchange@@HAAVCString@@PAVCRecordset@@@Z 5f713711 f   dbview.obj
 0001:000128d8       ?DDX_FieldCBStringExact@@YGXPAVCDataExchange@@HAAVCString@@PAVCRecordset@@@Z 5f7138d8 f   dbview.obj
 0001:000129a2       ?DDX_FieldCBIndex@@YGXPAVCDataExchange@@HAAHPAVCRecordset@@@Z 5f7139a2 f   dbview.obj
 0001:00012a0e       ?DDX_FieldScroll@@YGXPAVCDataExchange@@HAAHPAVCRecordset@@@Z 5f713a0e f   dbview.obj
 0001:00012a7a       ?DDX_FieldCheck@@YGXPAVCDataExchange@@HAAHPAVCRecordset@@@Z 5f713a7a f   dbview.obj
 0001:00012be7       ?DDX_FieldRadio@@YGXPAVCDataExchange@@HAAHPAVCRecordset@@@Z 5f713be7 f   dbview.obj
 0001:00012c82       ?AssertValid@CRecordView@@UBEXXZ 5f713c82 f   dbview.obj
 0001:00012c95       ?Dump@CRecordView@@UBEXAAVCDumpContext@@@Z 5f713c95 f   dbview.obj
 0001:00012cf7       ?OnMove@CRecordView@@IAEXHH@Z 5f713cf7 f   dbview.obj
 0001:00012d20       ??_ECRecordView@@UAEPAXI@Z 5f713d20 f i dbview.obj
 0001:00012d20       ??_GCRecordView@@UAEPAXI@Z 5f713d20 f i dbview.obj
 0001:00012d50       ??1CFormView@@UAE@XZ       5f713d50 f i dbview.obj
 0001:00012d70       ??_9@$BBBE@AE              5f713d70 f i dbview.obj
 0001:00012d80       ?RFX_Single@@YGXPAVCFieldExchange@@PBGAAM@Z 5f713d80 f   dbflt.obj
 0001:0001302c       ?RFX_Double@@YGXPAVCFieldExchange@@PBGAAN@Z 5f71402c f   dbflt.obj
 0001:00013314       ?RFX_Single_Bulk@@YGXPAVCFieldExchange@@PBGPAPAMPAPAJ@Z 5f714314 f   dbflt.obj
 0001:0001348d       ?RFX_Double_Bulk@@YGXPAVCFieldExchange@@PBGPAPANPAPAJ@Z 5f71448d f   dbflt.obj
 0001:00013606       ?DDX_FieldText@@YGXPAVCDataExchange@@HAAMPAVCRecordset@@@Z 5f714606 f   dbflt.obj
 0001:00013644       ?DDX_FieldText@@YGXPAVCDataExchange@@HAANPAVCRecordset@@@Z 5f714644 f   dbflt.obj
 0001:00013690       ??0CLongBinary@@QAE@XZ     5f714690 f   dblong.obj
 0001:000136b9       ??1CLongBinary@@UAE@XZ     5f7146b9 f   dblong.obj
 0001:000136f5       ?AssertValid@CLongBinary@@UBEXXZ 5f7146f5 f   dblong.obj
 0001:00013708       ?Dump@CLongBinary@@UBEXAAVCDumpContext@@@Z 5f714708 f   dblong.obj
 0001:00013770       ??_GCLongBinary@@UAEPAXI@Z 5f714770 f i dblong.obj
 0001:000137a0       ??0CDBVariant@@QAE@XZ      5f7147a0 f   dbvar.obj
 0001:000137c1       ?Clear@CDBVariant@@QAEXXZ  5f7147c1 f   dbvar.obj
 0001:00013865       ??1CDBVariant@@UAE@XZ      5f714865 f   dbvar.obj
 0001:00013890       ??_GCDBVariant@@UAEPAXI@Z  5f714890 f i dbvar.obj
 0001:00013890       ??_ECDBVariant@@UAEPAXI@Z  5f714890 f i dbvar.obj
 0001:000138c0       ??0_AFX_DAO_STATE@@QAE@XZ  5f7148c0 f   daocore.obj
 0001:0001392d       ??1_AFX_DAO_STATE@@UAE@XZ  5f71492d f   daocore.obj
 0001:000139f1       ?AfxDaoCheck@@YGXJPBD0HHH@Z 5f7149f1 f   daocore.obj
 0001:00013a78       ?AfxDaoTrace@@YGXJPBD0H@Z  5f714a78 f   daocore.obj
 0001:00013adc       ?Dump@CDaoErrorInfo@@UBEXAAVCDumpContext@@@Z 5f714adc f   daocore.obj
 0001:00013b92       ?Dump@CDaoWorkspaceInfo@@UBEXAAVCDumpContext@@@Z 5f714b92 f   daocore.obj
 0001:00013c13       ?Dump@CDaoDatabaseInfo@@UBEXAAVCDumpContext@@@Z 5f714c13 f   daocore.obj
 0001:00013d00       ?Dump@CDaoTableDefInfo@@UBEXAAVCDumpContext@@@Z 5f714d00 f   daocore.obj
 0001:00013e51       ?Dump@CDaoFieldInfo@@UBEXAAVCDumpContext@@@Z 5f714e51 f   daocore.obj
 0001:00013ff8       ?Dump@CDaoIndexFieldInfo@@UBEXAAVCDumpContext@@@Z 5f714ff8 f   daocore.obj
 0001:00014052       ??0CDaoIndexInfo@@QAE@XZ   5f715052 f   daocore.obj
 0001:00014091       ??1CDaoIndexInfo@@UAE@XZ   5f715091 f   daocore.obj
 0001:00014126       ?Dump@CDaoIndexInfo@@UBEXAAVCDumpContext@@@Z 5f715126 f   daocore.obj
 0001:00014290       ?Dump@CDaoRelationFieldInfo@@UBEXAAVCDumpContext@@@Z 5f715290 f   daocore.obj
 0001:000142e9       ??0CDaoRelationInfo@@QAE@XZ 5f7152e9 f   daocore.obj
 0001:0001436f       ??1CDaoRelationInfo@@UAE@XZ 5f71536f f   daocore.obj
 0001:00014422       ?Dump@CDaoRelationInfo@@UBEXAAVCDumpContext@@@Z 5f715422 f   daocore.obj
 0001:0001451e       ?Dump@CDaoQueryDefInfo@@UBEXAAVCDumpContext@@@Z 5f71551e f   daocore.obj
 0001:00014658       ?Dump@CDaoParameterInfo@@UBEXAAVCDumpContext@@@Z 5f715658 f   daocore.obj
 0001:00014721       ?_GetBaseClass@CDaoException@@KGPAUCRuntimeClass@@XZ 5f715721 f   daocore.obj
 0001:0001472b       ?GetRuntimeClass@CDaoException@@UBEPAUCRuntimeClass@@XZ 5f71572b f   daocore.obj
 0001:0001473b       ??0CDaoException@@QAE@XZ   5f71573b f   daocore.obj
 0001:00014778       ??1CDaoException@@UAE@XZ   5f715778 f   daocore.obj
 0001:00014842       ?GetErrorCount@CDaoException@@QAEFXZ 5f715842 f   daocore.obj
 0001:000148a5       ?GetErrorInfo@CDaoException@@QAEXH@Z 5f7158a5 f   daocore.obj
 0001:000149d6       ?GetErrorMessage@CDaoException@@UAEHPAGIPAI@Z 5f7159d6 f   daocore.obj
 0001:00014b15       ?InitErrorsCollection@CDaoException@@IAEXXZ 5f715b15 f   daocore.obj
 0001:00014b71       ?FillErrorInfo@CDaoException@@IAEXXZ 5f715b71 f   daocore.obj
 0001:00014d92       ?AfxThrowDaoException@@YGXHJ@Z 5f715d92 f   daocore.obj
 0001:00014f34       ?_GetBaseClass@CDaoWorkspace@@KGPAUCRuntimeClass@@XZ 5f715f34 f   daocore.obj
 0001:00014f3e       ?GetRuntimeClass@CDaoWorkspace@@UBEPAUCRuntimeClass@@XZ 5f715f3e f   daocore.obj
 0001:00014f4e       ??0CDaoWorkspace@@QAE@XZ   5f715f4e f   daocore.obj
 0001:00014fe3       ??1CDaoWorkspace@@UAE@XZ   5f715fe3 f   daocore.obj
 0001:00015082       ?Create@CDaoWorkspace@@UAEXPBG00@Z 5f716082 f   daocore.obj
 0001:00015200       ?Append@CDaoWorkspace@@UAEXXZ 5f716200 f   daocore.obj
 0001:00015377       ?Open@CDaoWorkspace@@UAEXPBG@Z 5f716377 f   daocore.obj
 0001:00015561       ?Close@CDaoWorkspace@@UAEXXZ 5f716561 f   daocore.obj
 0001:000156a3       ?GetVersion@CDaoWorkspace@@SG?AVCString@@XZ 5f7166a3 f   daocore.obj
 0001:00015752       ?GetIniPath@CDaoWorkspace@@SG?AVCString@@XZ 5f716752 f   daocore.obj
 0001:00015801       ?SetIniPath@CDaoWorkspace@@SGXPBG@Z 5f716801 f   daocore.obj
 0001:00015895       ?SetDefaultUser@CDaoWorkspace@@SGXPBG@Z 5f716895 f   daocore.obj
 0001:00015929       ?SetDefaultPassword@CDaoWorkspace@@SGXPBG@Z 5f716929 f   daocore.obj
 0001:000159bd       ?GetLoginTimeout@CDaoWorkspace@@SGFXZ 5f7169bd f   daocore.obj
 0001:00015a10       ?SetLoginTimeout@CDaoWorkspace@@SGXF@Z 5f716a10 f   daocore.obj
 0001:00015a60       ?GetName@CDaoWorkspace@@QAE?AVCString@@XZ 5f716a60 f   daocore.obj
 0001:00015b39       ?GetUserNameW@CDaoWorkspace@@QAE?AVCString@@XZ 5f716b39 f   daocore.obj
 0001:00015c12       ?SetIsolateODBCTrans@CDaoWorkspace@@QAEXH@Z 5f716c12 f   daocore.obj
 0001:00015c8e       ?GetIsolateODBCTrans@CDaoWorkspace@@QAEHXZ 5f716c8e f   daocore.obj
 0001:00015d12       ?CompactDatabase@CDaoWorkspace@@SGXPBG00H0@Z 5f716d12 f   daocore.obj
 0001:00015f5f       ?CompactDatabase@CDaoWorkspace@@SGXPBG00H@Z 5f716f5f f   daocore.obj
 0001:00015f7d       ?RepairDatabase@CDaoWorkspace@@SGXPBG@Z 5f716f7d f   daocore.obj
 0001:00016011       ?Idle@CDaoWorkspace@@SGXH@Z 5f717011 f   daocore.obj
 0001:000160e0       ?GetWorkspaceCount@CDaoWorkspace@@QAEFXZ 5f7170e0 f   daocore.obj
 0001:00016144       ?GetWorkspaceInfo@CDaoWorkspace@@QAEXHAAUCDaoWorkspaceInfo@@K@Z 5f717144 f   daocore.obj
 0001:00016248       ?GetWorkspaceInfo@CDaoWorkspace@@QAEXPBGAAUCDaoWorkspaceInfo@@K@Z 5f717248 f   daocore.obj
 0001:0001634c       ?GetDatabaseCount@CDaoWorkspace@@QAEFXZ 5f71734c f   daocore.obj
 0001:000163b0       ?GetDatabaseInfo@CDaoWorkspace@@QAEXHAAUCDaoDatabaseInfo@@K@Z 5f7173b0 f   daocore.obj
 0001:000164b4       ?GetDatabaseInfo@CDaoWorkspace@@QAEXPBGAAUCDaoDatabaseInfo@@K@Z 5f7174b4 f   daocore.obj
 0001:000165b8       ?BeginTrans@CDaoWorkspace@@QAEXXZ 5f7175b8 f   daocore.obj
 0001:00016650       ?CommitTrans@CDaoWorkspace@@QAEXXZ 5f717650 f   daocore.obj
 0001:0001677d       ?Rollback@CDaoWorkspace@@QAEXXZ 5f71777d f   daocore.obj
 0001:00016815       ?InitializeEngine@CDaoWorkspace@@KAXXZ 5f717815 f   daocore.obj
 0001:0001681f       ?InitWorkspacesCollection@CDaoWorkspace@@IAEXXZ 5f71781f f   daocore.obj
 0001:00016887       ?FillWorkspaceInfo@CDaoWorkspace@@IAEXPAUDAOWorkspace@@AAUCDaoWorkspaceInfo@@K@Z 5f717887 f   daocore.obj
 0001:00016a11       ?InitDatabasesCollection@CDaoWorkspace@@IAEXXZ 5f717a11 f   daocore.obj
 0001:00016a61       ?FillDatabaseInfo@CDaoWorkspace@@IAEXPAUDAODatabase@@AAUCDaoDatabaseInfo@@K@Z 5f717a61 f   daocore.obj
 0001:00016ccc       ?ThrowDaoException@CDaoWorkspace@@MAEXH@Z 5f717ccc f   daocore.obj
 0001:00016cf7       ?AssertValid@CDaoWorkspace@@UBEXXZ 5f717cf7 f   daocore.obj
 0001:00016d0a       ?Dump@CDaoWorkspace@@UBEXAAVCDumpContext@@@Z 5f717d0a f   daocore.obj
 0001:00016d94       ?_GetBaseClass@CDaoDatabase@@KGPAUCRuntimeClass@@XZ 5f717d94 f   daocore.obj
 0001:00016d9e       ?GetRuntimeClass@CDaoDatabase@@UBEPAUCRuntimeClass@@XZ 5f717d9e f   daocore.obj
 0001:00016dae       ??0CDaoDatabase@@QAE@PAVCDaoWorkspace@@@Z 5f717dae f   daocore.obj
 0001:00016e7a       ??1CDaoDatabase@@UAE@XZ    5f717e7a f   daocore.obj
 0001:00016f65       ?Create@CDaoDatabase@@UAEXPBG0H@Z 5f717f65 f   daocore.obj
 0001:000170d9       ?Open@CDaoDatabase@@UAEXPBGHH0@Z 5f7180d9 f   daocore.obj
 0001:0001731a       ?Close@CDaoDatabase@@UAEXXZ 5f71831a f   daocore.obj
 0001:0001750c       ?CanUpdate@CDaoDatabase@@QAEHXZ 5f71850c f   daocore.obj
 0001:000175b6       ?CanTransact@CDaoDatabase@@QAEHXZ 5f7185b6 f   daocore.obj
 0001:00017660       ?GetName@CDaoDatabase@@QAE?AVCString@@XZ 5f718660 f   daocore.obj
 0001:0001775e       ?GetConnect@CDaoDatabase@@QAE?AVCString@@XZ 5f71875e f   daocore.obj
 0001:0001785c       ?GetVersion@CDaoDatabase@@QAE?AVCString@@XZ 5f71885c f   daocore.obj
 0001:0001795a       ?GetQueryTimeout@CDaoDatabase@@QAEFXZ 5f71895a f   daocore.obj
 0001:000179fc       ?SetQueryTimeout@CDaoDatabase@@QAEXF@Z 5f7189fc f   daocore.obj
 0001:00017a9b       ?GetRecordsAffected@CDaoDatabase@@QAEJXZ 5f718a9b f   daocore.obj
 0001:00017b3c       ?DeleteTableDef@CDaoDatabase@@QAEXPBG@Z 5f718b3c f   daocore.obj
 0001:00017c0d       ?DeleteQueryDef@CDaoDatabase@@QAEXPBG@Z 5f718c0d f   daocore.obj
 0001:00017cde       ?CreateRelation@CDaoDatabase@@QAEXPBG00J00@Z 5f718cde f   daocore.obj
 0001:00017db5       ?CreateRelation@CDaoDatabase@@QAEXAAUCDaoRelationInfo@@@Z 5f718db5 f   daocore.obj
 0001:000183c4       ?DeleteRelation@CDaoDatabase@@QAEXPBG@Z 5f7193c4 f   daocore.obj
 0001:00018495       ?Execute@CDaoDatabase@@QAEXPBGH@Z 5f719495 f   daocore.obj
 0001:000185af       ?GetTableDefCount@CDaoDatabase@@QAEFXZ 5f7195af f   daocore.obj
 0001:00018613       ?GetTableDefInfo@CDaoDatabase@@QAEXHAAUCDaoTableDefInfo@@K@Z 5f719613 f   daocore.obj
 0001:00018717       ?GetTableDefInfo@CDaoDatabase@@QAEXPBGAAUCDaoTableDefInfo@@K@Z 5f719717 f   daocore.obj
 0001:0001881b       ?GetRelationCount@CDaoDatabase@@QAEFXZ 5f71981b f   daocore.obj
 0001:0001887f       ?GetRelationInfo@CDaoDatabase@@QAEXHAAUCDaoRelationInfo@@K@Z 5f71987f f   daocore.obj
 0001:00018983       ?GetRelationInfo@CDaoDatabase@@QAEXPBGAAUCDaoRelationInfo@@K@Z 5f719983 f   daocore.obj
 0001:00018a87       ?GetQueryDefCount@CDaoDatabase@@QAEFXZ 5f719a87 f   daocore.obj
 0001:00018aeb       ?GetQueryDefInfo@CDaoDatabase@@QAEXHAAUCDaoQueryDefInfo@@K@Z 5f719aeb f   daocore.obj
 0001:00018bef       ?GetQueryDefInfo@CDaoDatabase@@QAEXPBGAAUCDaoQueryDefInfo@@K@Z 5f719bef f   daocore.obj
 0001:00018cf3       ?InitWorkspace@CDaoDatabase@@IAEXXZ 5f719cf3 f   daocore.obj
 0001:00018ddb       ?InitTableDefsCollection@CDaoDatabase@@IAEXXZ 5f719ddb f   daocore.obj
 0001:00018e2b       ?FillTableDefInfo@CDaoDatabase@@IAEXPAU_DAOTableDef@@AAUCDaoTableDefInfo@@K@Z 5f719e2b f   daocore.obj
 0001:00019157       ?InitRelationsCollection@CDaoDatabase@@IAEXXZ 5f71a157 f   daocore.obj
 0001:000191a7       ?FillRelationInfo@CDaoDatabase@@IAEXPAU_DAORelation@@AAUCDaoRelationInfo@@K@Z 5f71a1a7 f   daocore.obj
 0001:000196fc       ?InitQueryDefsCollection@CDaoDatabase@@IAEXXZ 5f71a6fc f   daocore.obj
 0001:0001974c       ?FillQueryDefInfo@CDaoDatabase@@IAEXPAU_DAOQueryDef@@AAUCDaoQueryDefInfo@@K@Z 5f71a74c f   daocore.obj
 0001:00019a0c       ?ThrowDaoException@CDaoDatabase@@MAEXH@Z 5f71aa0c f   daocore.obj
 0001:00019a37       ?AssertValid@CDaoDatabase@@UBEXXZ 5f71aa37 f   daocore.obj
 0001:00019a4a       ?Dump@CDaoDatabase@@UBEXAAVCDumpContext@@@Z 5f71aa4a f   daocore.obj
 0001:00019ab9       ?_GetBaseClass@CDaoTableDef@@KGPAUCRuntimeClass@@XZ 5f71aab9 f   daocore.obj
 0001:00019ac3       ?GetRuntimeClass@CDaoTableDef@@UBEPAUCRuntimeClass@@XZ 5f71aac3 f   daocore.obj
 0001:00019ad3       ??0CDaoTableDef@@QAE@PAVCDaoDatabase@@@Z 5f71aad3 f   daocore.obj
 0001:00019b2f       ??1CDaoTableDef@@UAE@XZ    5f71ab2f f   daocore.obj
 0001:00019ba9       ?Create@CDaoTableDef@@UAEXPBGJ00@Z 5f71aba9 f   daocore.obj
 0001:00019e3f       ?Append@CDaoTableDef@@UAEXXZ 5f71ae3f f   daocore.obj
 0001:00019fa7       ?Open@CDaoTableDef@@UAEXPBG@Z 5f71afa7 f   daocore.obj
 0001:0001a19b       ?Close@CDaoTableDef@@UAEXXZ 5f71b19b f   daocore.obj
 0001:0001a24e       ?CanUpdate@CDaoTableDef@@QAEHXZ 5f71b24e f   daocore.obj
 0001:0001a2f8       ?SetName@CDaoTableDef@@QAEXPBG@Z 5f71b2f8 f   daocore.obj
 0001:0001a3e4       ?GetName@CDaoTableDef@@QAE?AVCString@@XZ 5f71b3e4 f   daocore.obj
 0001:0001a4e2       ?SetSourceTableName@CDaoTableDef@@QAEXPBG@Z 5f71b4e2 f   daocore.obj
 0001:0001a5ce       ?GetSourceTableName@CDaoTableDef@@QAE?AVCString@@XZ 5f71b5ce f   daocore.obj
 0001:0001a6cc       ?SetConnect@CDaoTableDef@@QAEXPBG@Z 5f71b6cc f   daocore.obj
 0001:0001a7b8       ?GetConnect@CDaoTableDef@@QAE?AVCString@@XZ 5f71b7b8 f   daocore.obj
 0001:0001a8b6       ?SetAttributes@CDaoTableDef@@QAEXJ@Z 5f71b8b6 f   daocore.obj
 0001:0001a95d       ?GetAttributes@CDaoTableDef@@QAEJXZ 5f71b95d f   daocore.obj
 0001:0001a9fe       ?GetDateCreated@CDaoTableDef@@QAE?AVCOleDateTime@@XZ 5f71b9fe f   daocore.obj
 0001:0001aaee       ?GetDateLastUpdated@CDaoTableDef@@QAE?AVCOleDateTime@@XZ 5f71baee f   daocore.obj
 0001:0001abde       ?SetValidationRule@CDaoTableDef@@QAEXPBG@Z 5f71bbde f   daocore.obj
 0001:0001acca       ?GetValidationRule@CDaoTableDef@@QAE?AVCString@@XZ 5f71bcca f   daocore.obj
 0001:0001adc8       ?SetValidationText@CDaoTableDef@@QAEXPBG@Z 5f71bdc8 f   daocore.obj
 0001:0001aeb4       ?GetValidationText@CDaoTableDef@@QAE?AVCString@@XZ 5f71beb4 f   daocore.obj
 0001:0001afb2       ?GetRecordCount@CDaoTableDef@@QAEJXZ 5f71bfb2 f   daocore.obj
 0001:0001b053       ?CreateField@CDaoTableDef@@QAEXPBGFJJ@Z 5f71c053 f   daocore.obj
 0001:0001b0f9       ?CreateField@CDaoTableDef@@QAEXAAUCDaoFieldInfo@@@Z 5f71c0f9 f   daocore.obj
 0001:0001b379       ?DeleteField@CDaoTableDef@@QAEXPBG@Z 5f71c379 f   daocore.obj
 0001:0001b444       ?DeleteField@CDaoTableDef@@QAEXH@Z 5f71c444 f   daocore.obj
 0001:0001b4c6       ?CreateIndex@CDaoTableDef@@QAEXAAUCDaoIndexInfo@@@Z 5f71c4c6 f   daocore.obj
 0001:0001b65e       ?DeleteIndex@CDaoTableDef@@QAEXPBG@Z 5f71c65e f   daocore.obj
 0001:0001b729       ?DeleteIndex@CDaoTableDef@@QAEXH@Z 5f71c729 f   daocore.obj
 0001:0001b7ab       ?GetFieldCount@CDaoTableDef@@QAEFXZ 5f71c7ab f   daocore.obj
 0001:0001b80f       ?GetFieldInfo@CDaoTableDef@@QAEXHAAUCDaoFieldInfo@@K@Z 5f71c80f f   daocore.obj
 0001:0001b913       ?GetFieldInfo@CDaoTableDef@@QAEXPBGAAUCDaoFieldInfo@@K@Z 5f71c913 f   daocore.obj
 0001:0001ba17       ?GetIndexCount@CDaoTableDef@@QAEFXZ 5f71ca17 f   daocore.obj
 0001:0001ba7b       ?GetIndexInfo@CDaoTableDef@@QAEXHAAUCDaoIndexInfo@@K@Z 5f71ca7b f   daocore.obj
 0001:0001bb7f       ?GetIndexInfo@CDaoTableDef@@QAEXPBGAAUCDaoIndexInfo@@K@Z 5f71cb7f f   daocore.obj
 0001:0001bc83       ?RefreshLink@CDaoTableDef@@QAEXXZ 5f71cc83 f   daocore.obj
 0001:0001bd1b       ?InitFieldsCollection@CDaoTableDef@@IAEXXZ 5f71cd1b f   daocore.obj
 0001:0001bd6b       ?InitIndexesCollection@CDaoTableDef@@IAEXXZ 5f71cd6b f   daocore.obj
 0001:0001bdbb       ?ThrowDaoException@CDaoTableDef@@MAEXH@Z 5f71cdbb f   daocore.obj
 0001:0001bde6       ?AssertValid@CDaoTableDef@@UBEXXZ 5f71cde6 f   daocore.obj
 0001:0001bdf9       ?Dump@CDaoTableDef@@UBEXAAVCDumpContext@@@Z 5f71cdf9 f   daocore.obj
 0001:0001be68       ?_GetBaseClass@CDaoQueryDef@@KGPAUCRuntimeClass@@XZ 5f71ce68 f   daocore.obj
 0001:0001be72       ?GetRuntimeClass@CDaoQueryDef@@UBEPAUCRuntimeClass@@XZ 5f71ce72 f   daocore.obj
 0001:0001be82       ??0CDaoQueryDef@@QAE@PAVCDaoDatabase@@@Z 5f71ce82 f   daocore.obj
 0001:0001bede       ??1CDaoQueryDef@@UAE@XZ    5f71cede f   daocore.obj
 0001:0001bf58       ?Create@CDaoQueryDef@@UAEXPBG0@Z 5f71cf58 f   daocore.obj
 0001:0001c1af       ?Append@CDaoQueryDef@@UAEXXZ 5f71d1af f   daocore.obj
 0001:0001c317       ?Open@CDaoQueryDef@@UAEXPBG@Z 5f71d317 f   daocore.obj
 0001:0001c50b       ?Close@CDaoQueryDef@@UAEXXZ 5f71d50b f   daocore.obj
 0001:0001c5e5       ?CanUpdate@CDaoQueryDef@@QAEHXZ 5f71d5e5 f   daocore.obj
 0001:0001c66e       ?GetName@CDaoQueryDef@@QAE?AVCString@@XZ 5f71d66e f   daocore.obj
 0001:0001c74a       ?SetName@CDaoQueryDef@@QAEXPBG@Z 5f71d74a f   daocore.obj
 0001:0001c813       ?GetSQL@CDaoQueryDef@@QAE?AVCString@@XZ 5f71d813 f   daocore.obj
 0001:0001c8ef       ?SetSQL@CDaoQueryDef@@QAEXPBG@Z 5f71d8ef f   daocore.obj
 0001:0001c9b8       ?GetType@CDaoQueryDef@@QAEFXZ 5f71d9b8 f   daocore.obj
 0001:0001ca37       ?GetDateCreated@CDaoQueryDef@@QAE?AVCOleDateTime@@XZ 5f71da37 f   daocore.obj
 0001:0001cb04       ?GetDateLastUpdated@CDaoQueryDef@@QAE?AVCOleDateTime@@XZ 5f71db04 f   daocore.obj
 0001:0001cbd1       ?GetConnect@CDaoQueryDef@@QAE?AVCString@@XZ 5f71dbd1 f   daocore.obj
 0001:0001ccad       ?SetConnect@CDaoQueryDef@@QAEXPBG@Z 5f71dcad f   daocore.obj
 0001:0001cd76       ?GetODBCTimeout@CDaoQueryDef@@QAEFXZ 5f71dd76 f   daocore.obj
 0001:0001cdf5       ?SetODBCTimeout@CDaoQueryDef@@QAEXF@Z 5f71ddf5 f   daocore.obj
 0001:0001ce7a       ?GetReturnsRecords@CDaoQueryDef@@QAEHXZ 5f71de7a f   daocore.obj
 0001:0001cf03       ?SetReturnsRecords@CDaoQueryDef@@QAEXH@Z 5f71df03 f   daocore.obj
 0001:0001cf8b       ?GetRecordsAffected@CDaoQueryDef@@QAEJXZ 5f71df8b f   daocore.obj
 0001:0001d009       ?Execute@CDaoQueryDef@@UAEXH@Z 5f71e009 f   daocore.obj
 0001:0001d101       ?GetParamValue@CDaoQueryDef@@UAE?AVCOleVariant@@PBG@Z 5f71e101 f   daocore.obj
 0001:0001d309       ?GetParamValue@CDaoQueryDef@@UAE?AVCOleVariant@@H@Z 5f71e309 f   daocore.obj
 0001:0001d511       ?SetParamValue@CDaoQueryDef@@UAEXPBGABVCOleVariant@@@Z 5f71e511 f   daocore.obj
 0001:0001d71d       ?SetParamValue@CDaoQueryDef@@UAEXHABVCOleVariant@@@Z 5f71e71d f   daocore.obj
 0001:0001d929       ?SetParamValueNull@CDaoQueryDef@@QAEXPBG@Z 5f71e929 f   daocore.obj
 0001:0001d9a0       ?SetParamValueNull@CDaoQueryDef@@QAEXH@Z 5f71e9a0 f   daocore.obj
 0001:0001da17       ?GetFieldCount@CDaoQueryDef@@QAEFXZ 5f71ea17 f   daocore.obj
 0001:0001da7b       ?GetFieldInfo@CDaoQueryDef@@QAEXHAAUCDaoFieldInfo@@K@Z 5f71ea7b f   daocore.obj
 0001:0001db7f       ?GetFieldInfo@CDaoQueryDef@@QAEXPBGAAUCDaoFieldInfo@@K@Z 5f71eb7f f   daocore.obj
 0001:0001dc83       ?GetParameterCount@CDaoQueryDef@@QAEFXZ 5f71ec83 f   daocore.obj
 0001:0001dce7       ?GetParameterInfo@CDaoQueryDef@@QAEXHAAUCDaoParameterInfo@@K@Z 5f71ece7 f   daocore.obj
 0001:0001ddeb       ?GetParameterInfo@CDaoQueryDef@@QAEXPBGAAUCDaoParameterInfo@@K@Z 5f71edeb f   daocore.obj
 0001:0001deef       ?InitFieldsCollection@CDaoQueryDef@@IAEXXZ 5f71eeef f   daocore.obj
 0001:0001df3f       ?InitParametersCollection@CDaoQueryDef@@IAEXXZ 5f71ef3f f   daocore.obj
 0001:0001df8f       ?FillParameterInfo@CDaoQueryDef@@IAEXPAUDAOParameter@@AAUCDaoParameterInfo@@K@Z 5f71ef8f f   daocore.obj
 0001:0001e14d       ?ThrowDaoException@CDaoQueryDef@@MAEXH@Z 5f71f14d f   daocore.obj
 0001:0001e178       ?AssertValid@CDaoQueryDef@@UBEXXZ 5f71f178 f   daocore.obj
 0001:0001e18b       ?Dump@CDaoQueryDef@@UBEXAAVCDumpContext@@@Z 5f71f18b f   daocore.obj
 0001:0001e1fa       ?_GetBaseClass@CDaoRecordset@@KGPAUCRuntimeClass@@XZ 5f71f1fa f   daocore.obj
 0001:0001e204       ?GetRuntimeClass@CDaoRecordset@@UBEPAUCRuntimeClass@@XZ 5f71f204 f   daocore.obj
 0001:0001e214       ??0CDaoRecordset@@QAE@PAVCDaoDatabase@@@Z 5f71f214 f   daocore.obj
 0001:0001e381       ??1CDaoRecordset@@UAE@XZ   5f71f381 f   daocore.obj
 0001:0001e4a2       ?Open@CDaoRecordset@@UAEXHPBGH@Z 5f71f4a2 f   daocore.obj
 0001:0001eeac       ?Open@CDaoRecordset@@UAEXPAVCDaoQueryDef@@HH@Z 5f71feac f   daocore.obj
 0001:0001f196       ?Open@CDaoRecordset@@UAEXPAVCDaoTableDef@@HH@Z 5f720196 f   daocore.obj
 0001:0001f432       ?Close@CDaoRecordset@@UAEXXZ 5f720432 f   daocore.obj
 0001:0001f729       ?Requery@CDaoRecordset@@UAEXXZ 5f720729 f   daocore.obj
 0001:0001f9ac       ?GetDefaultDBName@CDaoRecordset@@UAE?AVCString@@XZ 5f7209ac f   daocore.obj
 0001:0001f9ee       ?GetDefaultSQL@CDaoRecordset@@UAE?AVCString@@XZ 5f7209ee f   daocore.obj
 0001:0001fa30       ?DoFieldExchange@CDaoRecordset@@UAEXPAVCDaoFieldExchange@@@Z 5f720a30 f   daocore.obj
 0001:0001fa50       ?IsBOF@CDaoRecordset@@QBEHXZ 5f720a50 f   daocore.obj
 0001:0001fad9       ?IsEOF@CDaoRecordset@@QBEHXZ 5f720ad9 f   daocore.obj
 0001:0001fb62       ?IsDeleted@CDaoRecordset@@QBEHXZ 5f720b62 f   daocore.obj
 0001:0001fbb2       ?CanScroll@CDaoRecordset@@QBEHXZ 5f720bb2 f   daocore.obj
 0001:0001fc02       ?CanUpdate@CDaoRecordset@@QBEHXZ 5f720c02 f   daocore.obj
 0001:0001fc8b       ?CanAppend@CDaoRecordset@@QBEHXZ 5f720c8b f   daocore.obj
 0001:0001fcdb       ?CanRestart@CDaoRecordset@@QAEHXZ 5f720cdb f   daocore.obj
 0001:0001fd85       ?CanTransact@CDaoRecordset@@QAEHXZ 5f720d85 f   daocore.obj
 0001:0001fe0e       ?CanBookmark@CDaoRecordset@@QAEHXZ 5f720e0e f   daocore.obj
 0001:0001fe97       ?GetName@CDaoRecordset@@QAE?AVCString@@XZ 5f720e97 f   daocore.obj
 0001:0001ff95       ?GetType@CDaoRecordset@@QAEFXZ 5f720f95 f   daocore.obj
 0001:00020037       ?GetEditMode@CDaoRecordset@@QAEFXZ 5f721037 f   daocore.obj
 0001:000200dc       ?GetSQL@CDaoRecordset@@QBE?AVCString@@XZ 5f7210dc f   daocore.obj
 0001:0002016f       ?GetDateCreated@CDaoRecordset@@QAE?AVCOleDateTime@@XZ 5f72116f f   daocore.obj
 0001:0002025f       ?GetDateLastUpdated@CDaoRecordset@@QAE?AVCOleDateTime@@XZ 5f72125f f   daocore.obj
 0001:0002034f       ?GetLastModifiedBookmark@CDaoRecordset@@QAE?AVCOleVariant@@XZ 5f72134f f   daocore.obj
 0001:0002044d       ?GetValidationRule@CDaoRecordset@@QAE?AVCString@@XZ 5f72144d f   daocore.obj
 0001:0002054e       ?GetValidationText@CDaoRecordset@@QAE?AVCString@@XZ 5f72154e f   daocore.obj
 0001:0002064c       ?GetCurrentIndex@CDaoRecordset@@QAE?AVCString@@XZ 5f72164c f   daocore.obj
 0001:0002074a       ?SetCurrentIndex@CDaoRecordset@@QAEXPBG@Z 5f72174a f   daocore.obj
 0001:00020835       ?GetRecordCount@CDaoRecordset@@QAEJXZ 5f721835 f   daocore.obj
 0001:000208d6       ?SetFieldDirty@CDaoRecordset@@QAEXPAXH@Z 5f7218d6 f   daocore.obj
 0001:000209b2       ?IsFieldDirty@CDaoRecordset@@QAEHPAX@Z 5f7219b2 f   daocore.obj
 0001:00020aaa       ?SetFieldNull@CDaoRecordset@@QAEXPAXH@Z 5f721aaa f   daocore.obj
 0001:00020bc2       ?IsFieldNull@CDaoRecordset@@QAEHPAX@Z 5f721bc2 f   daocore.obj
 0001:00020ca5       ?IsFieldNullable@CDaoRecordset@@QAEHPAX@Z 5f721ca5 f   daocore.obj
 0001:00020e18       ?GetFieldCount@CDaoRecordset@@QAEFXZ 5f721e18 f   daocore.obj
 0001:00020e7c       ?GetFieldInfo@CDaoRecordset@@QAEXHAAUCDaoFieldInfo@@K@Z 5f721e7c f   daocore.obj
 0001:00020f80       ?GetFieldInfo@CDaoRecordset@@QAEXPBGAAUCDaoFieldInfo@@K@Z 5f721f80 f   daocore.obj
 0001:00021084       ?GetIndexCount@CDaoRecordset@@QAEFXZ 5f722084 f   daocore.obj
 0001:000210e8       ?GetIndexInfo@CDaoRecordset@@QAEXHAAUCDaoIndexInfo@@K@Z 5f7220e8 f   daocore.obj
 0001:000211ec       ?GetIndexInfo@CDaoRecordset@@QAEXPBGAAUCDaoIndexInfo@@K@Z 5f7221ec f   daocore.obj
 0001:000212f0       ?GetBookmark@CDaoRecordset@@QAE?AVCOleVariant@@XZ 5f7222f0 f   daocore.obj
 0001:000213ee       ?SetBookmark@CDaoRecordset@@QAEXVCOleVariant@@@Z 5f7223ee f   daocore.obj
 0001:000214c9       ?GetAbsolutePosition@CDaoRecordset@@QAEJXZ 5f7224c9 f   daocore.obj
 0001:0002156d       ?SetAbsolutePosition@CDaoRecordset@@QAEXJ@Z 5f72256d f   daocore.obj
 0001:00021616       ?GetPercentPosition@CDaoRecordset@@QAEMXZ 5f722616 f   daocore.obj
 0001:000216ba       ?SetPercentPosition@CDaoRecordset@@QAEXM@Z 5f7226ba f   daocore.obj
 0001:00021763       ?MoveNext@CDaoRecordset@@QAEXXZ 5f722763 f   daocore.obj
 0001:0002178e       ?MovePrev@CDaoRecordset@@QAEXXZ 5f72278e f   daocore.obj
 0001:000217b9       ?MoveFirst@CDaoRecordset@@QAEXXZ 5f7227b9 f   daocore.obj
 0001:000217e7       ?MoveLast@CDaoRecordset@@QAEXXZ 5f7227e7 f   daocore.obj
 0001:00021815       ?Move@CDaoRecordset@@UAEXJ@Z 5f722815 f   daocore.obj
 0001:00021a44       ?FindNext@CDaoRecordset@@QAEHPBG@Z 5f722a44 f   daocore.obj
 0001:00021a75       ?FindPrev@CDaoRecordset@@QAEHPBG@Z 5f722a75 f   daocore.obj
 0001:00021aa6       ?FindFirst@CDaoRecordset@@QAEHPBG@Z 5f722aa6 f   daocore.obj
 0001:00021ada       ?FindLast@CDaoRecordset@@QAEHPBG@Z 5f722ada f   daocore.obj
 0001:00021b0e       ?Find@CDaoRecordset@@UAEHJPBG@Z 5f722b0e f   daocore.obj
 0001:00021d0c       ?Seek@CDaoRecordset@@QAEHPBGPAVCOleVariant@@11@Z 5f722d0c f   daocore.obj
 0001:000220bd       ?Seek@CDaoRecordset@@QAEHPBGPAVCOleVariant@@G@Z 5f7230bd f   daocore.obj
 0001:00022436       ?CancelUpdate@CDaoRecordset@@UAEXXZ 5f723436 f   daocore.obj
 0001:000224eb       ?SetLockingMode@CDaoRecordset@@QAEXH@Z 5f7234eb f   daocore.obj
 0001:0002258d       ?GetLockingMode@CDaoRecordset@@QAEHXZ 5f72358d f   daocore.obj
 0001:00022637       ?SetCacheStart@CDaoRecordset@@QAEXVCOleVariant@@@Z 5f723637 f   daocore.obj
 0001:0002270d       ?GetCacheStart@CDaoRecordset@@QAE?AVCOleVariant@@XZ 5f72370d f   daocore.obj
 0001:0002280e       ?SetCacheSize@CDaoRecordset@@QAEXJ@Z 5f72380e f   daocore.obj
 0001:000228af       ?GetCacheSize@CDaoRecordset@@QAEJXZ 5f7238af f   daocore.obj
 0001:00022953       ?FillCache@CDaoRecordset@@QAEXPAJPAVCOleVariant@@@Z 5f723953 f   daocore.obj
 0001:00022af8       ?AddNew@CDaoRecordset@@UAEXXZ 5f723af8 f   daocore.obj
 0001:00022bed       ?Edit@CDaoRecordset@@UAEXXZ 5f723bed f   daocore.obj
 0001:00022cdf       ?Update@CDaoRecordset@@UAEXXZ 5f723cdf f   daocore.obj
 0001:00022dd8       ?Delete@CDaoRecordset@@UAEXXZ 5f723dd8 f   daocore.obj
 0001:00022ea7       ?GetFieldValue@CDaoRecordset@@UAE?AVCOleVariant@@PBG@Z 5f723ea7 f   daocore.obj
 0001:00022f22       ?GetFieldValue@CDaoRecordset@@UAE?AVCOleVariant@@H@Z 5f723f22 f   daocore.obj
 0001:00022f9d       ?GetFieldValue@CDaoRecordset@@UAEXPBGAAVCOleVariant@@@Z 5f723f9d f   daocore.obj
 0001:000230ca       ?GetFieldValue@CDaoRecordset@@UAEXHAAVCOleVariant@@@Z 5f7240ca f   daocore.obj
 0001:000231f7       ?SetFieldValue@CDaoRecordset@@UAEXPBGABVCOleVariant@@@Z 5f7241f7 f   daocore.obj
 0001:0002334e       ?SetFieldValue@CDaoRecordset@@UAEXHABVCOleVariant@@@Z 5f72434e f   daocore.obj
 0001:000234a5       ?SetFieldValue@CDaoRecordset@@QAEXHPBG@Z 5f7244a5 f   daocore.obj
 0001:0002350a       ?SetFieldValue@CDaoRecordset@@QAEXPBG0@Z 5f72450a f   daocore.obj
 0001:0002356f       ?SetFieldValueNull@CDaoRecordset@@QAEXPBG@Z 5f72456f f   daocore.obj
 0001:000235e6       ?SetFieldValueNull@CDaoRecordset@@QAEXH@Z 5f7245e6 f   daocore.obj
 0001:0002365d       ?GetParamValue@CDaoRecordset@@UAE?AVCOleVariant@@PBG@Z 5f72465d f   daocore.obj
 0001:000236f9       ?GetParamValue@CDaoRecordset@@UAE?AVCOleVariant@@H@Z 5f7246f9 f   daocore.obj
 0001:00023795       ?SetParamValue@CDaoRecordset@@UAEXPBGABVCOleVariant@@@Z 5f724795 f   daocore.obj
 0001:0002381d       ?SetParamValue@CDaoRecordset@@UAEXHABVCOleVariant@@@Z 5f72481d f   daocore.obj
 0001:000238a5       ?SetParamValueNull@CDaoRecordset@@QAEXPBG@Z 5f7248a5 f   daocore.obj
 0001:0002391c       ?SetParamValueNull@CDaoRecordset@@QAEXH@Z 5f72491c f   daocore.obj
 0001:00023993       ?GetFieldLength@CDaoRecordset@@QAEKH@Z 5f724993 f   daocore.obj
 0001:000239eb       ?InitFieldsCollection@CDaoRecordset@@IAEXXZ 5f7249eb f   daocore.obj
 0001:00023a6a       ?InitIndexesCollection@CDaoRecordset@@IAEXXZ 5f724a6a f   daocore.obj
 0001:00023aec       ?BuildSQL@CDaoRecordset@@IAEXXZ 5f724aec f   daocore.obj
 0001:00023c10       ?AllocDatabase@CDaoRecordset@@IAEXXZ 5f724c10 f   daocore.obj
 0001:00023d26       ?BuildSelectList@CDaoRecordset@@IAEXXZ 5f724d26 f   daocore.obj
 0001:00023d9e       ?BuildParameterList@CDaoRecordset@@IAEXXZ 5f724d9e f   daocore.obj
 0001:00023e39       ?BindFields@CDaoRecordset@@IAEXXZ 5f724e39 f   daocore.obj
 0001:0002401e       ?BindParameters@CDaoRecordset@@IAEXXZ 5f72501e f   daocore.obj
 0001:0002409c       ?Fixup@CDaoRecordset@@IAEXXZ 5f72509c f   daocore.obj
 0001:000240db       ?AllocCache@CDaoRecordset@@IAEXXZ 5f7250db f   daocore.obj
 0001:000241a1       ?StoreFields@CDaoRecordset@@IAEXXZ 5f7251a1 f   daocore.obj
 0001:0002421b       ?LoadFields@CDaoRecordset@@IAEXXZ 5f72521b f   daocore.obj
 0001:00024278       ?FreeCache@CDaoRecordset@@IAEXXZ 5f725278 f   daocore.obj
 0001:00024351       ?MarkForAddNew@CDaoRecordset@@IAEXXZ 5f725351 f   daocore.obj
 0001:00024390       ?MarkForEdit@CDaoRecordset@@IAEXXZ 5f725390 f   daocore.obj
 0001:000243cf       ?GetFieldIndex@CDaoRecordset@@IAEHPAX@Z 5f7253cf f   daocore.obj
 0001:0002443c       ?SetDirtyFields@CDaoRecordset@@MAEXXZ 5f72543c f   daocore.obj
 0001:0002448c       ?SetCursorAttributes@CDaoRecordset@@QAEXXZ 5f72548c f   daocore.obj
 0001:0002450b       ?GetDataAndFixupNulls@CDaoRecordset@@QAEXXZ 5f72550b f   daocore.obj
 0001:00024610       ?IsFieldStatusDirty@CDaoRecordset@@QAEHI@Z 5f725610 f   daocore.obj
 0001:0002464b       ?SetDirtyFieldStatus@CDaoRecordset@@QAEXI@Z 5f72564b f   daocore.obj
 0001:00024686       ?ClearDirtyFieldStatus@CDaoRecordset@@QAEXI@Z 5f725686 f   daocore.obj
 0001:000246c1       ?IsFieldStatusNull@CDaoRecordset@@QAEHI@Z 5f7256c1 f   daocore.obj
 0001:000246fa       ?SetNullFieldStatus@CDaoRecordset@@QAEXI@Z 5f7256fa f   daocore.obj
 0001:00024735       ?ClearNullFieldStatus@CDaoRecordset@@QAEXI@Z 5f725735 f   daocore.obj
 0001:00024770       ?IsFieldStatusNullable@CDaoRecordset@@QAEHI@Z 5f725770 f   daocore.obj
 0001:000247a9       ?SetNullableFieldStatus@CDaoRecordset@@QAEXI@Z 5f7257a9 f   daocore.obj
 0001:000247e4       ?IsFieldStatusNullableKnown@CDaoRecordset@@QAEHI@Z 5f7257e4 f   daocore.obj
 0001:0002481d       ?SetNullableKnownFieldStatus@CDaoRecordset@@QAEXI@Z 5f72581d f   daocore.obj
 0001:00024858       ?ClearFieldStatusFlags@CDaoRecordset@@QAEXXZ 5f725858 f   daocore.obj
 0001:0002488e       ?IsMatch@CDaoRecordset@@QAEHXZ 5f72588e f   daocore.obj
 0001:00024912       ?StripBrackets@CDaoRecordset@@SAXPBGPAG@Z 5f725912 f   daocore.obj
 0001:000249af       ?ThrowDaoException@CDaoRecordset@@MAEXH@Z 5f7259af f   daocore.obj
 0001:000249da       ?AssertValid@CDaoRecordset@@UBEXXZ 5f7259da f   daocore.obj
 0001:000249ed       ?Dump@CDaoRecordset@@UBEXAAVCDumpContext@@@Z 5f7259ed f   daocore.obj
 0001:00024bfc       ?AfxGetFieldInfo@@YAXPAU_DAOField@@AAUCDaoFieldInfo@@K@Z 5f725bfc f   daocore.obj
 0001:00025032       ?AfxSetFieldInfo@@YAXPAU_DAOField@@AAUCDaoFieldInfo@@@Z 5f726032 f   daocore.obj
 0001:000252a5       ?AfxGetDefaultValue@@YAXPAU_DAOField@@AAVCString@@@Z 5f7262a5 f   daocore.obj
 0001:0002537f       ?AfxSetDefaultValue@@YAXPAU_DAOField@@AAVCString@@@Z 5f72637f f   daocore.obj
 0001:0002547a       ?AfxGetIndexInfo@@YAXPAU_DAOIndex@@AAUCDaoIndexInfo@@K@Z 5f72647a f   daocore.obj
 0001:0002570d       ?AfxSetIndexInfo@@YAXPAU_DAOIndex@@AAUCDaoIndexInfo@@@Z 5f72670d f   daocore.obj
 0001:00025838       ?AfxGetIndexFields@@YAXPAU_DAOIndex@@PAPAUDAOIndexFields@@@Z 5f726838 f   daocore.obj
 0001:0002593e       ?AfxGetIndexFieldInfo@@YAXPAU_DAOIndex@@AAUCDaoIndexInfo@@@Z 5f72693e f   daocore.obj
 0001:00025dce       ?AfxSetIndexFieldInfo@@YAXPAU_DAOIndex@@AAUCDaoIndexInfo@@@Z 5f726dce f   daocore.obj
 0001:0002602e       ?ThrowGetRowsDaoException@@YAXJ@Z 5f72702e f   daocore.obj
 0001:00026234       ?AfxGetDaoState@@YAPAV_AFX_DAO_STATE@@XZ 5f727234 f   daocore.obj
 0001:000262ce       ?AfxDaoInit@@YGXXZ         5f7272ce f   daocore.obj
 0001:0002655c       ?AfxDaoGetEngine@@YGPAU_DAODBEngine@@XZ 5f72755c f   daocore.obj
 0001:00026569       ?AfxDaoTerm@@YGXXZ         5f727569 f   daocore.obj
 0001:00026617       ?IsOpen@CDaoWorkspace@@QBEHXZ 5f727617 f   daocore.obj
 0001:00026638       ?IsNew@CDaoWorkspace@@QBEHXZ 5f727638 f   daocore.obj
 0001:00026659       ?IsOpen@CDaoDatabase@@QBEHXZ 5f727659 f   daocore.obj
 0001:0002667a       ?IsOpen@CDaoTableDef@@QBEHXZ 5f72767a f   daocore.obj
 0001:0002669b       ?IsOpen@CDaoQueryDef@@QBEHXZ 5f72769b f   daocore.obj
 0001:000266bc       ?IsOpen@CDaoRecordset@@QBEHXZ 5f7276bc f   daocore.obj
 0001:000266e0       ??_G_AFX_DAO_STATE@@UAEPAXI@Z 5f7276e0 f i daocore.obj
 0001:000266e0       ??_E_AFX_DAO_STATE@@UAEPAXI@Z 5f7276e0 f i daocore.obj
 0001:00026710       ??_GCDaoIndexInfo@@UAEPAXI@Z 5f727710 f i daocore.obj
 0001:00026710       ??_ECDaoIndexInfo@@UAEPAXI@Z 5f727710 f i daocore.obj
 0001:00026740       ??_ECDaoIndexFieldInfo@@QAEPAXI@Z 5f727740 f i daocore.obj
 0001:000267b0       ??1CDaoIndexFieldInfo@@QAE@XZ 5f7277b0 f i daocore.obj
 0001:000267d0       ??_ECDaoRelationInfo@@UAEPAXI@Z 5f7277d0 f i daocore.obj
 0001:000267d0       ??_GCDaoRelationInfo@@UAEPAXI@Z 5f7277d0 f i daocore.obj
 0001:00026800       ??_ECDaoRelationFieldInfo@@QAEPAXI@Z 5f727800 f i daocore.obj
 0001:00026870       ??1CDaoRelationFieldInfo@@QAE@XZ 5f727870 f i daocore.obj
 0001:000268c0       ??_GCDaoException@@UAEPAXI@Z 5f7278c0 f i daocore.obj
 0001:000268f0       ??_GCDaoErrorInfo@@QAEPAXI@Z 5f7278f0 f i daocore.obj
 0001:00026920       ??1CDaoErrorInfo@@QAE@XZ   5f727920 f i daocore.obj
 0001:00026980       ??0CDaoErrorInfo@@QAE@XZ   5f727980 f i daocore.obj
 0001:000269f0       ??_GCDaoWorkspace@@UAEPAXI@Z 5f7279f0 f i daocore.obj
 0001:00026a20       ??_GCDaoDatabase@@UAEPAXI@Z 5f727a20 f i daocore.obj
 0001:00026a50       ??0CDaoRelationFieldInfo@@QAE@XZ 5f727a50 f i daocore.obj
 0001:00026ab0       ??_ECDaoTableDef@@UAEPAXI@Z 5f727ab0 f i daocore.obj
 0001:00026ab0       ??_GCDaoTableDef@@UAEPAXI@Z 5f727ab0 f i daocore.obj
 0001:00026ae0       ??0CDaoFieldInfo@@QAE@XZ   5f727ae0 f i daocore.obj
 0001:00026b90       ??1CDaoFieldInfo@@QAE@XZ   5f727b90 f i daocore.obj
 0001:00026c30       ??_ECDaoQueryDef@@UAEPAXI@Z 5f727c30 f i daocore.obj
 0001:00026c30       ??_GCDaoQueryDef@@UAEPAXI@Z 5f727c30 f i daocore.obj
 0001:00026c60       ??_GCDaoRecordset@@UAEPAXI@Z 5f727c60 f i daocore.obj
 0001:00026c90       ??0CDaoIndexFieldInfo@@QAE@XZ 5f727c90 f i daocore.obj
 0001:00026cc0       ??_9@$BEM@AG               5f727cc0 f i daocore.obj
 0001:00026cd0       ??_9@$BHE@AG               5f727cd0 f i daocore.obj
 0001:00026ce0       ??_9@$BHI@AG               5f727ce0 f i daocore.obj
 0001:00026cf0       ??0CDaoFieldExchange@@QAE@IPAVCDaoRecordset@@PAX@Z 5f727cf0 f   daodfx.obj
 0001:00026d5b       ?IsValidOperation@CDaoFieldExchange@@QAEHXZ 5f727d5b f   daodfx.obj
 0001:00026dd9       ?AppendParamType@CDaoFieldExchange@@SGXAAVCString@@K@Z 5f727dd9 f   daodfx.obj
 0001:000270b3       ?GetCacheValue@CDaoFieldExchange@@SGPAUCDaoFieldCache@@PAVCDaoRecordset@@PAX@Z 5f7280b3 f   daodfx.obj
 0001:000270e3       ?SetNullValue@CDaoFieldExchange@@SGXPAXK@Z 5f7280e3 f   daodfx.obj
 0001:000271f3       ?IsNullValue@CDaoFieldExchange@@SGHPAXK@Z 5f7281f3 f   daodfx.obj
 0001:00027389       ?AllocCacheValue@CDaoFieldExchange@@SGXAAPAUCDaoFieldCache@@K@Z 5f728389 f   daodfx.obj
 0001:00027695       ?DeleteCacheValue@CDaoFieldExchange@@SGXPAUCDaoFieldCache@@K@Z 5f728695 f   daodfx.obj
 0001:0002780a       ?CopyValue@CDaoFieldExchange@@SGXPAX0K@Z 5f72880a f   daodfx.obj
 0001:000279a1       ?CompareValue@CDaoFieldExchange@@SGHPAX0K@Z 5f7289a1 f   daodfx.obj
 0001:00027bf7       ?FillVariant@CDaoFieldExchange@@SGXPAXKPAPAVCOleVariant@@@Z 5f728bf7 f   daodfx.obj
 0001:00027e3c       ?Default@CDaoFieldExchange@@QAEXPBGPAXKK@Z 5f728e3c f   daodfx.obj
 0001:00028764       ?DFX_Text@@YGXPAVCDaoFieldExchange@@PBGAAVCString@@HK@Z 5f729764 f   daodfx.obj
 0001:00028904       ?DFX_Binary@@YGXPAVCDaoFieldExchange@@PBGAAVCByteArray@@HK@Z 5f729904 f   daodfx.obj
 0001:00028a15       ?DFX_LongBinary@@YGXPAVCDaoFieldExchange@@PBGAAVCLongBinary@@KK@Z 5f729a15 f   daodfx.obj
 0001:00028b60       ?DFX_Bool@@YGXPAVCDaoFieldExchange@@PBGAAHK@Z 5f729b60 f   daodfx.obj
 0001:00028cbc       ?DFX_Byte@@YGXPAVCDaoFieldExchange@@PBGAAEK@Z 5f729cbc f   daodfx.obj
 0001:00028de2       ?DFX_Short@@YGXPAVCDaoFieldExchange@@PBGAAFK@Z 5f729de2 f   daodfx.obj
 0001:00028f09       ?DFX_Long@@YGXPAVCDaoFieldExchange@@PBGAAJK@Z 5f729f09 f   daodfx.obj
 0001:0002902f       ?DFX_Currency@@YGXPAVCDaoFieldExchange@@PBGAAVCOleCurrency@@K@Z 5f72a02f f   daodfx.obj
 0001:000291af       ?DFX_Single@@YGXPAVCDaoFieldExchange@@PBGAAMK@Z 5f72a1af f   daodfx.obj
 0001:000292d5       ?DFX_Double@@YGXPAVCDaoFieldExchange@@PBGAANK@Z 5f72a2d5 f   daodfx.obj
 0001:000293f6       ?DFX_DateTime@@YGXPAVCDaoFieldExchange@@PBGAAVCOleDateTime@@K@Z 5f72a3f6 f   daodfx.obj
 0001:00029576       _DaoStringAllocCallback@12 5f72a576 f   daodfx.obj
 0001:0002962f       _DaoBinaryAllocCallback@12 5f72a62f f   daodfx.obj
 0001:000296fb       _DaoLongBinaryAllocCallback@12 5f72a6fb f   daodfx.obj
 0001:000297f4       ?AllocLongBinary@@YAXAAVCLongBinary@@K@Z 5f72a7f4 f   daodfx.obj
 0001:0002987e       ?SetFieldType@CDaoFieldExchange@@QAEXI@Z 5f72a87e f   daodfx.obj
 0001:000298c0       ??_GCOleVariant@@QAEPAXI@Z 5f72a8c0 f i daodfx.obj
 0001:000298f0       ?_GetBaseClass@CDaoRecordView@@KGPAUCRuntimeClass@@XZ 5f72a8f0 f   daoview.obj
 0001:000298fa       ?GetRuntimeClass@CDaoRecordView@@UBEPAUCRuntimeClass@@XZ 5f72a8fa f   daoview.obj
 0001:0002990a       ?_GetBaseMessageMap@CDaoRecordView@@KGPBUAFX_MSGMAP@@XZ 5f72a90a f   daoview.obj
 0001:00029914       ?GetMessageMap@CDaoRecordView@@MBEPBUAFX_MSGMAP@@XZ 5f72a914 f   daoview.obj
 0001:00029924       ??0CDaoRecordView@@IAE@PBG@Z 5f72a924 f   daoview.obj
 0001:000299e8       ??0CDaoRecordView@@IAE@I@Z 5f72a9e8 f   daoview.obj
 0001:00029aac       ??1CDaoRecordView@@UAE@XZ  5f72aaac f   daoview.obj
 0001:00029b27       ?OnInitialUpdate@CDaoRecordView@@UAEXXZ 5f72ab27 f   daoview.obj
 0001:00029d02       ?OnMove@CDaoRecordView@@UAEHI@Z 5f72ad02 f   daoview.obj
 0001:0002a254       ?IsOnFirstRecord@CDaoRecordView@@QAEHXZ 5f72b254 f   daoview.obj
 0001:0002a28a       ?IsOnLastRecord@CDaoRecordView@@QAEHXZ 5f72b28a f   daoview.obj
 0001:0002a2c0       ?AfxFieldText@@YGHPAVCDataExchange@@HPAXPAVCDaoRecordset@@@Z 5f72b2c0 f   daoview.obj
 0001:0002a3ac       ?DDX_FieldText@@YGXPAVCDataExchange@@HAAHPAVCDaoRecordset@@@Z 5f72b3ac f   daoview.obj
 0001:0002a3dd       ?DDX_FieldText@@YGXPAVCDataExchange@@HAAEPAVCDaoRecordset@@@Z 5f72b3dd f   daoview.obj
 0001:0002a40e       ?DDX_FieldText@@YGXPAVCDataExchange@@HAAFPAVCDaoRecordset@@@Z 5f72b40e f   daoview.obj
 0001:0002a43f       ?DDX_FieldText@@YGXPAVCDataExchange@@HAAJPAVCDaoRecordset@@@Z 5f72b43f f   daoview.obj
 0001:0002a470       ?DDX_FieldText@@YGXPAVCDataExchange@@HAAKPAVCDaoRecordset@@@Z 5f72b470 f   daoview.obj
 0001:0002a4a1       ?DDX_FieldText@@YGXPAVCDataExchange@@HAAVCOleCurrency@@PAVCDaoRecordset@@@Z 5f72b4a1 f   daoview.obj
 0001:0002a4d2       ?DDX_FieldText@@YGXPAVCDataExchange@@HAAMPAVCDaoRecordset@@@Z 5f72b4d2 f   daoview.obj
 0001:0002a503       ?DDX_FieldText@@YGXPAVCDataExchange@@HAANPAVCDaoRecordset@@@Z 5f72b503 f   daoview.obj
 0001:0002a534       ?DDX_FieldText@@YGXPAVCDataExchange@@HAAVCOleDateTime@@PAVCDaoRecordset@@@Z 5f72b534 f   daoview.obj
 0001:0002a565       ?DDX_FieldText@@YGXPAVCDataExchange@@HAAVCString@@PAVCDaoRecordset@@@Z 5f72b565 f   daoview.obj
 0001:0002a596       ?DDX_FieldText@@YGXPAVCDataExchange@@HPAGHPAVCDaoRecordset@@@Z 5f72b596 f   daoview.obj
 0001:0002a5cb       ?DDX_FieldLBString@@YGXPAVCDataExchange@@HAAVCString@@PAVCDaoRecordset@@@Z 5f72b5cb f   daoview.obj
 0001:0002a725       ?DDX_FieldLBStringExact@@YGXPAVCDataExchange@@HAAVCString@@PAVCDaoRecordset@@@Z 5f72b725 f   daoview.obj
 0001:0002a7ef       ?DDX_FieldCBString@@YGXPAVCDataExchange@@HAAVCString@@PAVCDaoRecordset@@@Z 5f72b7ef f   daoview.obj
 0001:0002a93d       ?DDX_FieldCBStringExact@@YGXPAVCDataExchange@@HAAVCString@@PAVCDaoRecordset@@@Z 5f72b93d f   daoview.obj
 0001:0002aa07       ?DDX_FieldLBIndex@@YGXPAVCDataExchange@@HAAHPAVCDaoRecordset@@@Z 5f72ba07 f   daoview.obj
 0001:0002aa73       ?DDX_FieldCBIndex@@YGXPAVCDataExchange@@HAAHPAVCDaoRecordset@@@Z 5f72ba73 f   daoview.obj
 0001:0002aadf       ?DDX_FieldScroll@@YGXPAVCDataExchange@@HAAHPAVCDaoRecordset@@@Z 5f72badf f   daoview.obj
 0001:0002ab4b       ?DDX_FieldSlider@@YGXPAVCDataExchange@@HAAHPAVCDaoRecordset@@@Z 5f72bb4b f   daoview.obj
 0001:0002abb7       ?DDX_FieldCheck@@YGXPAVCDataExchange@@HAAHPAVCDaoRecordset@@@Z 5f72bbb7 f   daoview.obj
 0001:0002ad24       ?DDX_FieldRadio@@YGXPAVCDataExchange@@HAAHPAVCDaoRecordset@@@Z 5f72bd24 f   daoview.obj
 0001:0002adbf       ?AssertValid@CDaoRecordView@@UBEXXZ 5f72bdbf f   daoview.obj
 0001:0002add2       ?Dump@CDaoRecordView@@UBEXAAVCDumpContext@@@Z 5f72bdd2 f   daoview.obj
 0001:0002af13       ?OnUpdateRecordFirst@CDaoRecordView@@IAEXPAVCCmdUI@@@Z 5f72bf13 f   daoview.obj
 0001:0002af47       ?OnUpdateRecordNext@CDaoRecordView@@IAEXPAVCCmdUI@@@Z 5f72bf47 f   daoview.obj
 0001:0002af7b       ?OnUpdateRecordPrev@CDaoRecordView@@IAEXPAVCCmdUI@@@Z 5f72bf7b f   daoview.obj
 0001:0002afaf       ?OnUpdateRecordLast@CDaoRecordView@@IAEXPAVCCmdUI@@@Z 5f72bfaf f   daoview.obj
 0001:0002afe3       ?OnMove@CDaoRecordView@@IAEXHH@Z 5f72bfe3 f   daoview.obj
 0001:0002b000       ??_GCDaoRecordView@@UAEPAXI@Z 5f72c000 f i daoview.obj
 0001:0002b000       ??_ECDaoRecordView@@UAEPAXI@Z 5f72c000 f i daoview.obj
 0001:0002b030       ??_Estringdispid@CComTypeInfoHolder@ATL@@QAEPAXI@Z 5f72c030 f i viewoled.obj
 0001:0002b0a0       ??1stringdispid@CComTypeInfoHolder@ATL@@QAE@XZ 5f72c0a0 f i viewoled.obj
 0001:0002b0c0       ??1CComBSTR@ATL@@QAE@XZ    5f72c0c0 f i viewoled.obj
 0001:0002b0e0       ?MovePrev@CRowset@ATL@@QAEJXZ 5f72c0e0 f i viewoled.obj
 0001:0002b100       ?MoveNext@CRowset@ATL@@QAEJXZ 5f72c100 f i viewoled.obj
 0001:0002b120       ?MoveNext@CRowset@ATL@@QAEJJ_N@Z 5f72c120 f i viewoled.obj
 0001:0002b230       ?AtlTrace2@ATL@@YAXKIPBGZZ 5f72c230 f i viewoled.obj
 0001:0002b2e0       ?ReleaseRows@CRowset@ATL@@QAEJXZ 5f72c2e0 f i viewoled.obj
 0001:0002b370       ?MoveFirst@CRowset@ATL@@QAEJXZ 5f72c370 f i viewoled.obj
 0001:0002b420       ?MoveLast@CRowset@ATL@@QAEJXZ 5f72c420 f i viewoled.obj
 0001:0002b530       ?GetData@CRowset@ATL@@QAEJXZ 5f72c530 f i viewoled.obj
 0001:0002b5e0       ?GetNumAccessors@CAccessorBase@ATL@@QBEKXZ 5f72c5e0 f i viewoled.obj
 0001:0002b600       ?IsAutoAccessor@CAccessorBase@ATL@@QBE_NK@Z 5f72c600 f i viewoled.obj
 0001:0002b690       ?GetData@CRowset@ATL@@QAEJH@Z 5f72c690 f i viewoled.obj
 0001:0002b780       ?GetHAccessor@CAccessorBase@ATL@@QBEKK@Z 5f72c780 f i viewoled.obj
 0001:0002b7e0       ?GetBuffer@CAccessorBase@ATL@@QBEPAEXZ 5f72c7e0 f i viewoled.obj
 0001:0002b800       ?SetData@CRowset@ATL@@QBEJH@Z 5f72c800 f i viewoled.obj
 0001:0002b8a2       ?AfxGetModuleState@@YGPAVAFX_MODULE_STATE@@XZ 5f72c8a2 f   MFC42UD:MFC42uD.DLL
 0001:0002b8a8       ?AfxTermThread@@YGXPAUHINSTANCE__@@@Z 5f72c8a8 f   MFC42UD:MFC42uD.DLL
 0001:0002b8ae       ?AfxTermExtensionModule@@YGXAAUAFX_EXTENSION_MODULE@@H@Z 5f72c8ae f   MFC42UD:MFC42uD.DLL
 0001:0002b8b4       ??0CDynLinkLibrary@@QAE@AAUAFX_EXTENSION_MODULE@@H@Z 5f72c8b4 f   MFC42UD:MFC42uD.DLL
 0001:0002b8ba       ??2CObject@@SGPAXI@Z       5f72c8ba f   MFC42UD:MFC42uD.DLL
 0001:0002b8c0       ?AfxAssertFailedLine@@YGHPBDH@Z 5f72c8c0 f   MFC42UD:MFC42uD.DLL
 0001:0002b8c6       ?AfxInitExtensionModule@@YGHAAUAFX_EXTENSION_MODULE@@PAUHINSTANCE__@@@Z 5f72c8c6 f   MFC42UD:MFC42uD.DLL
 0001:0002b8cc       ??3CObject@@SGXPAX@Z       5f72c8cc f   MFC42UD:MFC42uD.DLL
 0001:0002b8d2       ?AfxGetAppModuleState@@YGPAVAFX_MODULE_STATE@@XZ 5f72c8d2 f   MFC42UD:MFC42uD.DLL
 0001:0002b8d8       ??3@YAXPAX@Z               5f72c8d8 f   MFC42UD:MFC42uD.DLL
 0001:0002b8de       ??2@YAPAXI@Z               5f72c8de f   MFC42UD:MFC42uD.DLL
 0001:0002b8e4       ??3CException@@SGXPAX@Z    5f72c8e4 f   MFC42UD:MFC42uD.DLL
 0001:0002b8ea       ??3CException@@SGXPAXPBDH@Z 5f72c8ea f   MFC42UD:MFC42uD.DLL
 0001:0002b8f0       ?AfxTrace@@YAXPBGZZ        5f72c8f0 f   MFC42UD:MFC42uD.DLL
 0001:0002b8f6       ?LoadStringW@CString@@QAEHI@Z 5f72c8f6 f   MFC42UD:MFC42uD.DLL
 0001:0002b8fc       ??2CObject@@SGPAXIPBDH@Z   5f72c8fc f   MFC42UD:MFC42uD.DLL
 0001:0002b902       ?ReportError@CException@@UAEHII@Z 5f72c902 f   MFC42UD:MFC42uD.DLL
 0001:0002b908       ?Dump@CObject@@UBEXAAVCDumpContext@@@Z 5f72c908 f   MFC42UD:MFC42uD.DLL
 0001:0002b90e       ?AssertValid@CObject@@UBEXXZ 5f72c90e f   MFC42UD:MFC42uD.DLL
 0001:0002b914       ?Serialize@CObject@@UAEXAAVCArchive@@@Z 5f72c914 f   MFC42UD:MFC42uD.DLL
 0001:0002b91a       ??1CString@@QAE@XZ         5f72c91a f   MFC42UD:MFC42uD.DLL
 0001:0002b920       ??1CException@@UAE@XZ      5f72c920 f   MFC42UD:MFC42uD.DLL
 0001:0002b926       ??0CString@@QAE@XZ         5f72c926 f   MFC42UD:MFC42uD.DLL
 0001:0002b92c       ??0CException@@QAE@XZ      5f72c92c f   MFC42UD:MFC42uD.DLL
 0001:0002b932       ??H@YG?AVCString@@ABV0@PBG@Z 5f72c932 f   MFC42UD:MFC42uD.DLL
 0001:0002b938       ??H@YG?AVCString@@PBGABV0@@Z 5f72c938 f   MFC42UD:MFC42uD.DLL
 0001:0002b93e       ??4CString@@QAEABV0@ABV0@@Z 5f72c93e f   MFC42UD:MFC42uD.DLL
 0001:0002b944       ?Right@CString@@QBE?AV1@H@Z 5f72c944 f   MFC42UD:MFC42uD.DLL
 0001:0002b94a       ?GetLength@CString@@QBEHXZ 5f72c94a f   MFC42UD:MFC42uD.DLL
 0001:0002b950       ??YCString@@QAEABV0@ABV0@@Z 5f72c950 f   MFC42UD:MFC42uD.DLL
 0001:0002b956       ?Left@CString@@QBE?AV1@H@Z 5f72c956 f   MFC42UD:MFC42uD.DLL
 0001:0002b95c       ?Find@CString@@QBEHG@Z     5f72c95c f   MFC42UD:MFC42uD.DLL
 0001:0002b962       ??ACString@@QBEGH@Z        5f72c962 f   MFC42UD:MFC42uD.DLL
 0001:0002b968       ?IsEmpty@CString@@QBEHXZ   5f72c968 f   MFC42UD:MFC42uD.DLL
 0001:0002b96e       ??YCString@@QAEABV0@PBG@Z  5f72c96e f   MFC42UD:MFC42uD.DLL
 0001:0002b974       ??BCString@@QBEPBGXZ       5f72c974 f   MFC42UD:MFC42uD.DLL
 0001:0002b97a       ??4CString@@QAEABV0@PBE@Z  5f72c97a f   MFC42UD:MFC42uD.DLL
 0001:0002b980       ?AfxAssertValidObject@@YGXPBVCObject@@PBDH@Z 5f72c980 f   MFC42UD:MFC42uD.DLL
 0001:0002b986       ?AfxIsValidString@@YGHPBGH@Z 5f72c986 f   MFC42UD:MFC42uD.DLL
 0001:0002b98c       ??0CString@@QAE@PBG@Z      5f72c98c f   MFC42UD:MFC42uD.DLL
 0001:0002b992       ?Empty@CString@@QAEXXZ     5f72c992 f   MFC42UD:MFC42uD.DLL
 0001:0002b998       ??1CObject@@UAE@XZ         5f72c998 f   MFC42UD:MFC42uD.DLL
 0001:0002b99e       ??0CPtrList@@QAE@H@Z       5f72c99e f   MFC42UD:MFC42uD.DLL
 0001:0002b9a4       ??0CObject@@IAE@XZ         5f72c9a4 f   MFC42UD:MFC42uD.DLL
 0001:0002b9aa       ??1CPtrList@@UAE@XZ        5f72c9aa f   MFC42UD:MFC42uD.DLL
 0001:0002b9b0       ??4CString@@QAEABV0@PBG@Z  5f72c9b0 f   MFC42UD:MFC42uD.DLL
 0001:0002b9b6       ?IsKindOf@CObject@@QBEHPBUCRuntimeClass@@@Z 5f72c9b6 f   MFC42UD:MFC42uD.DLL
 0001:0002b9bc       ?AfxUnlockGlobals@@YGXH@Z  5f72c9bc f   MFC42UD:MFC42uD.DLL
 0001:0002b9c2       ?GetHead@CPtrList@@QAEAAPAXXZ 5f72c9c2 f   MFC42UD:MFC42uD.DLL
 0001:0002b9c8       ?IsEmpty@CPtrList@@QBEHXZ  5f72c9c8 f   MFC42UD:MFC42uD.DLL
 0001:0002b9ce       ?AfxLockGlobals@@YGXH@Z    5f72c9ce f   MFC42UD:MFC42uD.DLL
 0001:0002b9d4       ?Delete@CException@@QAEXXZ 5f72c9d4 f   MFC42UD:MFC42uD.DLL
 0001:0002b9da       ??0CString@@QAE@PBD@Z      5f72c9da f   MFC42UD:MFC42uD.DLL
 0001:0002b9e0       ?AfxThrowMemoryException@@YGXXZ 5f72c9e0 f   MFC42UD:MFC42uD.DLL
 0001:0002b9e6       ?GetSafeOwner_@CWnd@@SGPAUHWND__@@PAU2@PAPAU2@@Z 5f72c9e6 f   MFC42UD:MFC42uD.DLL
 0001:0002b9ec       ??4CString@@QAEABV0@PBD@Z  5f72c9ec f   MFC42UD:MFC42uD.DLL
 0001:0002b9f2       ?GetDepth@CDumpContext@@QBEHXZ 5f72c9f2 f   MFC42UD:MFC42uD.DLL
 0001:0002b9f8       ??6CDumpContext@@QAEAAV0@K@Z 5f72c9f8 f   MFC42UD:MFC42uD.DLL
 0001:0002b9fe       ??6CDumpContext@@QAEAAV0@H@Z 5f72c9fe f   MFC42UD:MFC42uD.DLL
 0001:0002ba04       ??6@YGAAVCDumpContext@@AAV0@ABVCString@@@Z 5f72ca04 f   MFC42UD:MFC42uD.DLL
 0001:0002ba0a       ??6CDumpContext@@QAEAAV0@PBX@Z 5f72ca0a f   MFC42UD:MFC42uD.DLL
 0001:0002ba10       ??6CDumpContext@@QAEAAV0@PBD@Z 5f72ca10 f   MFC42UD:MFC42uD.DLL
 0001:0002ba16       ??1CMapPtrToPtr@@UAE@XZ    5f72ca16 f   MFC42UD:MFC42uD.DLL
 0001:0002ba1c       ?AddHead@CPtrList@@QAEPAU__POSITION@@PAX@Z 5f72ca1c f   MFC42UD:MFC42uD.DLL
 0001:0002ba22       ?AfxIsValidAddress@@YGHPBXIH@Z 5f72ca22 f   MFC42UD:MFC42uD.DLL
 0001:0002ba28       ??0CMapPtrToPtr@@QAE@H@Z   5f72ca28 f   MFC42UD:MFC42uD.DLL
 0001:0002ba2e       ?RemoveAt@CPtrList@@QAEXPAU__POSITION@@@Z 5f72ca2e f   MFC42UD:MFC42uD.DLL
 0001:0002ba34       ?Find@CPtrList@@QBEPAU__POSITION@@PAXPAU2@@Z 5f72ca34 f   MFC42UD:MFC42uD.DLL
 0001:0002ba3a       ?Find@CString@@QBEHPBG@Z   5f72ca3a f   MFC42UD:MFC42uD.DLL
 0001:0002ba40       ??2@YAPAXIPBDH@Z           5f72ca40 f   MFC42UD:MFC42uD.DLL
 0001:0002ba46       ??3@YAXPAXPBDH@Z           5f72ca46 f   MFC42UD:MFC42uD.DLL
 0001:0002ba4c       ?GetBuffer@CString@@QAEPAGH@Z 5f72ca4c f   MFC42UD:MFC42uD.DLL
 0001:0002ba52       ?GetBufferSetLength@CString@@QAEPAGH@Z 5f72ca52 f   MFC42UD:MFC42uD.DLL
 0001:0002ba58       ??9@YG_NABVCString@@0@Z    5f72ca58 f   MFC42UD:MFC42uD.DLL
 0001:0002ba5e       ??3CObject@@SGXPAXPBDH@Z   5f72ca5e f   MFC42UD:MFC42uD.DLL
 0001:0002ba64       ?ReleaseBuffer@CString@@QAEXH@Z 5f72ca64 f   MFC42UD:MFC42uD.DLL
 0001:0002ba6a       ?MakeUpper@CString@@QAEXXZ 5f72ca6a f   MFC42UD:MFC42uD.DLL
 0001:0002ba70       ?SetAt@CString@@QAEXHG@Z   5f72ca70 f   MFC42UD:MFC42uD.DLL
 0001:0002ba76       ?Lookup@CMapPtrToPtr@@QBEHPAXAAPAX@Z 5f72ca76 f   MFC42UD:MFC42uD.DLL
 0001:0002ba7c       ??8@YG_NABVCString@@PBG@Z  5f72ca7c f   MFC42UD:MFC42uD.DLL
 0001:0002ba82       ??6CDumpContext@@QAEAAV0@PBVCObject@@@Z 5f72ca82 f   MFC42UD:MFC42uD.DLL
 0001:0002ba88       ??6CDumpContext@@QAEAAV0@J@Z 5f72ca88 f   MFC42UD:MFC42uD.DLL
 0001:0002ba8e       ??6CDumpContext@@QAEAAV0@I@Z 5f72ca8e f   MFC42UD:MFC42uD.DLL
 0001:0002ba94       ??1CProcessLocalObject@@QAE@XZ 5f72ca94 f   MFC42UD:MFC42uD.DLL
 0001:0002ba9a       ?GetData@CProcessLocalObject@@QAEPAVCNoTrackObject@@P6GPAV2@XZ@Z 5f72ca9a f   MFC42UD:MFC42uD.DLL
 0001:0002baa0       ??3CNoTrackObject@@SGXPAX@Z 5f72caa0 f   MFC42UD:MFC42uD.DLL
 0001:0002baa6       ??2CNoTrackObject@@SGPAXI@Z 5f72caa6 f   MFC42UD:MFC42uD.DLL
 0001:0002baac       ?GetData@CByteArray@@QAEPAEXZ 5f72caac f   MFC42UD:MFC42uD.DLL
 0001:0002bab2       ??YCString@@QAEABV0@D@Z    5f72cab2 f   MFC42UD:MFC42uD.DLL
 0001:0002bab8       ?SetAt@CMapPtrToPtr@@QAEXPAX0@Z 5f72cab8 f   MFC42UD:MFC42uD.DLL
 0001:0002babe       ??6CDumpContext@@QAEAAV0@PBG@Z 5f72cabe f   MFC42UD:MFC42uD.DLL
 0001:0002bac4       ?LockBuffer@CString@@QAEPAGXZ 5f72cac4 f   MFC42UD:MFC42uD.DLL
 0001:0002baca       ??6CDumpContext@@QAEAAV0@E@Z 5f72caca f   MFC42UD:MFC42uD.DLL
 0001:0002bad0       ??0CByteArray@@QAE@XZ      5f72cad0 f   MFC42UD:MFC42uD.DLL
 0001:0002bad6       ?SetSize@CByteArray@@QAEXHH@Z 5f72cad6 f   MFC42UD:MFC42uD.DLL
 0001:0002badc       ??ACByteArray@@QAEAAEH@Z   5f72cadc f   MFC42UD:MFC42uD.DLL
 0001:0002bae2       ?GetSize@CByteArray@@QBEHXZ 5f72cae2 f   MFC42UD:MFC42uD.DLL
 0001:0002bae8       ??6@YGAAVCDumpContext@@AAV0@VCTime@@@Z 5f72cae8 f   MFC42UD:MFC42uD.DLL
 0001:0002baee       ??0CTime@@QAE@XZ           5f72caee f   MFC42UD:MFC42uD.DLL
 0001:0002baf4       ??9CTime@@QBEHV0@@Z        5f72caf4 f   MFC42UD:MFC42uD.DLL
 0001:0002bafa       ??0CTime@@QAE@ABV0@@Z      5f72cafa f   MFC42UD:MFC42uD.DLL
 0001:0002bb00       ??0CTime@@QAE@HHHHHHH@Z    5f72cb00 f   MFC42UD:MFC42uD.DLL
 0001:0002bb06       ??4CTime@@QAEABV0@ABV0@@Z  5f72cb06 f   MFC42UD:MFC42uD.DLL
 0001:0002bb0c       ??0CTime@@QAE@J@Z          5f72cb0c f   MFC42UD:MFC42uD.DLL
 0001:0002bb12       ?GetSecond@CTime@@QBEHXZ   5f72cb12 f   MFC42UD:MFC42uD.DLL
 0001:0002bb18       ?GetMinute@CTime@@QBEHXZ   5f72cb18 f   MFC42UD:MFC42uD.DLL
 0001:0002bb1e       ?GetHour@CTime@@QBEHXZ     5f72cb1e f   MFC42UD:MFC42uD.DLL
 0001:0002bb24       ?GetDay@CTime@@QBEHXZ      5f72cb24 f   MFC42UD:MFC42uD.DLL
 0001:0002bb2a       ?GetMonth@CTime@@QBEHXZ    5f72cb2a f   MFC42UD:MFC42uD.DLL
 0001:0002bb30       ?GetYear@CTime@@QBEHXZ     5f72cb30 f   MFC42UD:MFC42uD.DLL
 0001:0002bb36       ??6CDumpContext@@QAEAAV0@G@Z 5f72cb36 f   MFC42UD:MFC42uD.DLL
 0001:0002bb3c       ??8CTime@@QBEHV0@@Z        5f72cb3c f   MFC42UD:MFC42uD.DLL
 0001:0002bb42       ??8@YG_NABVCString@@0@Z    5f72cb42 f   MFC42UD:MFC42uD.DLL
 0001:0002bb48       ?Copy@CByteArray@@QAEXABV1@@Z 5f72cb48 f   MFC42UD:MFC42uD.DLL
 0001:0002bb4e       ?OnEndPrintPreview@CView@@MAEXPAVCDC@@PAUCPrintInfo@@UtagPOINT@@PAVCPreviewView@@@Z 5f72cb4e f   MFC42UD:MFC42uD.DLL
 0001:0002bb54       ?OnEndPrinting@CView@@MAEXPAVCDC@@PAUCPrintInfo@@@Z 5f72cb54 f   MFC42UD:MFC42uD.DLL
 0001:0002bb5a       ?OnPrint@CView@@MAEXPAVCDC@@PAUCPrintInfo@@@Z 5f72cb5a f   MFC42UD:MFC42uD.DLL
 0001:0002bb60       ?OnBeginPrinting@CView@@MAEXPAVCDC@@PAUCPrintInfo@@@Z 5f72cb60 f   MFC42UD:MFC42uD.DLL
 0001:0002bb66       ?OnPreparePrinting@CView@@MAEHPAUCPrintInfo@@@Z 5f72cb66 f   MFC42UD:MFC42uD.DLL
 0001:0002bb6c       ?OnDraw@CFormView@@MAEXPAVCDC@@@Z 5f72cb6c f   MFC42UD:MFC42uD.DLL
 0001:0002bb72       ?OnUpdate@CView@@MAEXPAV1@JPAVCObject@@@Z 5f72cb72 f   MFC42UD:MFC42uD.DLL
 0001:0002bb78       ?OnActivateFrame@CFormView@@MAEXIPAVCFrameWnd@@@Z 5f72cb78 f   MFC42UD:MFC42uD.DLL
 0001:0002bb7e       ?OnActivateView@CFormView@@MAEXHPAVCView@@0@Z 5f72cb7e f   MFC42UD:MFC42uD.DLL
 0001:0002bb84       ?OnPrepareDC@CScrollView@@UAEXPAVCDC@@PAUCPrintInfo@@@Z 5f72cb84 f   MFC42UD:MFC42uD.DLL
 0001:0002bb8a       ?OnDragScroll@CView@@UAEKKVCPoint@@@Z 5f72cb8a f   MFC42UD:MFC42uD.DLL
 0001:0002bb90       ?OnDropEx@CView@@UAEKPAVCOleDataObject@@KKVCPoint@@@Z 5f72cb90 f   MFC42UD:MFC42uD.DLL
 0001:0002bb96       ?OnDrop@CView@@UAEHPAVCOleDataObject@@KVCPoint@@@Z 5f72cb96 f   MFC42UD:MFC42uD.DLL
 0001:0002bb9c       ?OnDragLeave@CView@@UAEXXZ 5f72cb9c f   MFC42UD:MFC42uD.DLL
 0001:0002bba2       ?OnDragOver@CView@@UAEKPAVCOleDataObject@@KVCPoint@@@Z 5f72cba2 f   MFC42UD:MFC42uD.DLL
 0001:0002bba8       ?OnDragEnter@CView@@UAEKPAVCOleDataObject@@KVCPoint@@@Z 5f72cba8 f   MFC42UD:MFC42uD.DLL
 0001:0002bbae       ?OnScrollBy@CScrollView@@UAEHVCSize@@H@Z 5f72cbae f   MFC42UD:MFC42uD.DLL
 0001:0002bbb4       ?OnScroll@CScrollView@@UAEHIIH@Z 5f72cbb4 f   MFC42UD:MFC42uD.DLL
 0001:0002bbba       ?IsSelected@CView@@UBEHPBVCObject@@@Z 5f72cbba f   MFC42UD:MFC42uD.DLL
 0001:0002bbc0       ?SetOccDialogInfo@CFormView@@MAEHPAU_AFX_OCC_DIALOG_INFO@@@Z 5f72cbc0 f   MFC42UD:MFC42uD.DLL
 0001:0002bbc6       ?IsFrameWnd@CWnd@@UBEHXZ   5f72cbc6 f   MFC42UD:MFC42uD.DLL
 0001:0002bbcc       ?CheckAutoCenter@CWnd@@UAEHXZ 5f72cbcc f   MFC42UD:MFC42uD.DLL
 0001:0002bbd2       ?OnChildNotify@CWnd@@MAEHIIJPAJ@Z 5f72cbd2 f   MFC42UD:MFC42uD.DLL
 0001:0002bbd8       ?PostNcDestroy@CView@@MAEXXZ 5f72cbd8 f   MFC42UD:MFC42uD.DLL
 0001:0002bbde       ?DefWindowProcW@CWnd@@MAEJIIJ@Z 5f72cbde f   MFC42UD:MFC42uD.DLL
 0001:0002bbe4       ?OnWndMsg@CWnd@@MAEHIIJPAJ@Z 5f72cbe4 f   MFC42UD:MFC42uD.DLL
 0001:0002bbea       ?WindowProc@CWnd@@MAEJIIJ@Z 5f72cbea f   MFC42UD:MFC42uD.DLL
 0001:0002bbf0       ?OnAmbientProperty@CWnd@@UAEHPAVCOleControlSite@@JPAUtagVARIANT@@@Z 5f72cbf0 f   MFC42UD:MFC42uD.DLL
 0001:0002bbf6       ?PreTranslateMessage@CFormView@@MAEHPAUtagMSG@@@Z 5f72cbf6 f   MFC42UD:MFC42uD.DLL
 0001:0002bbfc       ?EndModalState@CWnd@@UAEXXZ 5f72cbfc f   MFC42UD:MFC42uD.DLL
 0001:0002bc02       ?BeginModalState@CWnd@@UAEXXZ 5f72cc02 f   MFC42UD:MFC42uD.DLL
 0001:0002bc08       ?DoDataExchange@CWnd@@MAEXPAVCDataExchange@@@Z 5f72cc08 f   MFC42UD:MFC42uD.DLL
 0001:0002bc0e       ?GetSuperWndProcAddr@CWnd@@MAEPAP6GJPAUHWND__@@IIJ@ZXZ 5f72cc0e f   MFC42UD:MFC42uD.DLL
 0001:0002bc14       ?OnNotify@CWnd@@MAEHIJPAJ@Z 5f72cc14 f   MFC42UD:MFC42uD.DLL
 0001:0002bc1a       ?OnCommand@CWnd@@MAEHIJ@Z  5f72cc1a f   MFC42UD:MFC42uD.DLL
 0001:0002bc20       ?EndModalLoop@CWnd@@UAEXH@Z 5f72cc20 f   MFC42UD:MFC42uD.DLL
 0001:0002bc26       ?ContinueModal@CWnd@@UAEHXZ 5f72cc26 f   MFC42UD:MFC42uD.DLL
 0001:0002bc2c       ?WinHelpW@CWnd@@UAEXKI@Z   5f72cc2c f   MFC42UD:MFC42uD.DLL
 0001:0002bc32       ?GetScrollBarCtrl@CView@@UBEPAVCScrollBar@@H@Z 5f72cc32 f   MFC42UD:MFC42uD.DLL
 0001:0002bc38       ?OnToolHitTest@CWnd@@UBEHVCPoint@@PAUtagTOOLINFOW@@@Z 5f72cc38 f   MFC42UD:MFC42uD.DLL
 0001:0002bc3e       ?CalcWindowRect@CScrollView@@UAEXPAUtagRECT@@I@Z 5f72cc3e f   MFC42UD:MFC42uD.DLL
 0001:0002bc44       ?PreCreateWindow@CView@@MAEHAAUtagCREATESTRUCTW@@@Z 5f72cc44 f   MFC42UD:MFC42uD.DLL
 0001:0002bc4a       ?DestroyWindow@CWnd@@UAEHXZ 5f72cc4a f   MFC42UD:MFC42uD.DLL
 0001:0002bc50       ?Create@CFormView@@MAEHPBG0KABUtagRECT@@PAVCWnd@@IPAUCCreateContext@@@Z 5f72cc50 f   MFC42UD:MFC42uD.DLL
 0001:0002bc56       ?PreSubclassWindow@CWnd@@UAEXXZ 5f72cc56 f   MFC42UD:MFC42uD.DLL
 0001:0002bc5c       ?GetConnectionHook@CCmdTarget@@MAEPAUIConnectionPoint@@ABU_GUID@@@Z 5f72cc5c f   MFC42UD:MFC42uD.DLL
 0001:0002bc62       ?GetExtraConnectionPoints@CCmdTarget@@MAEHPAVCPtrArray@@@Z 5f72cc62 f   MFC42UD:MFC42uD.DLL
 0001:0002bc68       ?GetInterfaceHook@CCmdTarget@@UAEPAUIUnknown@@PBX@Z 5f72cc68 f   MFC42UD:MFC42uD.DLL
 0001:0002bc6e       ?OnCreateAggregates@CCmdTarget@@UAEHXZ 5f72cc6e f   MFC42UD:MFC42uD.DLL
 0001:0002bc74       ?GetEventSinkMap@CCmdTarget@@MBEPBUAFX_EVENTSINKMAP@@XZ 5f72cc74 f   MFC42UD:MFC42uD.DLL
 0001:0002bc7a       ?GetInterfaceMap@CCmdTarget@@MBEPBUAFX_INTERFACEMAP@@XZ 5f72cc7a f   MFC42UD:MFC42uD.DLL
 0001:0002bc80       ?GetConnectionMap@CCmdTarget@@MBEPBUAFX_CONNECTIONMAP@@XZ 5f72cc80 f   MFC42UD:MFC42uD.DLL
 0001:0002bc86       ?GetDispatchMap@CCmdTarget@@MBEPBUAFX_DISPMAP@@XZ 5f72cc86 f   MFC42UD:MFC42uD.DLL
 0001:0002bc8c       ?GetCommandMap@CCmdTarget@@MBEPBUAFX_OLECMDMAP@@XZ 5f72cc8c f   MFC42UD:MFC42uD.DLL
 0001:0002bc92       ?GetTypeLib@CCmdTarget@@UAEJKPAPAUITypeLib@@@Z 5f72cc92 f   MFC42UD:MFC42uD.DLL
 0001:0002bc98       ?GetTypeLibCache@CCmdTarget@@UAEPAVCTypeLibCache@@XZ 5f72cc98 f   MFC42UD:MFC42uD.DLL
 0001:0002bc9e       ?GetTypeInfoCount@CCmdTarget@@UAEIXZ 5f72cc9e f   MFC42UD:MFC42uD.DLL
 0001:0002bca4       ?GetDispatchIID@CCmdTarget@@UAEHPAU_GUID@@@Z 5f72cca4 f   MFC42UD:MFC42uD.DLL
 0001:0002bcaa       ?IsInvokeAllowed@CCmdTarget@@UAEHJ@Z 5f72ccaa f   MFC42UD:MFC42uD.DLL
 0001:0002bcb0       ?OnFinalRelease@CWnd@@UAEXXZ 5f72ccb0 f   MFC42UD:MFC42uD.DLL
 0001:0002bcb6       ?OnCmdMsg@CView@@UAEHIHPAXPAUAFX_CMDHANDLERINFO@@@Z 5f72ccb6 f   MFC42UD:MFC42uD.DLL
 0001:0002bcbc       ??0CFormView@@IAE@PBG@Z    5f72ccbc f   MFC42UD:MFC42uD.DLL
 0001:0002bcc2       ??0CFormView@@IAE@I@Z      5f72ccc2 f   MFC42UD:MFC42uD.DLL
 0001:0002bcc8       ??1CScrollView@@UAE@XZ     5f72ccc8 f   MFC42UD:MFC42uD.DLL
 0001:0002bcce       ?OnInitialUpdate@CFormView@@UAEXXZ 5f72ccce f   MFC42UD:MFC42uD.DLL
 0001:0002bcd4       ??1CWaitCursor@@QAE@XZ     5f72ccd4 f   MFC42UD:MFC42uD.DLL
 0001:0002bcda       ??0CWaitCursor@@QAE@XZ     5f72ccda f   MFC42UD:MFC42uD.DLL
 0001:0002bce0       ?UpdateData@CWnd@@QAEHH@Z  5f72cce0 f   MFC42UD:MFC42uD.DLL
 0001:0002bce6       ?AfxSetWindowText@@YGXPAUHWND__@@PBG@Z 5f72cce6 f   MFC42UD:MFC42uD.DLL
 0001:0002bcec       ?PrepareEditCtrl@CDataExchange@@QAEPAUHWND__@@H@Z 5f72ccec f   MFC42UD:MFC42uD.DLL
 0001:0002bcf2       ?DDX_Text@@YGXPAVCDataExchange@@HAAH@Z 5f72ccf2 f   MFC42UD:MFC42uD.DLL
 0001:0002bcf8       ?DDX_Text@@YGXPAVCDataExchange@@HAAE@Z 5f72ccf8 f   MFC42UD:MFC42uD.DLL
 0001:0002bcfe       ?DDX_Text@@YGXPAVCDataExchange@@HAAI@Z 5f72ccfe f   MFC42UD:MFC42uD.DLL
 0001:0002bd04       ?DDX_Text@@YGXPAVCDataExchange@@HAAJ@Z 5f72cd04 f   MFC42UD:MFC42uD.DLL
 0001:0002bd0a       ?DDX_Text@@YGXPAVCDataExchange@@HAAK@Z 5f72cd0a f   MFC42UD:MFC42uD.DLL
 0001:0002bd10       ?AfxFailMaxChars@@YGXPAVCDataExchange@@H@Z 5f72cd10 f   MFC42UD:MFC42uD.DLL
 0001:0002bd16       ?GetAllocLength@CString@@QBEHXZ 5f72cd16 f   MFC42UD:MFC42uD.DLL
 0001:0002bd1c       ?PrepareCtrl@CDataExchange@@QAEPAUHWND__@@H@Z 5f72cd1c f   MFC42UD:MFC42uD.DLL
 0001:0002bd22       ?DDX_LBIndex@@YGXPAVCDataExchange@@HAAH@Z 5f72cd22 f   MFC42UD:MFC42uD.DLL
 0001:0002bd28       ?DDX_CBIndex@@YGXPAVCDataExchange@@HAAH@Z 5f72cd28 f   MFC42UD:MFC42uD.DLL
 0001:0002bd2e       ?DDX_Scroll@@YGXPAVCDataExchange@@HAAH@Z 5f72cd2e f   MFC42UD:MFC42uD.DLL
 0001:0002bd34       ?AfxFailRadio@@YGXPAVCDataExchange@@@Z 5f72cd34 f   MFC42UD:MFC42uD.DLL
 0001:0002bd3a       ?DDX_Radio@@YGXPAVCDataExchange@@HAAH@Z 5f72cd3a f   MFC42UD:MFC42uD.DLL
 0001:0002bd40       ?AssertValid@CFormView@@UBEXXZ 5f72cd40 f   MFC42UD:MFC42uD.DLL
 0001:0002bd46       ?Dump@CFormView@@UBEXAAVCDumpContext@@@Z 5f72cd46 f   MFC42UD:MFC42uD.DLL
 0001:0002bd4c       ?OnMove@CWnd@@IAEXHH@Z     5f72cd4c f   MFC42UD:MFC42uD.DLL
 0001:0002bd52       ??6CDumpContext@@QAEAAV0@M@Z 5f72cd52 f   MFC42UD:MFC42uD.DLL
 0001:0002bd58       ??6CDumpContext@@QAEAAV0@N@Z 5f72cd58 f   MFC42UD:MFC42uD.DLL
 0001:0002bd5e       ?AfxTextFloatFormat@@YGXPAVCDataExchange@@HPAXNH@Z 5f72cd5e f   MFC42UD:MFC42uD.DLL
 0001:0002bd64       ?IsEmpty@CMapPtrToPtr@@QBEHXZ 5f72cd64 f   MFC42UD:MFC42uD.DLL
 0001:0002bd6a       ?RemoveKey@CMapPtrToPtr@@QAEHPAX@Z 5f72cd6a f   MFC42UD:MFC42uD.DLL
 0001:0002bd70       ?RemoveAll@CMapPtrToPtr@@QAEXXZ 5f72cd70 f   MFC42UD:MFC42uD.DLL
 0001:0002bd76       ?GetNextAssoc@CMapPtrToPtr@@QBEXAAPAU__POSITION@@AAPAX1@Z 5f72cd76 f   MFC42UD:MFC42uD.DLL
 0001:0002bd7c       ?GetStartPosition@CMapPtrToPtr@@QBEPAU__POSITION@@XZ 5f72cd7c f   MFC42UD:MFC42uD.DLL
 0001:0002bd82       ??0CString@@QAE@ABV0@@Z    5f72cd82 f   MFC42UD:MFC42uD.DLL
 0001:0002bd88       ??3CNoTrackObject@@SGXPAXPBDH@Z 5f72cd88 f   MFC42UD:MFC42uD.DLL
 0001:0002bd8e       ??2CNoTrackObject@@SGPAXIPBDH@Z 5f72cd8e f   MFC42UD:MFC42uD.DLL
 0001:0002bd94       ?AfxGetApp@@YGPAVCWinApp@@XZ 5f72cd94 f   MFC42UD:MFC42uD.DLL
 0001:0002bd9a       ??6CDumpContext@@QAEAAV0@ABVCObject@@@Z 5f72cd9a f   MFC42UD:MFC42uD.DLL
 0001:0002bda0       ?DDX_Text@@YGXPAVCDataExchange@@HAAF@Z 5f72cda0 f   MFC42UD:MFC42uD.DLL
 0001:0002bda6       ?DDX_Text@@YGXPAVCDataExchange@@HAAM@Z 5f72cda6 f   MFC42UD:MFC42uD.DLL
 0001:0002bdac       ?DDX_Text@@YGXPAVCDataExchange@@HAAN@Z 5f72cdac f   MFC42UD:MFC42uD.DLL
 0001:0002bdb2       ?DDX_Text@@YGXPAVCDataExchange@@HAAVCString@@@Z 5f72cdb2 f   MFC42UD:MFC42uD.DLL
 0001:0002bdb8       ?DDX_Text@@YGXPAVCDataExchange@@HPAGH@Z 5f72cdb8 f   MFC42UD:MFC42uD.DLL
 0001:0002bdbe       ?DDX_Slider@@YGXPAVCDataExchange@@HAAH@Z 5f72cdbe f   MFC42UD:MFC42uD.DLL
 0001:0002bdc4       ?Format@COleDateTime@@QBE?AVCString@@KK@Z 5f72cdc4 f   MFCO42UD:MFCO42uD.DLL
 0001:0002bdca       ?GetStatus@COleDateTime@@QBE?AW4DateTimeStatus@1@XZ 5f72cdca f   MFCO42UD:MFCO42uD.DLL
 0001:0002bdd0       ??4COleDateTime@@QAEABV0@ABV0@@Z 5f72cdd0 f   MFCO42UD:MFCO42uD.DLL
 0001:0002bdd6       ??0COleDateTime@@QAE@HHHHHH@Z 5f72cdd6 f   MFCO42UD:MFCO42uD.DLL
 0001:0002bddc       ?SetStatus@COleDateTime@@QAEXW4DateTimeStatus@1@@Z 5f72cddc f   MFCO42UD:MFCO42uD.DLL
 0001:0002bde2       ??0COleDateTime@@QAE@XZ    5f72cde2 f   MFCO42UD:MFCO42uD.DLL
 0001:0002bde8       ?GetSecond@COleDateTime@@QBEHXZ 5f72cde8 f   MFCO42UD:MFCO42uD.DLL
 0001:0002bdee       ?GetMinute@COleDateTime@@QBEHXZ 5f72cdee f   MFCO42UD:MFCO42uD.DLL
 0001:0002bdf4       ?GetHour@COleDateTime@@QBEHXZ 5f72cdf4 f   MFCO42UD:MFCO42uD.DLL
 0001:0002bdfa       ?GetDay@COleDateTime@@QBEHXZ 5f72cdfa f   MFCO42UD:MFCO42uD.DLL
 0001:0002be00       ?GetMonth@COleDateTime@@QBEHXZ 5f72ce00 f   MFCO42UD:MFCO42uD.DLL
 0001:0002be06       ?GetYear@COleDateTime@@QBEHXZ 5f72ce06 f   MFCO42UD:MFCO42uD.DLL
 0001:0002be0c       ??8COleDateTime@@QBEHABV0@@Z 5f72ce0c f   MFCO42UD:MFCO42uD.DLL
 0001:0002be12       ??6@YGAAVCDumpContext@@AAV0@VCOleDateTime@@@Z 5f72ce12 f   MFCO42UD:MFCO42uD.DLL
 0001:0002be18       ??0COleDateTime@@QAE@ABV0@@Z 5f72ce18 f   MFCO42UD:MFCO42uD.DLL
 0001:0002be1e       ??1COleVariant@@QAE@XZ     5f72ce1e f   MFCO42UD:MFCO42uD.DLL
 0001:0002be24       ??6@YGAAVCDumpContext@@AAV0@VCOleVariant@@@Z 5f72ce24 f   MFCO42UD:MFCO42uD.DLL
 0001:0002be2a       ??0COleVariant@@QAE@ABV0@@Z 5f72ce2a f   MFCO42UD:MFCO42uD.DLL
 0001:0002be30       ??0COleVariant@@QAE@JG@Z   5f72ce30 f   MFCO42UD:MFCO42uD.DLL
 0001:0002be36       ?Clear@COleVariant@@QAEXXZ 5f72ce36 f   MFCO42UD:MFCO42uD.DLL
 0001:0002be3c       ??0COleVariant@@QAE@XZ     5f72ce3c f   MFCO42UD:MFCO42uD.DLL
 0001:0002be42       ??0COleVariant@@QAE@PBGG@Z 5f72ce42 f   MFCO42UD:MFCO42uD.DLL
 0001:0002be48       ??4COleVariant@@QAEABV0@J@Z 5f72ce48 f   MFCO42UD:MFCO42uD.DLL
 0001:0002be4e       ??4COleDateTime@@QAEABV0@ABUtagVARIANT@@@Z 5f72ce4e f   MFCO42UD:MFCO42uD.DLL
 0001:0002be54       ??BCOleVariant@@QAEPAUtagVARIANT@@XZ 5f72ce54 f   MFCO42UD:MFCO42uD.DLL
 0001:0002be5a       ??0COleDateTime@@QAE@N@Z   5f72ce5a f   MFCO42UD:MFCO42uD.DLL
 0001:0002be60       ??0COleVariant@@QAE@FG@Z   5f72ce60 f   MFCO42UD:MFCO42uD.DLL
 0001:0002be66       ??0COleVariant@@QAE@ABUtagVARIANT@@@Z 5f72ce66 f   MFCO42UD:MFCO42uD.DLL
 0001:0002be6c       ??4COleVariant@@QAEABV0@QBG@Z 5f72ce6c f   MFCO42UD:MFCO42uD.DLL
 0001:0002be72       ?SetStatus@COleCurrency@@QAEXW4CurrencyStatus@1@@Z 5f72ce72 f   MFCO42UD:MFCO42uD.DLL
 0001:0002be78       ?GetStatus@COleCurrency@@QBE?AW4CurrencyStatus@1@XZ 5f72ce78 f   MFCO42UD:MFCO42uD.DLL
 0001:0002be7e       ??0COleCurrency@@QAE@XZ    5f72ce7e f   MFCO42UD:MFCO42uD.DLL
 0001:0002be84       ??4COleCurrency@@QAEABV0@ABV0@@Z 5f72ce84 f   MFCO42UD:MFCO42uD.DLL
 0001:0002be8a       ??9COleDateTime@@QBEHABV0@@Z 5f72ce8a f   MFCO42UD:MFCO42uD.DLL
 0001:0002be90       ??9COleCurrency@@QBEHABV0@@Z 5f72ce90 f   MFCO42UD:MFCO42uD.DLL
 0001:0002be96       ??4COleVariant@@QAEABV0@ABVCOleDateTime@@@Z 5f72ce96 f   MFCO42UD:MFCO42uD.DLL
 0001:0002be9c       ??4COleVariant@@QAEABV0@N@Z 5f72ce9c f   MFCO42UD:MFCO42uD.DLL
 0001:0002bea2       ??4COleVariant@@QAEABV0@M@Z 5f72cea2 f   MFCO42UD:MFCO42uD.DLL
 0001:0002bea8       ??4COleVariant@@QAEABV0@ABVCOleCurrency@@@Z 5f72cea8 f   MFCO42UD:MFCO42uD.DLL
 0001:0002beae       ??4COleVariant@@QAEABV0@F@Z 5f72ceae f   MFCO42UD:MFCO42uD.DLL
 0001:0002beb4       ??4COleVariant@@QAEABV0@E@Z 5f72ceb4 f   MFCO42UD:MFCO42uD.DLL
 0001:0002beba       ??4COleVariant@@QAEABV0@ABVCLongBinary@@@Z 5f72ceba f   MFCO42UD:MFCO42uD.DLL
 0001:0002bec0       ??4COleVariant@@QAEABV0@ABVCByteArray@@@Z 5f72cec0 f   MFCO42UD:MFCO42uD.DLL
 0001:0002bec6       ??6@YGAAVCDumpContext@@AAV0@VCOleCurrency@@@Z 5f72cec6 f   MFCO42UD:MFCO42uD.DLL
 0001:0002becc       ??0COleCurrency@@QAE@ABV0@@Z 5f72cecc f   MFCO42UD:MFCO42uD.DLL
 0001:0002bed2       ??4COleVariant@@QAEABV0@ABV0@@Z 5f72ced2 f   MFCO42UD:MFCO42uD.DLL
 0001:0002bed8       ??8COleVariant@@QBEHABUtagVARIANT@@@Z 5f72ced8 f   MFCO42UD:MFCO42uD.DLL
 0001:0002bede       ?DDX_Text@@YGXPAVCDataExchange@@HAAVCOleCurrency@@@Z 5f72cede f   MFCO42UD:MFCO42uD.DLL
 0001:0002bee4       ?DDX_Text@@YGXPAVCDataExchange@@HAAVCOleDateTime@@@Z 5f72cee4 f   MFCO42UD:MFCO42uD.DLL
 0001:0002beea       ___CxxFrameHandler         5f72ceea f   msvcrtd:MSVCRTD.dll
 0001:0002bef0       ??_L@YGXPAXIHP6EX0@Z1@Z    5f72cef0 f   msvcrtd:ehvecctr.obj
 0001:0002bf90       ??_M@YGXPAXIHP6EX0@Z@Z     5f72cf90 f   msvcrtd:ehvecdtr.obj
 0001:0002c040       ?__ArrayUnwind@@YGXPAXIHP6EX0@Z@Z 5f72d040 f   msvcrtd:ehvecdtr.obj
 0001:0002c0f0       ??0type_info@@AAE@ABV0@@Z  5f72d0f0 f   msvcrtd:ti_inst.obj
 0001:0002c110       ??_Gtype_info@@UAEPAXI@Z   5f72d110 f i msvcrtd:ti_inst.obj
 0001:0002c110       ??_Etype_info@@UAEPAXI@Z   5f72d110 f i msvcrtd:ti_inst.obj
 0001:0002c140       ??4type_info@@AAEAAV0@ABV0@@Z 5f72d140 f   msvcrtd:ti_inst.obj
 0001:0002c150       __CxxThrowException@8      5f72d150 f   msvcrtd:MSVCRTD.dll
 0001:0002c156       __wcsnicmp                 5f72d156 f   msvcrtd:MSVCRTD.dll
 0001:0002c160       __alloca_probe             5f72d160 f   msvcrtd:chkstk.obj
 0001:0002c160       __chkstk                   5f72d160 f   msvcrtd:chkstk.obj
 0001:0002c190       __CrtDbgReport             5f72d190 f   msvcrtd:MSVCRTD.dll
 0001:0002c196       _memset                    5f72d196 f   msvcrtd:MSVCRTD.dll
 0001:0002c19c       _memcpy                    5f72d19c f   msvcrtd:MSVCRTD.dll
 0001:0002c1a2       _wcsstr                    5f72d1a2 f   msvcrtd:MSVCRTD.dll
 0001:0002c1a8       _abs                       5f72d1a8 f   msvcrtd:MSVCRTD.dll
 0001:0002c1b0       __onexit                   5f72d1b0 f   msvcrtd:atonexit.obj
 0001:0002c1f0       _atexit                    5f72d1f0 f   msvcrtd:atonexit.obj
 0001:0002c208       _labs                      5f72d208 f   msvcrtd:MSVCRTD.dll
 0001:0002c20e       _memcmp                    5f72d20e f   msvcrtd:MSVCRTD.dll
 0001:0002c214       __purecall                 5f72d214 f   msvcrtd:MSVCRTD.dll
 0001:0002c21a       __vsnwprintf               5f72d21a f   msvcrtd:MSVCRTD.dll
 0001:0002c220       __CRT_INIT@12              5f72d220 f   msvcrtd:crtdll.obj
 0001:0002c330       __DllMainCRTStartup@12     5f72d330 f   msvcrtd:crtdll.obj
 0001:0002c424       __except_handler3          5f72d424 f   msvcrtd:MSVCRTD.dll
 0001:0002c42a       ?terminate@@YAXXZ          5f72d42a f   msvcrtd:MSVCRTD.dll
 0001:0002c430       ??1type_info@@UAE@XZ       5f72d430 f   msvcrtd:MSVCRTD.dll
 0001:0002c436       ___dllonexit               5f72d436 f   msvcrtd:MSVCRTD.dll
 0001:0002c43c       __free_dbg                 5f72d43c f   msvcrtd:MSVCRTD.dll
 0001:0002c442       __initterm                 5f72d442 f   msvcrtd:MSVCRTD.dll
 0001:0002c448       __malloc_dbg               5f72d448 f   msvcrtd:MSVCRTD.dll
 0001:0002c44e       _FreeLibrary@4             5f72d44e f   kernel32:KERNEL32.dll
 0001:0002c454       _GetModuleHandleA@4        5f72d454 f   kernel32:KERNEL32.dll
 0001:0002c45a       _LocalFree@4               5f72d45a f   kernel32:KERNEL32.dll
 0001:0002c460       _LocalAlloc@8              5f72d460 f   kernel32:KERNEL32.dll
 0001:0002c466       _LoadLibraryA@4            5f72d466 f   kernel32:KERNEL32.dll
 0001:0002c46c       _lstrcmpW@8                5f72d46c f   kernel32:KERNEL32.dll
 0001:0002c472       _lstrcpynW@12              5f72d472 f   kernel32:KERNEL32.dll
 0001:0002c478       _lstrlenW@4                5f72d478 f   kernel32:KERNEL32.dll
 0001:0002c47e       _WideCharToMultiByte@32    5f72d47e f   kernel32:KERNEL32.dll
 0001:0002c484       _lstrcmpA@8                5f72d484 f   kernel32:KERNEL32.dll
 0001:0002c48a       _lstrcpyW@8                5f72d48a f   kernel32:KERNEL32.dll
 0001:0002c490       _GlobalUnlock@4            5f72d490 f   kernel32:KERNEL32.dll
 0001:0002c496       _GlobalLock@4              5f72d496 f   kernel32:KERNEL32.dll
 0001:0002c49c       _GlobalAlloc@8             5f72d49c f   kernel32:KERNEL32.dll
 0001:0002c4a2       _GlobalReAlloc@12          5f72d4a2 f   kernel32:KERNEL32.dll
 0001:0002c4a8       _lstrlenA@4                5f72d4a8 f   kernel32:KERNEL32.dll
 0001:0002c4ae       _lstrcpyA@8                5f72d4ae f   kernel32:KERNEL32.dll
 0001:0002c4b4       _GlobalFree@4              5f72d4b4 f   kernel32:KERNEL32.dll
 0001:0002c4ba       _GlobalSize@4              5f72d4ba f   kernel32:KERNEL32.dll
 0001:0002c4c0       _OutputDebugStringW@4      5f72d4c0 f   kernel32:KERNEL32.dll
 0001:0002c4c6       _wsprintfW                 5f72d4c6 f   user32:USER32.dll
 0001:0002c4cc       _EnableWindow@8            5f72d4cc f   user32:USER32.dll
 0001:0002c4d2       _GetDesktopWindow@0        5f72d4d2 f   user32:USER32.dll
 0001:0002c4d8       _GetWindowTextW@12         5f72d4d8 f   user32:USER32.dll
 0001:0002c4de       _GetWindowTextLengthW@4    5f72d4de f   user32:USER32.dll
 0001:0002c4e4       _SendMessageW@16           5f72d4e4 f   user32:USER32.dll
 0001:0002c4ea       _GetWindowLongW@8          5f72d4ea f   user32:USER32.dll
 0001:0002c4f0       __imp_load__CoGetClassObject@20 5f72d4f0     ole32:ole32.dll
 0001:0002c4fc       __tailMerge_ole32          5f72d4fc     ole32:ole32.dll
 0001:0002c50a       _CoGetClassObject@20       5f72d50a     ole32:ole32.dll
 0001:0002c510       __imp_load__CoInitialize@4 5f72d510     ole32:ole32.dll
 0001:0002c51c       _CoInitialize@4            5f72d51c     ole32:ole32.dll
 0001:0002c522       __imp_load__CoUninitialize@0 5f72d522     ole32:ole32.dll
 0001:0002c52e       _CoUninitialize@0          5f72d52e     ole32:ole32.dll
 0001:0002c534       __imp_load__SysFreeString@4 5f72d534     oleaut32:OLEAUT32.dll
 0001:0002c540       __tailMerge_OLEAUT32       5f72d540     oleaut32:OLEAUT32.dll
 0001:0002c54e       _SysFreeString@4           5f72d54e     oleaut32:OLEAUT32.dll
 0001:0002c554       __imp_load__SQLError@32    5f72d554     odbc32:ODBC32.dll
 0001:0002c560       __tailMerge_ODBC32         5f72d560     odbc32:ODBC32.dll
 0001:0002c56e       _SQLError@32               5f72d56e     odbc32:ODBC32.dll
 0001:0002c574       __imp_load__SQLFreeStmt@8  5f72d574     odbc32:ODBC32.dll
 0001:0002c580       _SQLFreeStmt@8             5f72d580     odbc32:ODBC32.dll
 0001:0002c586       __imp_load__SQLCancel@4    5f72d586     odbc32:ODBC32.dll
 0001:0002c592       _SQLCancel@4               5f72d592     odbc32:ODBC32.dll
 0001:0002c598       __imp_load__SQLMoreResults@4 5f72d598     odbc32:ODBC32.dll
 0001:0002c5a4       _SQLMoreResults@4          5f72d5a4     odbc32:ODBC32.dll
 0001:0002c5aa       __imp_load__SQLFetch@4     5f72d5aa     odbc32:ODBC32.dll
 0001:0002c5b6       _SQLFetch@4                5f72d5b6     odbc32:ODBC32.dll
 0001:0002c5bc       __imp_load__SQLNumResultCols@8 5f72d5bc     odbc32:ODBC32.dll
 0001:0002c5c8       _SQLNumResultCols@8        5f72d5c8     odbc32:ODBC32.dll
 0001:0002c5ce       __imp_load__SQLExecDirect@12 5f72d5ce     odbc32:ODBC32.dll
 0001:0002c5da       _SQLExecDirect@12          5f72d5da     odbc32:ODBC32.dll
 0001:0002c5e0       __imp_load__SQLAllocStmt@8 5f72d5e0     odbc32:ODBC32.dll
 0001:0002c5ec       _SQLAllocStmt@8            5f72d5ec     odbc32:ODBC32.dll
 0001:0002c5f2       __imp_load__SQLFreeConnect@4 5f72d5f2     odbc32:ODBC32.dll
 0001:0002c5fe       _SQLFreeConnect@4          5f72d5fe     odbc32:ODBC32.dll
 0001:0002c604       __imp_load__SQLDisconnect@4 5f72d604     odbc32:ODBC32.dll
 0001:0002c610       _SQLDisconnect@4           5f72d610     odbc32:ODBC32.dll
 0001:0002c616       __imp_load__SQLFreeEnv@4   5f72d616     odbc32:ODBC32.dll
 0001:0002c622       _SQLFreeEnv@4              5f72d622     odbc32:ODBC32.dll
 0001:0002c628       __imp_load__SQLSetStmtOption@12 5f72d628     odbc32:ODBC32.dll
 0001:0002c634       _SQLSetStmtOption@12       5f72d634     odbc32:ODBC32.dll
 0001:0002c63a       __imp_load__SQLGetInfo@20  5f72d63a     odbc32:ODBC32.dll
 0001:0002c646       _SQLGetInfo@20             5f72d646     odbc32:ODBC32.dll
 0001:0002c64c       __imp_load__SQLSetConnectOption@12 5f72d64c     odbc32:ODBC32.dll
 0001:0002c658       _SQLSetConnectOption@12    5f72d658     odbc32:ODBC32.dll
 0001:0002c65e       __imp_load__SQLTransact@12 5f72d65e     odbc32:ODBC32.dll
 0001:0002c66a       _SQLTransact@12            5f72d66a     odbc32:ODBC32.dll
 0001:0002c670       __imp_load__SQLAllocConnect@8 5f72d670     odbc32:ODBC32.dll
 0001:0002c67c       _SQLAllocConnect@8         5f72d67c     odbc32:ODBC32.dll
 0001:0002c682       __imp_load__SQLAllocEnv@4  5f72d682     odbc32:ODBC32.dll
 0001:0002c68e       _SQLAllocEnv@4             5f72d68e     odbc32:ODBC32.dll
 0001:0002c694       __imp_load__SQLDriverConnect@32 5f72d694     odbc32:ODBC32.dll
 0001:0002c6a0       _SQLDriverConnect@32       5f72d6a0     odbc32:ODBC32.dll
 0001:0002c6a6       __imp_load__SQLGetData@24  5f72d6a6     odbc32:ODBC32.dll
 0001:0002c6b2       _SQLGetData@24             5f72d6b2     odbc32:ODBC32.dll
 0001:0002c6b8       __imp_load__SQLSetPos@16   5f72d6b8     odbc32:ODBC32.dll
 0001:0002c6c4       _SQLSetPos@16              5f72d6c4     odbc32:ODBC32.dll
 0001:0002c6ca       __imp_load__SQLExecute@4   5f72d6ca     odbc32:ODBC32.dll
 0001:0002c6d6       _SQLExecute@4              5f72d6d6     odbc32:ODBC32.dll
 0001:0002c6dc       __imp_load__SQLGetStmtOption@12 5f72d6dc     odbc32:ODBC32.dll
 0001:0002c6e8       _SQLGetStmtOption@12       5f72d6e8     odbc32:ODBC32.dll
 0001:0002c6ee       __imp_load__SQLPrepare@12  5f72d6ee     odbc32:ODBC32.dll
 0001:0002c6fa       _SQLPrepare@12             5f72d6fa     odbc32:ODBC32.dll
 0001:0002c700       __imp_load__SQLGetFunctions@12 5f72d700     odbc32:ODBC32.dll
 0001:0002c70c       _SQLGetFunctions@12        5f72d70c     odbc32:ODBC32.dll
 0001:0002c712       __imp_load__SQLDescribeCol@36 5f72d712     odbc32:ODBC32.dll
 0001:0002c71e       _SQLDescribeCol@36         5f72d71e     odbc32:ODBC32.dll
 0001:0002c724       __imp_load__SQLExtendedFetch@20 5f72d724     odbc32:ODBC32.dll
 0001:0002c730       _SQLExtendedFetch@20       5f72d730     odbc32:ODBC32.dll
 0001:0002c736       __imp_load__SQLGetCursorName@16 5f72d736     odbc32:ODBC32.dll
 0001:0002c742       _SQLGetCursorName@16       5f72d742     odbc32:ODBC32.dll
 0001:0002c748       __imp_load__SQLRowCount@8  5f72d748     odbc32:ODBC32.dll
 0001:0002c754       _SQLRowCount@8             5f72d754     odbc32:ODBC32.dll
 0001:0002c75a       __imp_load__SQLPutData@12  5f72d75a     odbc32:ODBC32.dll
 0001:0002c766       _SQLPutData@12             5f72d766     odbc32:ODBC32.dll
 0001:0002c76c       __imp_load__SQLParamData@8 5f72d76c     odbc32:ODBC32.dll
 0001:0002c778       _SQLParamData@8            5f72d778     odbc32:ODBC32.dll
 0001:0002c77e       __imp_load__SQLBindCol@24  5f72d77e     odbc32:ODBC32.dll
 0001:0002c78a       _SQLBindCol@24             5f72d78a     odbc32:ODBC32.dll
 0001:0002c790       __imp_load__SQLBindParameter@40 5f72d790     odbc32:ODBC32.dll
 0001:0002c79c       _SQLBindParameter@40       5f72d79c     odbc32:ODBC32.dll
 0001:0002c7a2       ___delayLoadHelper@8       5f72d7a2 f   delayimp:delayhlp.obj
 0001:0002c99b       ___FUnloadDelayLoadedDLL@4 5f72d99b f   delayimp:delayhlp.obj
 0001:0002ca4e       _GetProcAddress@8          5f72da4e f   kernel32:KERNEL32.dll
 0001:0002ca54       _InterlockedExchange@8     5f72da54 f   kernel32:KERNEL32.dll
 0001:0002ca5a       _RaiseException@16         5f72da5a f   kernel32:KERNEL32.dll
 0001:0002ca60       _GetLastError@0            5f72da60 f   kernel32:KERNEL32.dll
 0001:0002ca70       ?_GetBaseMessageMap@COleDBRecordView@@KGPBUAFX_MSGMAP@@XZ 5f72da70 f   viewoled.obj
 0001:0002ca7a       ?GetMessageMap@COleDBRecordView@@MBEPBUAFX_MSGMAP@@XZ 5f72da7a f   viewoled.obj
 0001:0002ca8a       ?OnInitialUpdate@COleDBRecordView@@UAEXXZ 5f72da8a f   viewoled.obj
 0001:0002ca9d       ?OnMove@COleDBRecordView@@UAEHI@Z 5f72da9d f   viewoled.obj
 0001:0002cc16       ?OnUpdateRecordFirst@COleDBRecordView@@IAEXPAVCCmdUI@@@Z 5f72dc16 f   viewoled.obj
 0001:0002cc3d       ?OnUpdateRecordPrev@COleDBRecordView@@IAEXPAVCCmdUI@@@Z 5f72dc3d f   viewoled.obj
 0001:0002cc64       ?OnUpdateRecordNext@COleDBRecordView@@IAEXPAVCCmdUI@@@Z 5f72dc64 f   viewoled.obj
 0001:0002cc8b       ?OnUpdateRecordLast@COleDBRecordView@@IAEXPAVCCmdUI@@@Z 5f72dc8b f   viewoled.obj
 0001:0002ccc0       _RawDllMain@12             5f72dcc0 f   dlldb.obj
 0001:0002cd7b       _DllMain@12                5f72dd7b f   dlldb.obj
 0001:0002ce3a       ?AfxDbInitModule@@YGXXZ    5f72de3a f   dlldb.obj
 0001:0002cf00       ?_GetBaseClass@CDBException@@KGPAUCRuntimeClass@@XZ 5f72df00 f   dbcore.obj
 0001:0002cf0a       ?GetRuntimeClass@CDBException@@UBEPAUCRuntimeClass@@XZ 5f72df0a f   dbcore.obj
 0001:0002cf1a       ?_GetBaseClass@CDatabase@@KGPAUCRuntimeClass@@XZ 5f72df1a f   dbcore.obj
 0001:0002cf24       ?GetRuntimeClass@CDatabase@@UBEPAUCRuntimeClass@@XZ 5f72df24 f   dbcore.obj
 0001:0002cf34       ?_GetBaseClass@CRecordset@@KGPAUCRuntimeClass@@XZ 5f72df34 f   dbcore.obj
 0001:0002cf3e       ?GetRuntimeClass@CRecordset@@UBEPAUCRuntimeClass@@XZ 5f72df3e f   dbcore.obj
 0001:0002cf90       ??1?$CProcessLocal@V_AFX_DB_STATE@@@@QAE@XZ 5f72df90 f i dbcore.obj
 0001:0002cfb0       ??B?$CProcessLocal@V_AFX_DB_STATE@@@@QAEPAV_AFX_DB_STATE@@XZ 5f72dfb0 f i dbcore.obj
 0001:0002cfd0       ?GetData@?$CProcessLocal@V_AFX_DB_STATE@@@@QAEPAV_AFX_DB_STATE@@XZ 5f72dfd0 f i dbcore.obj
 0001:0002d020       ?CreateObject@?$CProcessLocal@V_AFX_DB_STATE@@@@SGPAVCNoTrackObject@@XZ 5f72e020 f i dbcore.obj
 0001:0002d090       ??0_AFX_DB_STATE@@QAE@XZ   5f72e090 f i dbcore.obj
 0001:0002d0b0       ??_E_AFX_DB_STATE@@UAEPAXI@Z 5f72e0b0 f i dbcore.obj
 0001:0002d0b0       ??_G_AFX_DB_STATE@@UAEPAXI@Z 5f72e0b0 f i dbcore.obj
 0001:0002d0e0       ??0CNoTrackObject@@QAE@XZ  5f72e0e0 f i dbcore.obj
 0001:0002d100       ??1_AFX_DB_STATE@@UAE@XZ   5f72e100 f i dbcore.obj
 0001:0002d120       ?_GetBaseClass@CRecordView@@KGPAUCRuntimeClass@@XZ 5f72e120 f   dbview.obj
 0001:0002d12a       ?GetRuntimeClass@CRecordView@@UBEPAUCRuntimeClass@@XZ 5f72e12a f   dbview.obj
 0001:0002d140       ?_GetBaseClass@CLongBinary@@KGPAUCRuntimeClass@@XZ 5f72e140 f   dblong.obj
 0001:0002d14a       ?GetRuntimeClass@CLongBinary@@UBEPAUCRuntimeClass@@XZ 5f72e14a f   dblong.obj
 0001:0002d160       ?_GetBaseClass@COleDBRecordView@@KGPAUCRuntimeClass@@XZ 5f72e160 f   viewoled.obj
 0001:0002d16a       ?GetRuntimeClass@COleDBRecordView@@UBEPAUCRuntimeClass@@XZ 5f72e16a f   viewoled.obj
 0001:0002d180       ??C?$CComPtr@UIRowsetChange@@@ATL@@QBEPAV?$_NoAddRefReleaseOnCComPtr@UIRowsetChange@@@1@XZ 5f72e180 f i viewoled.obj
 0001:0002d180       ??C?$CComPtr@UIRowset@@@ATL@@QBEPAV?$_NoAddRefReleaseOnCComPtr@UIRowset@@@1@XZ 5f72e180 f i viewoled.obj
 0001:0002d1d0       ??B?$CComPtr@UIRowsetChange@@@ATL@@QBEPAUIRowsetChange@@XZ 5f72e1d0 f i viewoled.obj
 0001:0002d1d0       ??B?$CComPtr@UIRowset@@@ATL@@QBEPAUIRowset@@XZ 5f72e1d0 f i viewoled.obj
 0001:0002d470       ??_ECDatabase@@UAEPAXI@Z   5f72e470 f i dlldb.obj
 0001:0002d4e0       ??_ECLongBinary@@UAEPAXI@Z 5f72e4e0 f i dlldb.obj
 0001:0002d550       ??_ECDaoWorkspace@@UAEPAXI@Z 5f72e550 f i dlldb.obj
 0001:0002d5c0       ??_ECDaoException@@UAEPAXI@Z 5f72e5c0 f i dlldb.obj
 0001:0002d630       ??_ECDaoDatabase@@UAEPAXI@Z 5f72e630 f i dlldb.obj
 0001:0002d6a0       ??_FCDaoDatabase@@QAEXXZ   5f72e6a0 f i dlldb.obj
 0001:0002d6c0       ??_ECDaoRecordset@@UAEPAXI@Z 5f72e6c0 f i dlldb.obj
 0001:0002d730       ??_FCDaoRecordset@@QAEXXZ  5f72e730 f i dlldb.obj
 0001:0002d750       ??B?$CTypedSimpleList@PAUCRuntimeClass@@@@QAEPAUCRuntimeClass@@XZ 5f72e750 f i dlldb.obj
 0001:0002d750       ??B?$CTypedSimpleList@PAVCOleObjectFactory@@@@QAEPAVCOleObjectFactory@@XZ 5f72e750 f i dlldb.obj
 0002:00000000       __imp__FreeLibrary@4       5f731000     kernel32:KERNEL32.dll
 0002:00000004       __imp__GetModuleHandleA@4  5f731004     kernel32:KERNEL32.dll
 0002:00000008       __imp__LocalFree@4         5f731008     kernel32:KERNEL32.dll
 0002:0000000c       __imp__LocalAlloc@8        5f73100c     kernel32:KERNEL32.dll
 0002:00000010       __imp__LoadLibraryA@4      5f731010     kernel32:KERNEL32.dll
 0002:00000014       __imp__lstrcmpW@8          5f731014     kernel32:KERNEL32.dll
 0002:00000018       __imp__lstrcpynW@12        5f731018     kernel32:KERNEL32.dll
 0002:0000001c       __imp__lstrlenW@4          5f73101c     kernel32:KERNEL32.dll
 0002:00000020       __imp__WideCharToMultiByte@32 5f731020     kernel32:KERNEL32.dll
 0002:00000024       __imp__lstrcmpA@8          5f731024     kernel32:KERNEL32.dll
 0002:00000028       __imp__lstrcpyW@8          5f731028     kernel32:KERNEL32.dll
 0002:0000002c       __imp__GlobalUnlock@4      5f73102c     kernel32:KERNEL32.dll
 0002:00000030       __imp__GlobalLock@4        5f731030     kernel32:KERNEL32.dll
 0002:00000034       __imp__GlobalAlloc@8       5f731034     kernel32:KERNEL32.dll
 0002:00000038       __imp__GlobalReAlloc@12    5f731038     kernel32:KERNEL32.dll
 0002:0000003c       __imp__lstrlenA@4          5f73103c     kernel32:KERNEL32.dll
 0002:00000040       __imp__lstrcpyA@8          5f731040     kernel32:KERNEL32.dll
 0002:00000044       __imp__GlobalFree@4        5f731044     kernel32:KERNEL32.dll
 0002:00000048       __imp__GlobalSize@4        5f731048     kernel32:KERNEL32.dll
 0002:0000004c       __imp__OutputDebugStringW@4 5f73104c     kernel32:KERNEL32.dll
 0002:00000050       __imp__GetProcAddress@8    5f731050     kernel32:KERNEL32.dll
 0002:00000054       __imp__InterlockedExchange@8 5f731054     kernel32:KERNEL32.dll
 0002:00000058       __imp__RaiseException@16   5f731058     kernel32:KERNEL32.dll
 0002:0000005c       __imp__GetLastError@0      5f73105c     kernel32:KERNEL32.dll
 0002:00000060       \177KERNEL32_NULL_THUNK_DATA 5f731060     kernel32:KERNEL32.dll
 0002:00000064       __imp_??4CString@@QAEABV0@ABV0@@Z 5f731064     MFC42UD:MFC42uD.DLL
 0002:00000068       __imp_?Right@CString@@QBE?AV1@H@Z 5f731068     MFC42UD:MFC42uD.DLL
 0002:0000006c       __imp_?GetLength@CString@@QBEHXZ 5f73106c     MFC42UD:MFC42uD.DLL
 0002:00000070       __imp_??YCString@@QAEABV0@ABV0@@Z 5f731070     MFC42UD:MFC42uD.DLL
 0002:00000074       __imp_??H@YG?AVCString@@PBGABV0@@Z 5f731074     MFC42UD:MFC42uD.DLL
 0002:00000078       __imp_?Left@CString@@QBE?AV1@H@Z 5f731078     MFC42UD:MFC42uD.DLL
 0002:0000007c       __imp_?Find@CString@@QBEHG@Z 5f73107c     MFC42UD:MFC42uD.DLL
 0002:00000080       __imp_??ACString@@QBEGH@Z  5f731080     MFC42UD:MFC42uD.DLL
 0002:00000084       __imp_?IsEmpty@CString@@QBEHXZ 5f731084     MFC42UD:MFC42uD.DLL
 0002:00000088       __imp_??YCString@@QAEABV0@PBG@Z 5f731088     MFC42UD:MFC42uD.DLL
 0002:0000008c       __imp_??BCString@@QBEPBGXZ 5f73108c     MFC42UD:MFC42uD.DLL
 0002:00000090       __imp_??4CString@@QAEABV0@PBE@Z 5f731090     MFC42UD:MFC42uD.DLL
 0002:00000094       __imp_?AfxAssertValidObject@@YGXPBVCObject@@PBDH@Z 5f731094     MFC42UD:MFC42uD.DLL
 0002:00000098       __imp_?AfxIsValidString@@YGHPBGH@Z 5f731098     MFC42UD:MFC42uD.DLL
 0002:0000009c       __imp_??0CString@@QAE@PBG@Z 5f73109c     MFC42UD:MFC42uD.DLL
 0002:000000a0       __imp_?Empty@CString@@QAEXXZ 5f7310a0     MFC42UD:MFC42uD.DLL
 0002:000000a4       __imp_??1CObject@@UAE@XZ   5f7310a4     MFC42UD:MFC42uD.DLL
 0002:000000a8       __imp_??0CPtrList@@QAE@H@Z 5f7310a8     MFC42UD:MFC42uD.DLL
 0002:000000ac       __imp_??0CObject@@IAE@XZ   5f7310ac     MFC42UD:MFC42uD.DLL
 0002:000000b0       __imp_??1CPtrList@@UAE@XZ  5f7310b0     MFC42UD:MFC42uD.DLL
 0002:000000b4       __imp_??4CString@@QAEABV0@PBG@Z 5f7310b4     MFC42UD:MFC42uD.DLL
 0002:000000b8       __imp_?IsKindOf@CObject@@QBEHPBUCRuntimeClass@@@Z 5f7310b8     MFC42UD:MFC42uD.DLL
 0002:000000bc       __imp_?classCException@CException@@2UCRuntimeClass@@B 5f7310bc     MFC42UD:MFC42uD.DLL
 0002:000000c0       __imp_?AfxUnlockGlobals@@YGXH@Z 5f7310c0     MFC42UD:MFC42uD.DLL
 0002:000000c4       __imp_?GetHead@CPtrList@@QAEAAPAXXZ 5f7310c4     MFC42UD:MFC42uD.DLL
 0002:000000c8       __imp_?IsEmpty@CPtrList@@QBEHXZ 5f7310c8     MFC42UD:MFC42uD.DLL
 0002:000000cc       __imp_?AfxLockGlobals@@YGXH@Z 5f7310cc     MFC42UD:MFC42uD.DLL
 0002:000000d0       __imp_?Delete@CException@@QAEXXZ 5f7310d0     MFC42UD:MFC42uD.DLL
 0002:000000d4       __imp_??0CString@@QAE@PBD@Z 5f7310d4     MFC42UD:MFC42uD.DLL
 0002:000000d8       __imp_?afxTraceFlags@@3IA  5f7310d8     MFC42UD:MFC42uD.DLL
 0002:000000dc       __imp_?AfxThrowMemoryException@@YGXXZ 5f7310dc     MFC42UD:MFC42uD.DLL
 0002:000000e0       __imp_?GetSafeOwner_@CWnd@@SGPAUHWND__@@PAU2@PAPAU2@@Z 5f7310e0     MFC42UD:MFC42uD.DLL
 0002:000000e4       __imp_??4CString@@QAEABV0@PBD@Z 5f7310e4     MFC42UD:MFC42uD.DLL
 0002:000000e8       __imp_?GetDepth@CDumpContext@@QBEHXZ 5f7310e8     MFC42UD:MFC42uD.DLL
 0002:000000ec       __imp_??6CDumpContext@@QAEAAV0@K@Z 5f7310ec     MFC42UD:MFC42uD.DLL
 0002:000000f0       __imp_??6CDumpContext@@QAEAAV0@H@Z 5f7310f0     MFC42UD:MFC42uD.DLL
 0002:000000f4       __imp_??6@YGAAVCDumpContext@@AAV0@ABVCString@@@Z 5f7310f4     MFC42UD:MFC42uD.DLL
 0002:000000f8       __imp_??6CDumpContext@@QAEAAV0@PBX@Z 5f7310f8     MFC42UD:MFC42uD.DLL
 0002:000000fc       __imp_??6CDumpContext@@QAEAAV0@PBD@Z 5f7310fc     MFC42UD:MFC42uD.DLL
 0002:00000100       __imp_??1CMapPtrToPtr@@UAE@XZ 5f731100     MFC42UD:MFC42uD.DLL
 0002:00000104       __imp_?AddHead@CPtrList@@QAEPAU__POSITION@@PAX@Z 5f731104     MFC42UD:MFC42uD.DLL
 0002:00000108       __imp_?AfxIsValidAddress@@YGHPBXIH@Z 5f731108     MFC42UD:MFC42uD.DLL
 0002:0000010c       __imp_??0CMapPtrToPtr@@QAE@H@Z 5f73110c     MFC42UD:MFC42uD.DLL
 0002:00000110       __imp_?RemoveAt@CPtrList@@QAEXPAU__POSITION@@@Z 5f731110     MFC42UD:MFC42uD.DLL
 0002:00000114       __imp_?Find@CPtrList@@QBEPAU__POSITION@@PAXPAU2@@Z 5f731114     MFC42UD:MFC42uD.DLL
 0002:00000118       __imp_?Find@CString@@QBEHPBG@Z 5f731118     MFC42UD:MFC42uD.DLL
 0002:0000011c       __imp_??2@YAPAXIPBDH@Z     5f73111c     MFC42UD:MFC42uD.DLL
 0002:00000120       __imp_??3@YAXPAXPBDH@Z     5f731120     MFC42UD:MFC42uD.DLL
 0002:00000124       __imp_?GetBuffer@CString@@QAEPAGH@Z 5f731124     MFC42UD:MFC42uD.DLL
 0002:00000128       __imp_?GetBufferSetLength@CString@@QAEPAGH@Z 5f731128     MFC42UD:MFC42uD.DLL
 0002:0000012c       __imp_??9@YG_NABVCString@@0@Z 5f73112c     MFC42UD:MFC42uD.DLL
 0002:00000130       __imp_??3CObject@@SGXPAXPBDH@Z 5f731130     MFC42UD:MFC42uD.DLL
 0002:00000134       __imp_?ReleaseBuffer@CString@@QAEXH@Z 5f731134     MFC42UD:MFC42uD.DLL
 0002:00000138       __imp_?MakeUpper@CString@@QAEXXZ 5f731138     MFC42UD:MFC42uD.DLL
 0002:0000013c       __imp_?SetAt@CString@@QAEXHG@Z 5f73113c     MFC42UD:MFC42uD.DLL
 0002:00000140       __imp_?Lookup@CMapPtrToPtr@@QBEHPAXAAPAX@Z 5f731140     MFC42UD:MFC42uD.DLL
 0002:00000144       __imp_??8@YG_NABVCString@@PBG@Z 5f731144     MFC42UD:MFC42uD.DLL
 0002:00000148       __imp_??6CDumpContext@@QAEAAV0@PBVCObject@@@Z 5f731148     MFC42UD:MFC42uD.DLL
 0002:0000014c       __imp_??6CDumpContext@@QAEAAV0@J@Z 5f73114c     MFC42UD:MFC42uD.DLL
 0002:00000150       __imp_??6CDumpContext@@QAEAAV0@I@Z 5f731150     MFC42UD:MFC42uD.DLL
 0002:00000154       __imp_?classCObject@CObject@@2UCRuntimeClass@@B 5f731154     MFC42UD:MFC42uD.DLL
 0002:00000158       __imp_??1CProcessLocalObject@@QAE@XZ 5f731158     MFC42UD:MFC42uD.DLL
 0002:0000015c       __imp_?GetData@CProcessLocalObject@@QAEPAVCNoTrackObject@@P6GPAV2@XZ@Z 5f73115c     MFC42UD:MFC42uD.DLL
 0002:00000160       __imp_??3CNoTrackObject@@SGXPAX@Z 5f731160     MFC42UD:MFC42uD.DLL
 0002:00000164       __imp_??2CNoTrackObject@@SGPAXI@Z 5f731164     MFC42UD:MFC42uD.DLL
 0002:00000168       __imp_?GetData@CByteArray@@QAEPAEXZ 5f731168     MFC42UD:MFC42uD.DLL
 0002:0000016c       __imp_??YCString@@QAEABV0@D@Z 5f73116c     MFC42UD:MFC42uD.DLL
 0002:00000170       __imp_?SetAt@CMapPtrToPtr@@QAEXPAX0@Z 5f731170     MFC42UD:MFC42uD.DLL
 0002:00000174       __imp_??6CDumpContext@@QAEAAV0@PBG@Z 5f731174     MFC42UD:MFC42uD.DLL
 0002:00000178       __imp_?LockBuffer@CString@@QAEPAGXZ 5f731178     MFC42UD:MFC42uD.DLL
 0002:0000017c       __imp_??6CDumpContext@@QAEAAV0@E@Z 5f73117c     MFC42UD:MFC42uD.DLL
 0002:00000180       __imp_??0CByteArray@@QAE@XZ 5f731180     MFC42UD:MFC42uD.DLL
 0002:00000184       __imp_?SetSize@CByteArray@@QAEXHH@Z 5f731184     MFC42UD:MFC42uD.DLL
 0002:00000188       __imp_??ACByteArray@@QAEAAEH@Z 5f731188     MFC42UD:MFC42uD.DLL
 0002:0000018c       __imp_?GetSize@CByteArray@@QBEHXZ 5f73118c     MFC42UD:MFC42uD.DLL
 0002:00000190       __imp_??6@YGAAVCDumpContext@@AAV0@VCTime@@@Z 5f731190     MFC42UD:MFC42uD.DLL
 0002:00000194       __imp_??0CTime@@QAE@XZ     5f731194     MFC42UD:MFC42uD.DLL
 0002:00000198       __imp_??9CTime@@QBEHV0@@Z  5f731198     MFC42UD:MFC42uD.DLL
 0002:0000019c       __imp_??0CTime@@QAE@ABV0@@Z 5f73119c     MFC42UD:MFC42uD.DLL
 0002:000001a0       __imp_??0CTime@@QAE@HHHHHHH@Z 5f7311a0     MFC42UD:MFC42uD.DLL
 0002:000001a4       __imp_??4CTime@@QAEABV0@ABV0@@Z 5f7311a4     MFC42UD:MFC42uD.DLL
 0002:000001a8       __imp_??0CTime@@QAE@J@Z    5f7311a8     MFC42UD:MFC42uD.DLL
 0002:000001ac       __imp_?GetSecond@CTime@@QBEHXZ 5f7311ac     MFC42UD:MFC42uD.DLL
 0002:000001b0       __imp_?GetMinute@CTime@@QBEHXZ 5f7311b0     MFC42UD:MFC42uD.DLL
 0002:000001b4       __imp_?GetHour@CTime@@QBEHXZ 5f7311b4     MFC42UD:MFC42uD.DLL
 0002:000001b8       __imp_?GetDay@CTime@@QBEHXZ 5f7311b8     MFC42UD:MFC42uD.DLL
 0002:000001bc       __imp_?GetMonth@CTime@@QBEHXZ 5f7311bc     MFC42UD:MFC42uD.DLL
 0002:000001c0       __imp_?GetYear@CTime@@QBEHXZ 5f7311c0     MFC42UD:MFC42uD.DLL
 0002:000001c4       __imp_??6CDumpContext@@QAEAAV0@G@Z 5f7311c4     MFC42UD:MFC42uD.DLL
 0002:000001c8       __imp_??8CTime@@QBEHV0@@Z  5f7311c8     MFC42UD:MFC42uD.DLL
 0002:000001cc       __imp_??8@YG_NABVCString@@0@Z 5f7311cc     MFC42UD:MFC42uD.DLL
 0002:000001d0       __imp_?Copy@CByteArray@@QAEXABV1@@Z 5f7311d0     MFC42UD:MFC42uD.DLL
 0002:000001d4       __imp_?messageMap@CFormView@@1UAFX_MSGMAP@@B 5f7311d4     MFC42UD:MFC42uD.DLL
 0002:000001d8       __imp_?OnEndPrintPreview@CView@@MAEXPAVCDC@@PAUCPrintInfo@@UtagPOINT@@PAVCPreviewView@@@Z 5f7311d8     MFC42UD:MFC42uD.DLL
 0002:000001dc       __imp_?OnEndPrinting@CView@@MAEXPAVCDC@@PAUCPrintInfo@@@Z 5f7311dc     MFC42UD:MFC42uD.DLL
 0002:000001e0       __imp_?OnPrint@CView@@MAEXPAVCDC@@PAUCPrintInfo@@@Z 5f7311e0     MFC42UD:MFC42uD.DLL
 0002:000001e4       __imp_?OnBeginPrinting@CView@@MAEXPAVCDC@@PAUCPrintInfo@@@Z 5f7311e4     MFC42UD:MFC42uD.DLL
 0002:000001e8       __imp_?OnPreparePrinting@CView@@MAEHPAUCPrintInfo@@@Z 5f7311e8     MFC42UD:MFC42uD.DLL
 0002:000001ec       __imp_?OnDraw@CFormView@@MAEXPAVCDC@@@Z 5f7311ec     MFC42UD:MFC42uD.DLL
 0002:000001f0       __imp_??0CException@@QAE@XZ 5f7311f0     MFC42UD:MFC42uD.DLL
 0002:000001f4       __imp_??H@YG?AVCString@@ABV0@PBG@Z 5f7311f4     MFC42UD:MFC42uD.DLL
 0002:000001f8       __imp_?OnActivateView@CFormView@@MAEXHPAVCView@@0@Z 5f7311f8     MFC42UD:MFC42uD.DLL
 0002:000001fc       __imp_?OnPrepareDC@CScrollView@@UAEXPAVCDC@@PAUCPrintInfo@@@Z 5f7311fc     MFC42UD:MFC42uD.DLL
 0002:00000200       __imp_?OnDragScroll@CView@@UAEKKVCPoint@@@Z 5f731200     MFC42UD:MFC42uD.DLL
 0002:00000204       __imp_?OnDropEx@CView@@UAEKPAVCOleDataObject@@KKVCPoint@@@Z 5f731204     MFC42UD:MFC42uD.DLL
 0002:00000208       __imp_?OnDrop@CView@@UAEHPAVCOleDataObject@@KVCPoint@@@Z 5f731208     MFC42UD:MFC42uD.DLL
 0002:0000020c       __imp_?OnDragLeave@CView@@UAEXXZ 5f73120c     MFC42UD:MFC42uD.DLL
 0002:00000210       __imp_?OnDragOver@CView@@UAEKPAVCOleDataObject@@KVCPoint@@@Z 5f731210     MFC42UD:MFC42uD.DLL
 0002:00000214       __imp_?OnDragEnter@CView@@UAEKPAVCOleDataObject@@KVCPoint@@@Z 5f731214     MFC42UD:MFC42uD.DLL
 0002:00000218       __imp_?OnScrollBy@CScrollView@@UAEHVCSize@@H@Z 5f731218     MFC42UD:MFC42uD.DLL
 0002:0000021c       __imp_?OnScroll@CScrollView@@UAEHIIH@Z 5f73121c     MFC42UD:MFC42uD.DLL
 0002:00000220       __imp_?IsSelected@CView@@UBEHPBVCObject@@@Z 5f731220     MFC42UD:MFC42uD.DLL
 0002:00000224       __imp_?SetOccDialogInfo@CFormView@@MAEHPAU_AFX_OCC_DIALOG_INFO@@@Z 5f731224     MFC42UD:MFC42uD.DLL
 0002:00000228       __imp_?IsFrameWnd@CWnd@@UBEHXZ 5f731228     MFC42UD:MFC42uD.DLL
 0002:0000022c       __imp_?CheckAutoCenter@CWnd@@UAEHXZ 5f73122c     MFC42UD:MFC42uD.DLL
 0002:00000230       __imp_?OnChildNotify@CWnd@@MAEHIIJPAJ@Z 5f731230     MFC42UD:MFC42uD.DLL
 0002:00000234       __imp_?PostNcDestroy@CView@@MAEXXZ 5f731234     MFC42UD:MFC42uD.DLL
 0002:00000238       __imp_?DefWindowProcW@CWnd@@MAEJIIJ@Z 5f731238     MFC42UD:MFC42uD.DLL
 0002:0000023c       __imp_?OnWndMsg@CWnd@@MAEHIIJPAJ@Z 5f73123c     MFC42UD:MFC42uD.DLL
 0002:00000240       __imp_?WindowProc@CWnd@@MAEJIIJ@Z 5f731240     MFC42UD:MFC42uD.DLL
 0002:00000244       __imp_?OnAmbientProperty@CWnd@@UAEHPAVCOleControlSite@@JPAUtagVARIANT@@@Z 5f731244     MFC42UD:MFC42uD.DLL
 0002:00000248       __imp_?PreTranslateMessage@CFormView@@MAEHPAUtagMSG@@@Z 5f731248     MFC42UD:MFC42uD.DLL
 0002:0000024c       __imp_?EndModalState@CWnd@@UAEXXZ 5f73124c     MFC42UD:MFC42uD.DLL
 0002:00000250       __imp_?BeginModalState@CWnd@@UAEXXZ 5f731250     MFC42UD:MFC42uD.DLL
 0002:00000254       __imp_?DoDataExchange@CWnd@@MAEXPAVCDataExchange@@@Z 5f731254     MFC42UD:MFC42uD.DLL
 0002:00000258       __imp_?GetSuperWndProcAddr@CWnd@@MAEPAP6GJPAUHWND__@@IIJ@ZXZ 5f731258     MFC42UD:MFC42uD.DLL
 0002:0000025c       __imp_?OnNotify@CWnd@@MAEHIJPAJ@Z 5f73125c     MFC42UD:MFC42uD.DLL
 0002:00000260       __imp_?OnCommand@CWnd@@MAEHIJ@Z 5f731260     MFC42UD:MFC42uD.DLL
 0002:00000264       __imp_?EndModalLoop@CWnd@@UAEXH@Z 5f731264     MFC42UD:MFC42uD.DLL
 0002:00000268       __imp_?ContinueModal@CWnd@@UAEHXZ 5f731268     MFC42UD:MFC42uD.DLL
 0002:0000026c       __imp_?WinHelpW@CWnd@@UAEXKI@Z 5f73126c     MFC42UD:MFC42uD.DLL
 0002:00000270       __imp_?GetScrollBarCtrl@CView@@UBEPAVCScrollBar@@H@Z 5f731270     MFC42UD:MFC42uD.DLL
 0002:00000274       __imp_?OnToolHitTest@CWnd@@UBEHVCPoint@@PAUtagTOOLINFOW@@@Z 5f731274     MFC42UD:MFC42uD.DLL
 0002:00000278       __imp_?CalcWindowRect@CScrollView@@UAEXPAUtagRECT@@I@Z 5f731278     MFC42UD:MFC42uD.DLL
 0002:0000027c       __imp_?PreCreateWindow@CView@@MAEHAAUtagCREATESTRUCTW@@@Z 5f73127c     MFC42UD:MFC42uD.DLL
 0002:00000280       __imp_?DestroyWindow@CWnd@@UAEHXZ 5f731280     MFC42UD:MFC42uD.DLL
 0002:00000284       __imp_?Create@CFormView@@MAEHPBG0KABUtagRECT@@PAVCWnd@@IPAUCCreateContext@@@Z 5f731284     MFC42UD:MFC42uD.DLL
 0002:00000288       __imp_?PreSubclassWindow@CWnd@@UAEXXZ 5f731288     MFC42UD:MFC42uD.DLL
 0002:0000028c       __imp_?GetConnectionHook@CCmdTarget@@MAEPAUIConnectionPoint@@ABU_GUID@@@Z 5f73128c     MFC42UD:MFC42uD.DLL
 0002:00000290       __imp_?GetExtraConnectionPoints@CCmdTarget@@MAEHPAVCPtrArray@@@Z 5f731290     MFC42UD:MFC42uD.DLL
 0002:00000294       __imp_?AfxGetModuleState@@YGPAVAFX_MODULE_STATE@@XZ 5f731294     MFC42UD:MFC42uD.DLL
 0002:00000298       __imp_?OnCreateAggregates@CCmdTarget@@UAEHXZ 5f731298     MFC42UD:MFC42uD.DLL
 0002:0000029c       __imp_?GetEventSinkMap@CCmdTarget@@MBEPBUAFX_EVENTSINKMAP@@XZ 5f73129c     MFC42UD:MFC42uD.DLL
 0002:000002a0       __imp_?GetInterfaceMap@CCmdTarget@@MBEPBUAFX_INTERFACEMAP@@XZ 5f7312a0     MFC42UD:MFC42uD.DLL
 0002:000002a4       __imp_?GetConnectionMap@CCmdTarget@@MBEPBUAFX_CONNECTIONMAP@@XZ 5f7312a4     MFC42UD:MFC42uD.DLL
 0002:000002a8       __imp_?GetDispatchMap@CCmdTarget@@MBEPBUAFX_DISPMAP@@XZ 5f7312a8     MFC42UD:MFC42uD.DLL
 0002:000002ac       __imp_?GetCommandMap@CCmdTarget@@MBEPBUAFX_OLECMDMAP@@XZ 5f7312ac     MFC42UD:MFC42uD.DLL
 0002:000002b0       __imp_?GetTypeLib@CCmdTarget@@UAEJKPAPAUITypeLib@@@Z 5f7312b0     MFC42UD:MFC42uD.DLL
 0002:000002b4       __imp_?GetTypeLibCache@CCmdTarget@@UAEPAVCTypeLibCache@@XZ 5f7312b4     MFC42UD:MFC42uD.DLL
 0002:000002b8       __imp_?GetTypeInfoCount@CCmdTarget@@UAEIXZ 5f7312b8     MFC42UD:MFC42uD.DLL
 0002:000002bc       __imp_?GetDispatchIID@CCmdTarget@@UAEHPAU_GUID@@@Z 5f7312bc     MFC42UD:MFC42uD.DLL
 0002:000002c0       __imp_?IsInvokeAllowed@CCmdTarget@@UAEHJ@Z 5f7312c0     MFC42UD:MFC42uD.DLL
 0002:000002c4       __imp_?OnFinalRelease@CWnd@@UAEXXZ 5f7312c4     MFC42UD:MFC42uD.DLL
 0002:000002c8       __imp_?OnCmdMsg@CView@@UAEHIHPAXPAUAFX_CMDHANDLERINFO@@@Z 5f7312c8     MFC42UD:MFC42uD.DLL
 0002:000002cc       __imp_??0CFormView@@IAE@PBG@Z 5f7312cc     MFC42UD:MFC42uD.DLL
 0002:000002d0       __imp_??0CFormView@@IAE@I@Z 5f7312d0     MFC42UD:MFC42uD.DLL
 0002:000002d4       __imp_??1CScrollView@@UAE@XZ 5f7312d4     MFC42UD:MFC42uD.DLL
 0002:000002d8       __imp_?OnInitialUpdate@CFormView@@UAEXXZ 5f7312d8     MFC42UD:MFC42uD.DLL
 0002:000002dc       __imp_??1CWaitCursor@@QAE@XZ 5f7312dc     MFC42UD:MFC42uD.DLL
 0002:000002e0       __imp_??0CWaitCursor@@QAE@XZ 5f7312e0     MFC42UD:MFC42uD.DLL
 0002:000002e4       __imp_?UpdateData@CWnd@@QAEHH@Z 5f7312e4     MFC42UD:MFC42uD.DLL
 0002:000002e8       __imp_?AfxSetWindowText@@YGXPAUHWND__@@PBG@Z 5f7312e8     MFC42UD:MFC42uD.DLL
 0002:000002ec       __imp_?PrepareEditCtrl@CDataExchange@@QAEPAUHWND__@@H@Z 5f7312ec     MFC42UD:MFC42uD.DLL
 0002:000002f0       __imp_?DDX_Text@@YGXPAVCDataExchange@@HAAH@Z 5f7312f0     MFC42UD:MFC42uD.DLL
 0002:000002f4       __imp_?DDX_Text@@YGXPAVCDataExchange@@HAAE@Z 5f7312f4     MFC42UD:MFC42uD.DLL
 0002:000002f8       __imp_?DDX_Text@@YGXPAVCDataExchange@@HAAI@Z 5f7312f8     MFC42UD:MFC42uD.DLL
 0002:000002fc       __imp_?DDX_Text@@YGXPAVCDataExchange@@HAAJ@Z 5f7312fc     MFC42UD:MFC42uD.DLL
 0002:00000300       __imp_?DDX_Text@@YGXPAVCDataExchange@@HAAK@Z 5f731300     MFC42UD:MFC42uD.DLL
 0002:00000304       __imp_?AfxFailMaxChars@@YGXPAVCDataExchange@@H@Z 5f731304     MFC42UD:MFC42uD.DLL
 0002:00000308       __imp_?GetAllocLength@CString@@QBEHXZ 5f731308     MFC42UD:MFC42uD.DLL
 0002:0000030c       __imp_?PrepareCtrl@CDataExchange@@QAEPAUHWND__@@H@Z 5f73130c     MFC42UD:MFC42uD.DLL
 0002:00000310       __imp_?DDX_LBIndex@@YGXPAVCDataExchange@@HAAH@Z 5f731310     MFC42UD:MFC42uD.DLL
 0002:00000314       __imp_?DDX_CBIndex@@YGXPAVCDataExchange@@HAAH@Z 5f731314     MFC42UD:MFC42uD.DLL
 0002:00000318       __imp_?DDX_Scroll@@YGXPAVCDataExchange@@HAAH@Z 5f731318     MFC42UD:MFC42uD.DLL
 0002:0000031c       __imp_?AfxFailRadio@@YGXPAVCDataExchange@@@Z 5f73131c     MFC42UD:MFC42uD.DLL
 0002:00000320       __imp_?DDX_Radio@@YGXPAVCDataExchange@@HAAH@Z 5f731320     MFC42UD:MFC42uD.DLL
 0002:00000324       __imp_?AssertValid@CFormView@@UBEXXZ 5f731324     MFC42UD:MFC42uD.DLL
 0002:00000328       __imp_?Dump@CFormView@@UBEXAAVCDumpContext@@@Z 5f731328     MFC42UD:MFC42uD.DLL
 0002:0000032c       __imp_?OnMove@CWnd@@IAEXHH@Z 5f73132c     MFC42UD:MFC42uD.DLL
 0002:00000330       __imp_?classCFormView@CFormView@@2UCRuntimeClass@@B 5f731330     MFC42UD:MFC42uD.DLL
 0002:00000334       __imp_??6CDumpContext@@QAEAAV0@M@Z 5f731334     MFC42UD:MFC42uD.DLL
 0002:00000338       __imp_??6CDumpContext@@QAEAAV0@N@Z 5f731338     MFC42UD:MFC42uD.DLL
 0002:0000033c       __imp_?AfxTextFloatFormat@@YGXPAVCDataExchange@@HPAXNH@Z 5f73133c     MFC42UD:MFC42uD.DLL
 0002:00000340       __imp_?IsEmpty@CMapPtrToPtr@@QBEHXZ 5f731340     MFC42UD:MFC42uD.DLL
 0002:00000344       __imp_?RemoveKey@CMapPtrToPtr@@QAEHPAX@Z 5f731344     MFC42UD:MFC42uD.DLL
 0002:00000348       __imp_?RemoveAll@CMapPtrToPtr@@QAEXXZ 5f731348     MFC42UD:MFC42uD.DLL
 0002:0000034c       __imp_?GetNextAssoc@CMapPtrToPtr@@QBEXAAPAU__POSITION@@AAPAX1@Z 5f73134c     MFC42UD:MFC42uD.DLL
 0002:00000350       __imp_?GetStartPosition@CMapPtrToPtr@@QBEPAU__POSITION@@XZ 5f731350     MFC42UD:MFC42uD.DLL
 0002:00000354       __imp_??0CString@@QAE@ABV0@@Z 5f731354     MFC42UD:MFC42uD.DLL
 0002:00000358       __imp_??3CNoTrackObject@@SGXPAXPBDH@Z 5f731358     MFC42UD:MFC42uD.DLL
 0002:0000035c       __imp_??2CNoTrackObject@@SGPAXIPBDH@Z 5f73135c     MFC42UD:MFC42uD.DLL
 0002:00000360       __imp_?AfxGetApp@@YGPAVCWinApp@@XZ 5f731360     MFC42UD:MFC42uD.DLL
 0002:00000364       __imp_??6CDumpContext@@QAEAAV0@ABVCObject@@@Z 5f731364     MFC42UD:MFC42uD.DLL
 0002:00000368       __imp_?DDX_Text@@YGXPAVCDataExchange@@HAAF@Z 5f731368     MFC42UD:MFC42uD.DLL
 0002:0000036c       __imp_?DDX_Text@@YGXPAVCDataExchange@@HAAM@Z 5f73136c     MFC42UD:MFC42uD.DLL
 0002:00000370       __imp_?DDX_Text@@YGXPAVCDataExchange@@HAAN@Z 5f731370     MFC42UD:MFC42uD.DLL
 0002:00000374       __imp_?DDX_Text@@YGXPAVCDataExchange@@HAAVCString@@@Z 5f731374     MFC42UD:MFC42uD.DLL
 0002:00000378       __imp_?DDX_Text@@YGXPAVCDataExchange@@HPAGH@Z 5f731378     MFC42UD:MFC42uD.DLL
 0002:0000037c       __imp_?DDX_Slider@@YGXPAVCDataExchange@@HAAH@Z 5f73137c     MFC42UD:MFC42uD.DLL
 0002:00000380       __imp_??0CString@@QAE@XZ   5f731380     MFC42UD:MFC42uD.DLL
 0002:00000384       __imp_??1CException@@UAE@XZ 5f731384     MFC42UD:MFC42uD.DLL
 0002:00000388       __imp_??1CString@@QAE@XZ   5f731388     MFC42UD:MFC42uD.DLL
 0002:0000038c       __imp_?Serialize@CObject@@UAEXAAVCArchive@@@Z 5f73138c     MFC42UD:MFC42uD.DLL
 0002:00000390       __imp_?AssertValid@CObject@@UBEXXZ 5f731390     MFC42UD:MFC42uD.DLL
 0002:00000394       __imp_?Dump@CObject@@UBEXAAVCDumpContext@@@Z 5f731394     MFC42UD:MFC42uD.DLL
 0002:00000398       __imp_?ReportError@CException@@UAEHII@Z 5f731398     MFC42UD:MFC42uD.DLL
 0002:0000039c       __imp_??2CObject@@SGPAXIPBDH@Z 5f73139c     MFC42UD:MFC42uD.DLL
 0002:000003a0       __imp_?LoadStringW@CString@@QAEHI@Z 5f7313a0     MFC42UD:MFC42uD.DLL
 0002:000003a4       __imp_?AfxTrace@@YAXPBGZZ  5f7313a4     MFC42UD:MFC42uD.DLL
 0002:000003a8       __imp_??3CException@@SGXPAXPBDH@Z 5f7313a8     MFC42UD:MFC42uD.DLL
 0002:000003ac       __imp_??3CException@@SGXPAX@Z 5f7313ac     MFC42UD:MFC42uD.DLL
 0002:000003b0       __imp_??2@YAPAXI@Z         5f7313b0     MFC42UD:MFC42uD.DLL
 0002:000003b4       __imp_??3@YAXPAX@Z         5f7313b4     MFC42UD:MFC42uD.DLL
 0002:000003b8       __imp_?AfxGetAppModuleState@@YGPAVAFX_MODULE_STATE@@XZ 5f7313b8     MFC42UD:MFC42uD.DLL
 0002:000003bc       __imp_??3CObject@@SGXPAX@Z 5f7313bc     MFC42UD:MFC42uD.DLL
 0002:000003c0       __imp_?AfxInitExtensionModule@@YGHAAUAFX_EXTENSION_MODULE@@PAUHINSTANCE__@@@Z 5f7313c0     MFC42UD:MFC42uD.DLL
 0002:000003c4       __imp_?AfxAssertFailedLine@@YGHPBDH@Z 5f7313c4     MFC42UD:MFC42uD.DLL
 0002:000003c8       __imp_??2CObject@@SGPAXI@Z 5f7313c8     MFC42UD:MFC42uD.DLL
 0002:000003cc       __imp_??0CDynLinkLibrary@@QAE@AAUAFX_EXTENSION_MODULE@@H@Z 5f7313cc     MFC42UD:MFC42uD.DLL
 0002:000003d0       __imp_?AfxTermExtensionModule@@YGXAAUAFX_EXTENSION_MODULE@@H@Z 5f7313d0     MFC42UD:MFC42uD.DLL
 0002:000003d4       __imp_?AfxTermThread@@YGXPAUHINSTANCE__@@@Z 5f7313d4     MFC42UD:MFC42uD.DLL
 0002:000003d8       __imp_?OnActivateFrame@CFormView@@MAEXIPAVCFrameWnd@@@Z 5f7313d8     MFC42UD:MFC42uD.DLL
 0002:000003dc       __imp_?OnUpdate@CView@@MAEXPAV1@JPAVCObject@@@Z 5f7313dc     MFC42UD:MFC42uD.DLL
 0002:000003e0       __imp_?GetInterfaceHook@CCmdTarget@@UAEPAUIUnknown@@PBX@Z 5f7313e0     MFC42UD:MFC42uD.DLL
 0002:000003e4       \177MFC42uD_NULL_THUNK_DATA 5f7313e4     MFC42UD:MFC42uD.DLL
 0002:000003e8       __imp_??0COleDateTime@@QAE@HHHHHH@Z 5f7313e8     MFCO42UD:MFCO42uD.DLL
 0002:000003ec       __imp_??0COleVariant@@QAE@FG@Z 5f7313ec     MFCO42UD:MFCO42uD.DLL
 0002:000003f0       __imp_??0COleVariant@@QAE@ABUtagVARIANT@@@Z 5f7313f0     MFCO42UD:MFCO42uD.DLL
 0002:000003f4       __imp_??4COleVariant@@QAEABV0@QBG@Z 5f7313f4     MFCO42UD:MFCO42uD.DLL
 0002:000003f8       __imp_?SetStatus@COleCurrency@@QAEXW4CurrencyStatus@1@@Z 5f7313f8     MFCO42UD:MFCO42uD.DLL
 0002:000003fc       __imp_?GetStatus@COleCurrency@@QBE?AW4CurrencyStatus@1@XZ 5f7313fc     MFCO42UD:MFCO42uD.DLL
 0002:00000400       __imp_??0COleCurrency@@QAE@XZ 5f731400     MFCO42UD:MFCO42uD.DLL
 0002:00000404       __imp_??4COleCurrency@@QAEABV0@ABV0@@Z 5f731404     MFCO42UD:MFCO42uD.DLL
 0002:00000408       __imp_??9COleDateTime@@QBEHABV0@@Z 5f731408     MFCO42UD:MFCO42uD.DLL
 0002:0000040c       __imp_??9COleCurrency@@QBEHABV0@@Z 5f73140c     MFCO42UD:MFCO42uD.DLL
 0002:00000410       __imp_??4COleVariant@@QAEABV0@ABVCOleDateTime@@@Z 5f731410     MFCO42UD:MFCO42uD.DLL
 0002:00000414       __imp_??4COleVariant@@QAEABV0@N@Z 5f731414     MFCO42UD:MFCO42uD.DLL
 0002:00000418       __imp_??4COleVariant@@QAEABV0@M@Z 5f731418     MFCO42UD:MFCO42uD.DLL
 0002:0000041c       __imp_??4COleVariant@@QAEABV0@ABVCOleCurrency@@@Z 5f73141c     MFCO42UD:MFCO42uD.DLL
 0002:00000420       __imp_??4COleVariant@@QAEABV0@F@Z 5f731420     MFCO42UD:MFCO42uD.DLL
 0002:00000424       __imp_??4COleVariant@@QAEABV0@E@Z 5f731424     MFCO42UD:MFCO42uD.DLL
 0002:00000428       __imp_??4COleVariant@@QAEABV0@ABVCLongBinary@@@Z 5f731428     MFCO42UD:MFCO42uD.DLL
 0002:0000042c       __imp_??4COleVariant@@QAEABV0@ABVCByteArray@@@Z 5f73142c     MFCO42UD:MFCO42uD.DLL
 0002:00000430       __imp_??6@YGAAVCDumpContext@@AAV0@VCOleCurrency@@@Z 5f731430     MFCO42UD:MFCO42uD.DLL
 0002:00000434       __imp_??0COleCurrency@@QAE@ABV0@@Z 5f731434     MFCO42UD:MFCO42uD.DLL
 0002:00000438       __imp_??4COleVariant@@QAEABV0@ABV0@@Z 5f731438     MFCO42UD:MFCO42uD.DLL
 0002:0000043c       __imp_??8COleVariant@@QBEHABUtagVARIANT@@@Z 5f73143c     MFCO42UD:MFCO42uD.DLL
 0002:00000440       __imp_?DDX_Text@@YGXPAVCDataExchange@@HAAVCOleCurrency@@@Z 5f731440     MFCO42UD:MFCO42uD.DLL
 0002:00000444       __imp_?DDX_Text@@YGXPAVCDataExchange@@HAAVCOleDateTime@@@Z 5f731444     MFCO42UD:MFCO42uD.DLL
 0002:00000448       __imp_??BCOleVariant@@QAEPAUtagVARIANT@@XZ 5f731448     MFCO42UD:MFCO42uD.DLL
 0002:0000044c       __imp_??4COleDateTime@@QAEABV0@ABUtagVARIANT@@@Z 5f73144c     MFCO42UD:MFCO42uD.DLL
 0002:00000450       __imp_?Format@COleDateTime@@QBE?AVCString@@KK@Z 5f731450     MFCO42UD:MFCO42uD.DLL
 0002:00000454       __imp_?SetStatus@COleDateTime@@QAEXW4DateTimeStatus@1@@Z 5f731454     MFCO42UD:MFCO42uD.DLL
 0002:00000458       __imp_?GetStatus@COleDateTime@@QBE?AW4DateTimeStatus@1@XZ 5f731458     MFCO42UD:MFCO42uD.DLL
 0002:0000045c       __imp_?GetSecond@COleDateTime@@QBEHXZ 5f73145c     MFCO42UD:MFCO42uD.DLL
 0002:00000460       __imp_?GetMinute@COleDateTime@@QBEHXZ 5f731460     MFCO42UD:MFCO42uD.DLL
 0002:00000464       __imp_??0COleDateTime@@QAE@XZ 5f731464     MFCO42UD:MFCO42uD.DLL
 0002:00000468       __imp_?GetDay@COleDateTime@@QBEHXZ 5f731468     MFCO42UD:MFCO42uD.DLL
 0002:0000046c       __imp_?GetMonth@COleDateTime@@QBEHXZ 5f73146c     MFCO42UD:MFCO42uD.DLL
 0002:00000470       __imp_??4COleDateTime@@QAEABV0@ABV0@@Z 5f731470     MFCO42UD:MFCO42uD.DLL
 0002:00000474       __imp_?GetHour@COleDateTime@@QBEHXZ 5f731474     MFCO42UD:MFCO42uD.DLL
 0002:00000478       __imp_??4COleVariant@@QAEABV0@J@Z 5f731478     MFCO42UD:MFCO42uD.DLL
 0002:0000047c       __imp_??8COleDateTime@@QBEHABV0@@Z 5f73147c     MFCO42UD:MFCO42uD.DLL
 0002:00000480       __imp_??6@YGAAVCDumpContext@@AAV0@VCOleDateTime@@@Z 5f731480     MFCO42UD:MFCO42uD.DLL
 0002:00000484       __imp_??0COleDateTime@@QAE@N@Z 5f731484     MFCO42UD:MFCO42uD.DLL
 0002:00000488       __imp_?GetYear@COleDateTime@@QBEHXZ 5f731488     MFCO42UD:MFCO42uD.DLL
 0002:0000048c       __imp_??0COleVariant@@QAE@PBGG@Z 5f73148c     MFCO42UD:MFCO42uD.DLL
 0002:00000490       __imp_??1COleVariant@@QAE@XZ 5f731490     MFCO42UD:MFCO42uD.DLL
 0002:00000494       __imp_??6@YGAAVCDumpContext@@AAV0@VCOleVariant@@@Z 5f731494     MFCO42UD:MFCO42uD.DLL
 0002:00000498       __imp_??0COleDateTime@@QAE@ABV0@@Z 5f731498     MFCO42UD:MFCO42uD.DLL
 0002:0000049c       __imp_??0COleVariant@@QAE@JG@Z 5f73149c     MFCO42UD:MFCO42uD.DLL
 0002:000004a0       __imp_?Clear@COleVariant@@QAEXXZ 5f7314a0     MFCO42UD:MFCO42uD.DLL
 0002:000004a4       __imp_??0COleVariant@@QAE@XZ 5f7314a4     MFCO42UD:MFCO42uD.DLL
 0002:000004a8       __imp_??0COleVariant@@QAE@ABV0@@Z 5f7314a8     MFCO42UD:MFCO42uD.DLL
 0002:000004ac       \177MFCO42uD_NULL_THUNK_DATA 5f7314ac     MFCO42UD:MFCO42uD.DLL
 0002:000004b0       __imp___malloc_dbg         5f7314b0     msvcrtd:MSVCRTD.dll
 0002:000004b4       __imp_??1type_info@@UAE@XZ 5f7314b4     msvcrtd:MSVCRTD.dll
 0002:000004b8       __imp__memcmp              5f7314b8     msvcrtd:MSVCRTD.dll
 0002:000004bc       __imp___adjust_fdiv        5f7314bc     msvcrtd:MSVCRTD.dll
 0002:000004c0       __imp___onexit             5f7314c0     msvcrtd:MSVCRTD.dll
 0002:000004c4       __imp___initterm           5f7314c4     msvcrtd:MSVCRTD.dll
 0002:000004c8       __imp___free_dbg           5f7314c8     msvcrtd:MSVCRTD.dll
 0002:000004cc       __imp___vsnwprintf         5f7314cc     msvcrtd:MSVCRTD.dll
 0002:000004d0       __imp_?terminate@@YAXXZ    5f7314d0     msvcrtd:MSVCRTD.dll
 0002:000004d4       __imp___except_handler3    5f7314d4     msvcrtd:MSVCRTD.dll
 0002:000004d8       __imp__wcsstr              5f7314d8     msvcrtd:MSVCRTD.dll
 0002:000004dc       __imp__labs                5f7314dc     msvcrtd:MSVCRTD.dll
 0002:000004e0       __imp__abs                 5f7314e0     msvcrtd:MSVCRTD.dll
 0002:000004e4       __imp___CrtDbgReport       5f7314e4     msvcrtd:MSVCRTD.dll
 0002:000004e8       __imp__memcpy              5f7314e8     msvcrtd:MSVCRTD.dll
 0002:000004ec       __imp__memset              5f7314ec     msvcrtd:MSVCRTD.dll
 0002:000004f0       __imp____CxxFrameHandler   5f7314f0     msvcrtd:MSVCRTD.dll
 0002:000004f4       __imp___wcsnicmp           5f7314f4     msvcrtd:MSVCRTD.dll
 0002:000004f8       __imp___CxxThrowException@8 5f7314f8     msvcrtd:MSVCRTD.dll
 0002:000004fc       __imp___purecall           5f7314fc     msvcrtd:MSVCRTD.dll
 0002:00000500       __imp____dllonexit         5f731500     msvcrtd:MSVCRTD.dll
 0002:00000504       \177MSVCRTD_NULL_THUNK_DATA 5f731504     msvcrtd:MSVCRTD.dll
 0002:00000508       __imp__SendMessageW@16     5f731508     user32:USER32.dll
 0002:0000050c       __imp__GetWindowLongW@8    5f73150c     user32:USER32.dll
 0002:00000510       __imp__GetWindowTextW@12   5f731510     user32:USER32.dll
 0002:00000514       __imp__GetDesktopWindow@0  5f731514     user32:USER32.dll
 0002:00000518       __imp__EnableWindow@8      5f731518     user32:USER32.dll
 0002:0000051c       __imp__wsprintfW           5f73151c     user32:USER32.dll
 0002:00000520       __imp__GetWindowTextLengthW@4 5f731520     user32:USER32.dll
 0002:00000524       \177USER32_NULL_THUNK_DATA 5f731524     user32:USER32.dll
 0002:00000550       _IID_IDocHostUIHandlerDispatch 5f731550     dlldb.obj
 0002:00000560       _IID_IInternalConnection   5f731560     dlldb.obj
 0002:00000570       _IID_IAxWinAmbientDispatch 5f731570     dlldb.obj
 0002:00000580       _IID_IAxWinHostWindow      5f731580     dlldb.obj
 0002:00000590       _IID_IRegistrar            5f731590     dlldb.obj
 0002:000005a0       _CLSID_Registrar           5f7315a0     dlldb.obj
 0002:000005b0       _LIBID_ATLLib              5f7315b0     dlldb.obj
 0002:000005c0       ??_C@_0N@IJBO@MFCO42UD?4DLL?$AA@ 5f7315c0     dlldb.obj
 0002:000005d0       ??_C@_0M@IGON@MFC42UD?4DLL?$AA@ 5f7315d0     dlldb.obj
 0002:000005e0       ?classCRecordset@CRecordset@@2UCRuntimeClass@@B 5f7315e0     dbcore.obj
 0002:000005f8       ??_C@_0L@FKJL@CRecordset?$AA@ 5f7315f8     dbcore.obj
 0002:00000608       ?classCDatabase@CDatabase@@2UCRuntimeClass@@B 5f731608     dbcore.obj
 0002:00000620       ??_C@_09CDJB@CDatabase?$AA@ 5f731620     dbcore.obj
 0002:00000630       ?classCDBException@CDBException@@2UCRuntimeClass@@B 5f731630     dbcore.obj
 0002:00000648       ??_C@_0N@GGEG@CDBException?$AA@ 5f731648     dbcore.obj
 0002:00000658       ?_afxODBCDLL@@3QBDB        5f731658     dbcore.obj
 0002:00000664       ?_afxDriverNotCapable@@3QBGB 5f731664     dbcore.obj
 0002:0000067c       ?_afxOutOfSequence@@3QBGB  5f73167c     dbcore.obj
 0002:00000694       ?_afxInfoRange@@3QBGB      5f731694     dbcore.obj
 0002:000006ac       ?_afxDataTruncated@@3QBGB  5f7316ac     dbcore.obj
 0002:000006c4       ?_afxRowFetch@@3QBGB       5f7316c4     dbcore.obj
 0002:000006dc       ?_afxForUpdate@@3QBGB      5f7316dc     dbcore.obj
 0002:000006f8       ?_afxOrderBy@@3QBGB        5f7316f8     dbcore.obj
 0002:00000710       ?_afxWhere@@3QBGB          5f731710     dbcore.obj
 0002:00000720       ?_afxFrom@@3QBGB           5f731720     dbcore.obj
 0002:00000730       ?_afxSelect@@3QBGB         5f731730     dbcore.obj
 0002:00000740       ?_afxParamCall@@3QBGB      5f731740     dbcore.obj
 0002:00000748       ?_afxCall@@3QBGB           5f731748     dbcore.obj
 0002:00000758       ?_afxLiteralSeparator@@3GB 5f731758     dbcore.obj
 0002:0000075c       ?_afxComma@@3QBGB          5f73175c     dbcore.obj
 0002:00000760       ?_afxODBCTrail@@3QBGB      5f731760     dbcore.obj
 0002:0000076c       ??_C@_17JNCL@?$AA?$CF?$AAs?$AA?6?$AA?$AA@ 5f73176c     dbcore.obj
 0002:00000778       ??_7CDBException@@6B@      5f731778     dbcore.obj
 0002:00000798       ??_C@_1O@JCG@?$AAS?$AAt?$AAa?$AAt?$AAe?$AA?3?$AA?$AA@ 5f731798     dbcore.obj
 0002:000007a8       ??_C@_13DEJI@?$AA?6?$AA?$AA@ 5f7317a8     dbcore.obj
 0002:000007ac       ??_C@_1CI@LDEF@?$AA?0?$AAN?$AAa?$AAt?$AAi?$AAv?$AAe?$AA?3?$AA?$CF?$AAl?$AAd?$AA?0?$AAO?$AAr?$AAi?$AAg?$AAi?$AAn?$AA?3?$AA?$AA@ 5f7317ac     dbcore.obj
 0002:000007d4       ??_C@_1M@MKCN@?$AA0?$AA0?$AA0?$AA0?$AA0?$AA?$AA@ 5f7317d4     dbcore.obj
 0002:000007e4       ??_7CDatabase@@6B@         5f7317e4     dbcore.obj
 0002:00000814       ??_C@_1M@BHKK@?$AA?$DL?$AAD?$AAS?$AAN?$AA?$DN?$AA?$AA@ 5f731814     dbcore.obj
 0002:00000820       ??_C@_15DEDE@?$AA?$CF?$AAs?$AA?$AA@ 5f731820     dbcore.obj
 0002:00000828       ??_C@_1GC@FDFL@?$AAE?$AAr?$AAr?$AAo?$AAr?$AA?3?$AA?5?$AAM?$AAi?$AAs?$AAs?$AAi?$AAn?$AAg?$AA?5?$AA?8?$AAO?$AAD?$AAB?$AAC@ 5f731828     dbcore.obj
 0002:0000088c       ??_C@_08PEKM@lpa?5?$CB?$DN?50?$AA@ 5f73188c     dbcore.obj
 0002:00000898       ??_C@_0CH@IIKL@E?3?28168?2vc98?2mfc?2atl?2include?2atl@ 5f731898     dbcore.obj
 0002:000008c0       ??_C@_08NDGO@lpw?5?$CB?$DN?50?$AA@ 5f7318c0     dbcore.obj
 0002:000008cc       ??_C@_1HC@GCMH@?$AAE?$AAr?$AAr?$AAo?$AAr?$AA?3?$AA?5?$AAS?$AAQ?$AAL?$AAF?$AAr?$AAe?$AAe?$AAE?$AAn?$AAv?$AA?5?$AAf?$AAa@ 5f7318cc     dbcore.obj
 0002:00000940       ??_C@_1IM@MBOF@?$AAE?$AAr?$AAr?$AAo?$AAr?$AA?3?$AA?5?$AAe?$AAx?$AAc?$AAe?$AAp?$AAt?$AAi?$AAo?$AAn?$AA?5?$AAb?$AAy?$AA?5@ 5f731940     dbcore.obj
 0002:000009cc       ??_C@_1EE@PKHL@?$AAW?$AAa?$AAr?$AAn?$AAi?$AAn?$AAg?$AA?3?$AA?5?$AAO?$AAD?$AAB?$AAC?$AA?5?$AAS?$AAu?$AAc?$AAc?$AAe?$AAs@ 5f7319cc     dbcore.obj
 0002:00000a10       ??_C@_1GC@IKIO@?$AAW?$AAa?$AAr?$AAn?$AAi?$AAn?$AAg?$AA?3?$AA?5?$AAF?$AAa?$AAi?$AAl?$AAu?$AAr?$AAe?$AA?5?$AAs?$AAe?$AAt@ 5f731a10     dbcore.obj
 0002:00000a74       ??_C@_1FC@ECMP@?$AAW?$AAa?$AAr?$AAn?$AAi?$AAn?$AAg?$AA?3?$AA?5?$AAF?$AAa?$AAi?$AAl?$AAu?$AAr?$AAe?$AA?5?$AAs?$AAe?$AAt@ 5f731a74     dbcore.obj
 0002:00000ac8       ??_C@_0N@PKHK@odbccall?4txt?$AA@ 5f731ac8     dbcore.obj
 0002:00000ad8       ??_C@_1JE@FNFO@?$AAE?$AAr?$AAr?$AAo?$AAr?$AA?3?$AA?5?$AAN?$AAo?$AA?5?$AAd?$AAe?$AAf?$AAa?$AAu?$AAl?$AAt?$AA?5?$AAw?$AAi@ 5f731ad8     dbcore.obj
 0002:00000b6c       ??_C@_1BO@PBOK@?$AA?0?$AA?5?$AAV?$AAe?$AAr?$AAs?$AAi?$AAo?$AAn?$AA?3?$AA?5?$AA?$CF?$AAs?$AA?6?$AA?$AA@ 5f731b6c     dbcore.obj
 0002:00000b8c       ??_C@_1BE@PKHH@?$AAD?$AAB?$AAM?$AAS?$AA?3?$AA?5?$AA?$CF?$AAs?$AA?6?$AA?$AA@ 5f731b8c     dbcore.obj
 0002:00000ba0       ??_C@_1EG@GIAC@?$AAW?$AAa?$AAr?$AAn?$AAi?$AAn?$AAg?$AA?3?$AA?5?$AAd?$AAa?$AAt?$AAa?$AA?5?$AAs?$AAo?$AAu?$AAr?$AAc?$AAe@ 5f731ba0     dbcore.obj
 0002:00000be8       ??_C@_01PCJP@Y?$AA@        5f731be8     dbcore.obj
 0002:00000bec       ??_C@_01BJG@?6?$AA@        5f731bec     dbcore.obj
 0002:00000bf0       ??_C@_0BI@MNAB@?6?7henvAllConnections?5?$DN?5?$AA@ 5f731bf0     dbcore.obj
 0002:00000c08       ??_C@_0BA@LDLC@?6?7nAllocated?5?$DN?5?$AA@ 5f731c08     dbcore.obj
 0002:00000c18       ??_C@_0L@OKHO@?6with?5env?3?$AA@ 5f731c18     dbcore.obj
 0002:00000c24       ??_C@_0BF@DMHA@?6m_dwQueryTimeout?5?$DN?5?$AA@ 5f731c24     dbcore.obj
 0002:00000c3c       ??_C@_0BF@BECC@?6m_dwLoginTimeout?5?$DN?5?$AA@ 5f731c3c     dbcore.obj
 0002:00000c54       ??_C@_0BK@IHG@?6m_bTransactionPending?5?$DN?5?$AA@ 5f731c54     dbcore.obj
 0002:00000c70       ??_C@_0BE@HNE@?6m_bTransactions?5?$DN?5?$AA@ 5f731c70     dbcore.obj
 0002:00000c84       ??_C@_0BB@FGMM@?6m_bUpdatable?5?$DN?5?$AA@ 5f731c84     dbcore.obj
 0002:00000c98       ??_C@_0BB@MLGK@?6m_strConnect?5?$DN?5?$AA@ 5f731c98     dbcore.obj
 0002:00000cac       ??_C@_09DBDF@m_hdbc?5?$DN?5?$AA@ 5f731cac     dbcore.obj
 0002:00000cbc       ??_7CRecordset@@6B@        5f731cbc     dbcore.obj
 0002:00000d24       ??_C@_1FI@LOMJ@?$AAE?$AAr?$AAr?$AAo?$AAr?$AA?3?$AA?5?$AAE?$AAx?$AAc?$AAe?$AAp?$AAt?$AAi?$AAo?$AAn?$AA?5?$AAi?$AAg?$AAn@ 5f731d24     dbcore.obj
 0002:00000d7c       ??_C@_1FA@JJEP@?$AA?6?$AAt?$AAo?$AA?5?$AAC?$AAl?$AAo?$AAs?$AAe?$AA?5?$AAo?$AAr?$AA?5?$AAm?$AAe?$AAm?$AAo?$AAr?$AAy?$AA?5@ 5f731d7c     dbcore.obj
 0002:00000dcc       ??_C@_1FO@BMOB@?$AA?6?$AAU?$AAs?$AAe?$AA?5?$AAo?$AAf?$AA?5?$AAm?$AAu?$AAl?$AAt?$AAi?$AA?5?$AAr?$AAo?$AAw?$AA?5?$AAf?$AAe@ 5f731dcc     dbcore.obj
 0002:00000e2c       ??_C@_1GG@HFNK@?$AA?6?$AAW?$AAA?$AAR?$AAN?$AAI?$AAN?$AAG?$AA?3?$AA?5?$AAC?$AAl?$AAo?$AAs?$AAe?$AA?5?$AAc?$AAa?$AAl?$AAl@ 5f731e2c     dbcore.obj
 0002:00000e94       ??_C@_1IC@IKNF@?$AAW?$AAA?$AAR?$AAN?$AAI?$AAN?$AAG?$AA?3?$AA?5?$AAC?$AAR?$AAe?$AAc?$AAo?$AAr?$AAd?$AAs?$AAe?$AAt?$AA?5@ 5f731e94     dbcore.obj
 0002:00000f18       ??_C@_1GC@IMCJ@?$AAE?$AAr?$AAr?$AAo?$AAr?$AA?3?$AA?5?$AAS?$AAQ?$AAL?$AAN?$AAu?$AAm?$AAR?$AAe?$AAs?$AAu?$AAl?$AAt?$AAC@ 5f731f18     dbcore.obj
 0002:00000f7c       ??_C@_1EE@IMDG@?$AAW?$AAa?$AAr?$AAn?$AAi?$AAn?$AAg?$AA?3?$AA?5?$AAO?$AAD?$AAB?$AAC?$AA?5?$AAS?$AAu?$AAc?$AAc?$AAe?$AAs@ 5f731f7c     dbcore.obj
 0002:00000fc0       ??_C@_1EE@MLLI@?$AAE?$AAr?$AAr?$AAo?$AAr?$AA?3?$AA?5?$AAf?$AAe?$AAt?$AAc?$AAh?$AAi?$AAn?$AAg?$AA?5?$AAr?$AAo?$AAw?$AA?5@ 5f731fc0     dbcore.obj
 0002:00001004       ??_C@_1GA@EOEG@?$AAE?$AAr?$AAr?$AAo?$AAr?$AA?3?$AA?5?$AAf?$AAi?$AAe?$AAl?$AAd?$AA?5?$AAd?$AAa?$AAt?$AAa?$AA?5?$AAt?$AAr@ 5f732004     dbcore.obj
 0002:00001064       ??_C@_1EM@CBAG@?$AAE?$AAr?$AAr?$AAo?$AAr?$AA?3?$AA?5?$AAG?$AAe?$AAt?$AAB?$AAo?$AAo?$AAk?$AAm?$AAa?$AAr?$AAk?$AA?5?$AAo@ 5f732064     dbcore.obj
 0002:000010b0       ??_C@_1HI@MFN@?$AAE?$AAr?$AAr?$AAo?$AAr?$AA?3?$AA?5?$AAa?$AAt?$AAt?$AAe?$AAm?$AAp?$AAt?$AA?5?$AAt?$AAo?$AA?5?$AAl?$AAo@ 5f7320b0     dbcore.obj
 0002:00001128       ??_C@_1FO@PJLA@?$AAE?$AAr?$AAr?$AAo?$AAr?$AA?3?$AA?5?$AAE?$AAd?$AAi?$AAt?$AA?5?$AAa?$AAt?$AAt?$AAe?$AAm?$AAp?$AAt?$AA?5@ 5f732128     dbcore.obj
 0002:00001188       ??_C@_1HA@MJPF@?$AAE?$AAr?$AAr?$AAo?$AAr?$AA?3?$AA?5?$AAm?$AAu?$AAs?$AAt?$AA?5?$AAe?$AAn?$AAt?$AAe?$AAr?$AA?5?$AAE?$AAd@ 5f732188     dbcore.obj
 0002:000011f8       ??_C@_1IA@KHHB@?$AAE?$AAr?$AAr?$AAo?$AAr?$AA?3?$AA?5?$AAa?$AAt?$AAt?$AAe?$AAm?$AAp?$AAt?$AAe?$AAd?$AA?5?$AAt?$AAo?$AA?5@ 5f7321f8     dbcore.obj
 0002:00001278       ??_C@_1EO@NPH@?$AAE?$AAr?$AAr?$AAo?$AAr?$AA?3?$AA?5?$AAa?$AAt?$AAt?$AAe?$AAm?$AAp?$AAt?$AA?5?$AAF?$AAl?$AAu?$AAs?$AAh@ 5f732278     dbcore.obj
 0002:000012c8       ??_C@_1EA@LJGK@?$AAE?$AAr?$AAr?$AAo?$AAr?$AA?3?$AA?5?$AAR?$AAe?$AAq?$AAu?$AAe?$AAr?$AAy?$AA?5?$AAa?$AAt?$AAt?$AAe?$AAm@ 5f7322c8     dbcore.obj
 0002:00001308       ??_C@_11A@?$AA?$AA@        5f732308     dbcore.obj
 0002:0000130c       ??_C@_1GE@ENCI@?$AAW?$AAa?$AAr?$AAn?$AAi?$AAn?$AAg?$AA?3?$AA?5?$AAS?$AAe?$AAt?$AAt?$AAi?$AAn?$AAg?$AA?5?$AAf?$AAo?$AAr@ 5f73230c     dbcore.obj
 0002:00001370       ??_C@_1GA@JKDO@?$AAE?$AAr?$AAr?$AAo?$AAr?$AA?3?$AA?5?$AAC?$AAD?$AAa?$AAt?$AAa?$AAb?$AAa?$AAs?$AAe?$AA?5?$AAc?$AAr?$AAe@ 5f732370     dbcore.obj
 0002:000013d0       ??_C@_1GO@CABB@?$AAE?$AAr?$AAr?$AAo?$AAr?$AA?3?$AA?5?$AAO?$AAD?$AAB?$AAC?$AA?5?$AAf?$AAa?$AAi?$AAl?$AAu?$AAr?$AAe?$AA?5@ 5f7323d0     dbcore.obj
 0002:00001440       ??_C@_1EO@KAHP@?$AA?7?$AAM?$AAa?$AAr?$AAk?$AAi?$AAn?$AAg?$AA?5?$AAC?$AAR?$AAe?$AAc?$AAo?$AAr?$AAd?$AAs?$AAe?$AAt?$AA?5@ 5f732440     dbcore.obj
 0002:00001490       ??_C@_1FC@CANC@?$AAW?$AAa?$AAr?$AAn?$AAi?$AAn?$AAg?$AA?3?$AA?5?$AAC?$AAo?$AAn?$AAc?$AAu?$AAr?$AAr?$AAe?$AAn?$AAc?$AAy@ 5f732490     dbcore.obj
 0002:000014e4       ??_C@_1GI@BFIP@?$AAE?$AAr?$AAr?$AAo?$AAr?$AA?3?$AA?5?$AAO?$AAD?$AAB?$AAC?$AA?5?$AAf?$AAa?$AAi?$AAl?$AAu?$AAr?$AAe?$AA?5@ 5f7324e4     dbcore.obj
 0002:0000154c       ??_C@_1GI@OEHO@?$AAE?$AAr?$AAr?$AAo?$AAr?$AA?3?$AA?5?$AAO?$AAD?$AAB?$AAC?$AA?5?$AAf?$AAa?$AAi?$AAl?$AAu?$AAr?$AAe?$AA?5@ 5f73254c     dbcore.obj
 0002:000015b4       ??_C@_1EO@PBJM@?$AAW?$AAa?$AAr?$AAn?$AAi?$AAn?$AAg?$AA?3?$AA?5?$AAS?$AAe?$AAt?$AAt?$AAi?$AAn?$AAg?$AA?5?$AAr?$AAe?$AAc@ 5f7325b4     dbcore.obj
 0002:00001604       ??_C@_1HC@NIEI@?$AAW?$AAa?$AAr?$AAn?$AAi?$AAn?$AAg?$AA?3?$AA?5?$AAD?$AAr?$AAi?$AAv?$AAe?$AAr?$AA?5?$AAd?$AAo?$AAe?$AAs@ 5f732604     dbcore.obj
 0002:00001678       ??_C@_1DA@JIHM@?$AAf?$AAo?$AAr?$AA?5?$AAu?$AAs?$AAe?$AA?5?$AAw?$AAi?$AAt?$AAh?$AA?5?$AAS?$AAQ?$AAL?$AAF?$AAe?$AAt?$AAc@ 5f732678     dbcore.obj
 0002:000016a8       ??_C@_1HA@KAAN@?$AAa?$AAn?$AAd?$AA?1?$AAo?$AAr?$AA?5?$AAc?$AAu?$AAr?$AAs?$AAo?$AAr?$AA?5?$AAl?$AAi?$AAb?$AAr?$AAa?$AAr@ 5f7326a8     dbcore.obj
 0002:00001718       ??_C@_1GG@DFEH@?$AAW?$AAa?$AAr?$AAn?$AAi?$AAn?$AAg?$AA?3?$AA?5?$AAS?$AAQ?$AAL?$AAE?$AAx?$AAt?$AAe?$AAn?$AAd?$AAe?$AAd@ 5f732718     dbcore.obj
 0002:00001780       ??_C@_1IE@IGCD@?$AAE?$AAr?$AAr?$AAo?$AAr?$AA?3?$AA?5?$AAO?$AAD?$AAB?$AAC?$AA?5?$AAf?$AAa?$AAi?$AAl?$AAu?$AAr?$AAe?$AA?5@ 5f732780     dbcore.obj
 0002:00001804       ??_C@_1FK@GDGL@?$AAE?$AAr?$AAr?$AAo?$AAr?$AA?3?$AA?5?$AAO?$AAD?$AAB?$AAC?$AA?5?$AAf?$AAa?$AAi?$AAl?$AAu?$AAr?$AAe?$AA?5@ 5f732804     dbcore.obj
 0002:00001860       ??_C@_1DM@IDP@?$AAE?$AAr?$AAr?$AAo?$AAr?$AA?3?$AA?5?$AAC?$AAa?$AAn?$AA?8?$AAt?$AA?5?$AAg?$AAe?$AAt?$AA?5?$AAf?$AAi?$AAe@ 5f732860     dbcore.obj
 0002:0000189c       ??_C@_1EO@FAIK@?$AAE?$AAr?$AAr?$AAo?$AAr?$AA?3?$AA?5?$AAC?$AAa?$AAn?$AA?8?$AAt?$AA?5?$AAe?$AAn?$AAa?$AAb?$AAl?$AAe?$AA?5@ 5f73289c     dbcore.obj
 0002:000018ec       ??_C@_1GI@DJFL@?$AAE?$AAr?$AAr?$AAo?$AAr?$AA?3?$AA?5?$AAO?$AAD?$AAB?$AAC?$AA?5?$AAf?$AAa?$AAi?$AAl?$AAu?$AAr?$AAe?$AA?5@ 5f7328ec     dbcore.obj
 0002:00001954       ??_C@_1HM@IPPG@?$AAW?$AAa?$AAr?$AAn?$AAi?$AAn?$AAg?$AA?3?$AA?5?$AAl?$AAo?$AAc?$AAk?$AAi?$AAn?$AAg?$AA?5?$AAn?$AAo?$AAt@ 5f732954     dbcore.obj
 0002:000019d0       ??_C@_1GM@LADD@?$AAE?$AAr?$AAr?$AAo?$AAr?$AA?3?$AA?5?$AAO?$AAD?$AAB?$AAC?$AA?5?$AAf?$AAa?$AAi?$AAl?$AAu?$AAr?$AAe?$AA?5@ 5f7329d0     dbcore.obj
 0002:00001a3c       ??_C@_1GM@ENHA@?$AAW?$AAa?$AAr?$AAn?$AAi?$AAn?$AAg?$AA?3?$AA?5?$AAS?$AAQ?$AAL?$AA?5?$AAc?$AAo?$AAn?$AAt?$AAa?$AAi?$AAn@ 5f732a3c     dbcore.obj
 0002:00001aa8       ??_C@_1HG@DJNJ@?$AAW?$AAa?$AAr?$AAn?$AAi?$AAn?$AAg?$AA?3?$AA?5?$AAS?$AAQ?$AAL?$AA?5?$AAc?$AAo?$AAn?$AAt?$AAa?$AAi?$AAn@ 5f732aa8     dbcore.obj
 0002:00001b20       ??_C@_1BA@FFIB@?$AA?5?$AAU?$AAN?$AAI?$AAO?$AAN?$AA?5?$AA?$AA@ 5f732b20     dbcore.obj
 0002:00001b30       ??_C@_1HM@CAKC@?$AAW?$AAa?$AAr?$AAn?$AAi?$AAn?$AAg?$AA?3?$AA?5?$AAS?$AAQ?$AAL?$AA?5?$AAc?$AAo?$AAn?$AAt?$AAa?$AAi?$AAn@ 5f732b30     dbcore.obj
 0002:00001bac       ??_C@_1BG@CONM@?$AA?5?$AAG?$AAR?$AAO?$AAU?$AAP?$AA?5?$AAB?$AAY?$AA?5?$AA?$AA@ 5f732bac     dbcore.obj
 0002:00001bc4       ??_C@_1GK@HMOJ@?$AAW?$AAa?$AAr?$AAn?$AAi?$AAn?$AAg?$AA?3?$AA?5?$AAM?$AAi?$AAs?$AAs?$AAi?$AAn?$AAg?$AA?5?$AA?8?$AA?5?$AAF@ 5f732bc4     dbcore.obj
 0002:00001c30       ??_C@_1O@LFLK@?$AA?5?$AAJ?$AAO?$AAI?$AAN?$AA?5?$AA?$AA@ 5f732c30     dbcore.obj
 0002:00001c40       ??_C@_1EM@NJB@?$AAE?$AAr?$AAr?$AAo?$AAr?$AA?3?$AA?5?$AAa?$AAt?$AAt?$AAe?$AAm?$AAp?$AAt?$AAe?$AAd?$AA?5?$AAt?$AAo?$AA?5@ 5f732c40     dbcore.obj
 0002:00001c8c       ??_C@_1EI@GPFM@?$AAE?$AAr?$AAr?$AAo?$AAr?$AA?3?$AA?5?$AAa?$AAt?$AAt?$AAe?$AAm?$AAp?$AAt?$AAe?$AAd?$AA?5?$AAt?$AAo?$AA?5@ 5f732c8c     dbcore.obj
 0002:00001cd4       ??_C@_1HC@CIAE@?$AAE?$AAr?$AAr?$AAo?$AAr?$AA?3?$AA?5?$AAa?$AAt?$AAt?$AAe?$AAm?$AAp?$AAt?$AAe?$AAd?$AA?5?$AAt?$AAo?$AA?5@ 5f732cd4     dbcore.obj
 0002:00001d48       ??_C@_1GO@CMCO@?$AAE?$AAr?$AAr?$AAo?$AAr?$AA?3?$AA?5?$AAf?$AAo?$AAr?$AAw?$AAa?$AAr?$AAd?$AA?9?$AAo?$AAn?$AAl?$AAy?$AA?5@ 5f732d48     dbcore.obj
 0002:00001db8       ??_C@_1FM@MFNO@?$AAE?$AAr?$AAr?$AAo?$AAr?$AA?3?$AA?5?$AAn?$AAo?$AA?5?$AAf?$AAi?$AAe?$AAl?$AAd?$AA?5?$AAn?$AAa?$AAm?$AAe@ 5f732db8     dbcore.obj
 0002:00001e14       ??_C@_13JKDK@?$AA?0?$AA?$AA@ 5f732e14     dbcore.obj
 0002:00001e18       ??_C@_1JC@FFNF@?$AAW?$AAa?$AAr?$AAn?$AAi?$AAn?$AAg?$AA?3?$AA?5?$AAS?$AAe?$AAt?$AAt?$AAi?$AAn?$AAg?$AA?5?$AAr?$AAe?$AAc@ 5f732e18     dbcore.obj
 0002:00001eac       ??_C@_1EE@DHLD@?$AA?7?$AAW?$AAi?$AAl?$AAl?$AA?5?$AAu?$AAs?$AAe?$AA?5?$AAp?$AAo?$AAs?$AAi?$AAt?$AAi?$AAo?$AAn?$AAe?$AAd@ 5f732eac     dbcore.obj
 0002:00001ef0       ??_C@_1IC@EACK@?$AAW?$AAa?$AAr?$AAn?$AAi?$AAn?$AAg?$AA?3?$AA?5?$AAC?$AAa?$AAn?$AA?8?$AAt?$AA?5?$AAu?$AAs?$AAe?$AA?5?$AAS@ 5f732ef0     dbcore.obj
 0002:00001f74       ??_C@_1EC@LHPG@?$AAE?$AAr?$AAr?$AAo?$AAr?$AA?3?$AA?5?$AAf?$AAa?$AAi?$AAl?$AAu?$AAr?$AAe?$AA?5?$AAu?$AAp?$AAd?$AAa?$AAt@ 5f732f74     dbcore.obj
 0002:00001fb8       ??_C@_1FM@DCDN@?$AAE?$AAr?$AAr?$AAo?$AAr?$AA?3?$AA?5?$AAf?$AAa?$AAi?$AAl?$AAu?$AAr?$AAe?$AA?5?$AAt?$AAo?$AA?5?$AAa?$AAl@ 5f732fb8     dbcore.obj
 0002:00002014       ??_C@_1CG@BIKJ@?$AA?5?$AAW?$AAH?$AAE?$AAR?$AAE?$AA?5?$AAC?$AAU?$AAR?$AAR?$AAE?$AAN?$AAT?$AA?5?$AAO?$AAF?$AA?5?$AA?$AA@ 5f733014     dbcore.obj
 0002:0000203c       ??_C@_1M@FJED@?$AA?5?$AAS?$AAE?$AAT?$AA?5?$AA?$AA@ 5f73303c     dbcore.obj
 0002:00002048       ??_C@_1BA@MDEN@?$AAU?$AAP?$AAD?$AAA?$AAT?$AAE?$AA?5?$AA?$AA@ 5f733048     dbcore.obj
 0002:00002058       ??_C@_1BE@LEJJ@?$AA?5?$AAV?$AAA?$AAL?$AAU?$AAE?$AAS?$AA?5?$AA?$CI?$AA?$AA@ 5f733058     dbcore.obj
 0002:0000206c       ??_C@_15NGMK@?$AA?5?$AA?$CI?$AA?$AA@ 5f73306c     dbcore.obj
 0002:00002074       ??_C@_1BK@ECOF@?$AAI?$AAN?$AAS?$AAE?$AAR?$AAT?$AA?5?$AAI?$AAN?$AAT?$AAO?$AA?5?$AA?$AA@ 5f733074     dbcore.obj
 0002:00002090       ??_C@_1BK@FPKL@?$AAD?$AAE?$AAL?$AAE?$AAT?$AAE?$AA?5?$AAF?$AAR?$AAO?$AAM?$AA?5?$AA?$AA@ 5f733090     dbcore.obj
 0002:000020ac       ??_C@_1HK@IFFI@?$AAW?$AAa?$AAr?$AAn?$AAi?$AAn?$AAg?$AA?3?$AA?5?$AA?$CF?$AAu?$AA?5?$AAr?$AAo?$AAw?$AAs?$AA?5?$AAa?$AAf?$AAf@ 5f7330ac     dbcore.obj
 0002:00002128       ??_C@_1HE@KANF@?$AAE?$AAr?$AAr?$AAo?$AAr?$AA?3?$AA?5?$AAf?$AAa?$AAi?$AAl?$AAu?$AAr?$AAe?$AA?5?$AAh?$AAa?$AAn?$AAd?$AAl@ 5f733128     dbcore.obj
 0002:0000219c       ??_C@_1IG@NFEH@?$AAE?$AAr?$AAr?$AAo?$AAr?$AA?3?$AA?5?$AAa?$AAt?$AAt?$AAe?$AAm?$AAp?$AAt?$AAi?$AAn?$AAg?$AA?5?$AAt?$AAo@ 5f73319c     dbcore.obj
 0002:00002224       ??_C@_1GG@CEAL@?$AAE?$AAr?$AAr?$AAo?$AAr?$AA?3?$AA?5?$AAa?$AAt?$AAt?$AAe?$AAm?$AAp?$AAt?$AAe?$AAd?$AA?5?$AAt?$AAo?$AA?5@ 5f733224     dbcore.obj
 0002:0000228c       ??_C@_1HI@NPFJ@?$AAE?$AAr?$AAr?$AAo?$AAr?$AA?3?$AA?5?$AAa?$AAt?$AAt?$AAe?$AAm?$AAp?$AAt?$AAe?$AAd?$AA?5?$AAt?$AAo?$AA?5@ 5f73328c     dbcore.obj
 0002:00002304       ??_C@_1EO@CKND@?$AA?7?$AAD?$AAa?$AAt?$AAa?$AA?5?$AAa?$AAl?$AAr?$AAe?$AAa?$AAd?$AAy?$AA?5?$AAf?$AAe?$AAt?$AAc?$AAh?$AAe@ 5f733304     dbcore.obj
 0002:00002354       ??_C@_1GI@CONN@?$AAE?$AAr?$AAr?$AAo?$AAr?$AA?3?$AA?5?$AAG?$AAe?$AAt?$AAF?$AAi?$AAe?$AAl?$AAd?$AAV?$AAa?$AAl?$AAu?$AAe@ 5f733354     dbcore.obj
 0002:000023bc       ??_C@_1FM@LIBK@?$AAW?$AAa?$AAr?$AAn?$AAi?$AAn?$AAg?$AA?3?$AA?5?$AAO?$AAD?$AAB?$AAC?$AA?5?$AAS?$AAu?$AAc?$AAc?$AAe?$AAs@ 5f7333bc     dbcore.obj
 0002:00002418       ??_C@_0BA@BGHA@with?5database?3?5?$AA@ 5f733418     dbcore.obj
 0002:00002428       ??_C@_0BC@MKGN@with?5no?5database?6?$AA@ 5f733428     dbcore.obj
 0002:0000243c       ??_C@_0CP@HPBB@?6Dump?5values?5for?5each?5field?5in?5c@ 5f73343c     dbcore.obj
 0002:0000246c       ??_C@_0BC@JNKN@?6m_hstmtUpdate?5?$DN?5?$AA@ 5f73346c     dbcore.obj
 0002:00002480       ??_C@_0BE@OFAF@?6m_strCursorName?5?$DN?5?$AA@ 5f733480     dbcore.obj
 0002:00002494       ??_C@_0BA@CDEP@?6m_nEditMode?5?$DN?5?$AA@ 5f733494     dbcore.obj
 0002:000024a4       ??_C@_0BA@GJB@?6m_bLockMode?5?$DN?5?$AA@ 5f7334a4     dbcore.obj
 0002:000024b4       ??_C@_0P@NFAJ@?6m_bDeleted?5?$DN?5?$AA@ 5f7334b4     dbcore.obj
 0002:000024c4       ??_C@_0L@IPIJ@?6m_bBOF?5?$DN?5?$AA@ 5f7334c4     dbcore.obj
 0002:000024d0       ??_C@_0L@GHOJ@?6m_bEOF?5?$DN?5?$AA@ 5f7334d0     dbcore.obj
 0002:000024dc       ??_C@_0O@DPF@?6m_nParams?5?$DN?5?$AA@ 5f7334dc     dbcore.obj
 0002:000024ec       ??_C@_0BD@GPPK@?6m_nFieldsBound?5?$DN?5?$AA@ 5f7334ec     dbcore.obj
 0002:00002500       ??_C@_0O@ECP@?6m_nFields?5?$DN?5?$AA@ 5f733500     dbcore.obj
 0002:00002510       ??_C@_0BC@IMFD@?6m_bAppendable?5?$DN?5?$AA@ 5f733510     dbcore.obj
 0002:00002524       ??_C@_0BC@CBKM@?6m_bScrollable?5?$DN?5?$AA@ 5f733524     dbcore.obj
 0002:00002538       ??_C@_0M@CNKH@?6m_lOpen?5?$DN?5?$AA@ 5f733538     dbcore.obj
 0002:00002544       ??_C@_0BD@DHNL@?6m_bRecordsetDb?5?$DN?5?$AA@ 5f733544     dbcore.obj
 0002:00002558       ??_C@_0M@JKLH@?6m_hstmt?5?$DN?5?$AA@ 5f733558     dbcore.obj
 0002:00002564       ??_C@_0N@MDHJ@?6m_strSQL?5?$DN?5?$AA@ 5f733564     dbcore.obj
 0002:00002574       ??_C@_0P@KPIA@m_nOpenType?5?$DN?5?$AA@ 5f733574     dbcore.obj
 0002:00002584       ??_C@_1HG@CEAC@?$AAE?$AAr?$AAr?$AAo?$AAr?$AA?3?$AA?5?$AAS?$AAe?$AAt?$AAS?$AAy?$AAn?$AAc?$AAh?$AAr?$AAo?$AAn?$AAo?$AAu@ 5f733584     dbcore.obj
 0002:000025fc       ??_C@_0CH@KFAI@E?3?28168?2vc98?2mfc?2mfc?2include?2afx@ 5f7335fc     dbcore.obj
 0002:00002628       ??_7_AFX_DB_STATE@@6B@     5f733628     dbcore.obj
 0002:00002630       ??_7CNoTrackObject@@6B@    5f733630     dbcore.obj
 0002:00002634       ??_C@_1FO@CG@?$AAE?$AAr?$AAr?$AAo?$AAr?$AA?3?$AA?5?$AAf?$AAi?$AAe?$AAl?$AAd?$AA?5?$AAa?$AAd?$AAd?$AAr?$AAe?$AAs?$AAs@ 5f733634     dbrfx.obj
 0002:00002694       ??_C@_03FGJK@?5?$DN?5?$AA@ 5f733694     dbrfx.obj
 0002:00002698       ??_C@_1GA@LPOM@?$AAE?$AAr?$AAr?$AAo?$AAr?$AA?3?$AA?5?$AAb?$AAu?$AAf?$AAf?$AAe?$AAr?$AA?5?$AA?$CI?$AAc?$AAo?$AAl?$AAu?$AAm@ 5f733698     dbrfx.obj
 0002:000026f8       ??_C@_1FM@KDBP@?$AAW?$AAa?$AAr?$AAn?$AAi?$AAn?$AAg?$AA?3?$AA?5?$AAs?$AAt?$AAr?$AAi?$AAn?$AAg?$AA?5?$AAc?$AAo?$AAn?$AAv@ 5f7336f8     dbrfx.obj
 0002:00002754       ??_C@_1HA@IBMC@?$AAE?$AAr?$AAr?$AAo?$AAr?$AA?3?$AA?5?$AAC?$AAS?$AAt?$AAr?$AAi?$AAn?$AAg?$AA?5?$AAb?$AAu?$AAf?$AAf?$AAe@ 5f733754     dbrfx.obj
 0002:000027c4       ??_C@_1FO@OFHM@?$AAW?$AAa?$AAr?$AAn?$AAi?$AAn?$AAg?$AA?3?$AA?5?$AAC?$AAS?$AAt?$AAr?$AAi?$AAn?$AAg?$AA?5?$AAc?$AAo?$AAn@ 5f7337c4     dbrfx.obj
 0002:00002824       ??_C@_1FG@FIKO@?$AAW?$AAa?$AAr?$AAn?$AAi?$AAn?$AAg?$AA?3?$AA?5?$AAi?$AAn?$AAt?$AA?5?$AAc?$AAo?$AAn?$AAv?$AAe?$AAr?$AAt@ 5f733824     dbrfx.obj
 0002:0000287c       ??_C@_1FI@BKDC@?$AAW?$AAa?$AAr?$AAn?$AAi?$AAn?$AAg?$AA?3?$AA?5?$AAl?$AAo?$AAn?$AAg?$AA?5?$AAc?$AAo?$AAn?$AAv?$AAe?$AAr@ 5f73387c     dbrfx.obj
 0002:000028d4       ??_C@_1FI@OIHI@?$AAW?$AAa?$AAr?$AAn?$AAi?$AAn?$AAg?$AA?3?$AA?5?$AAB?$AAY?$AAT?$AAE?$AA?5?$AAc?$AAo?$AAn?$AAv?$AAe?$AAr@ 5f7338d4     dbrfx.obj
 0002:0000292c       ??_C@_1FI@MODJ@?$AAW?$AAa?$AAr?$AAn?$AAi?$AAn?$AAg?$AA?3?$AA?5?$AAB?$AAO?$AAO?$AAL?$AA?5?$AAc?$AAo?$AAn?$AAv?$AAe?$AAr@ 5f73392c     dbrfx.obj
 0002:00002984       ??_C@_01PKAG@?3?$AA@       5f733984     dbrfx.obj
 0002:00002988       ??_C@_1GE@KBIF@?$AAW?$AAa?$AAr?$AAn?$AAi?$AAn?$AAg?$AA?3?$AA?5?$AAC?$AAB?$AAy?$AAt?$AAe?$AAA?$AAr?$AAr?$AAa?$AAy?$AA?5@ 5f733988     dbrfx.obj
 0002:000029ec       ??_C@_1EC@JJBD@?$AAW?$AAa?$AAr?$AAn?$AAi?$AAn?$AAg?$AA?3?$AA?5?$AAi?$AAg?$AAn?$AAo?$AAr?$AAi?$AAn?$AAg?$AA?5?$AAm?$AAi@ 5f7339ec     dbrfx.obj
 0002:00002a30       ??_C@_1HC@POCA@?$AAW?$AAa?$AAr?$AAn?$AAi?$AAn?$AAg?$AA?3?$AA?5?$AAd?$AAa?$AAt?$AAe?$AA?5?$AAv?$AAa?$AAl?$AAu?$AAe?$AA?5@ 5f733a30     dbrfx.obj
 0002:00002aa4       ??_C@_1FK@JFDN@?$AAW?$AAa?$AAr?$AAn?$AAi?$AAn?$AAg?$AA?3?$AA?5?$AAC?$AAT?$AAi?$AAm?$AAe?$AA?5?$AAc?$AAo?$AAn?$AAv?$AAe@ 5f733aa4     dbrfx.obj
 0002:00002b00       ??_C@_0N@OGBI@?4fraction?5?$DN?5?$AA@ 5f733b00     dbrfx.obj
 0002:00002b10       ??_C@_0L@BFHB@?4second?5?$DN?5?$AA@ 5f733b10     dbrfx.obj
 0002:00002b1c       ??_C@_0L@JFIG@?4minute?5?$DN?5?$AA@ 5f733b1c     dbrfx.obj
 0002:00002b28       ??_C@_08PGJP@?4hour?5?$DN?5?$AA@ 5f733b28     dbrfx.obj
 0002:00002b34       ??_C@_07JEIM@?4day?5?$DN?5?$AA@ 5f733b34     dbrfx.obj
 0002:00002b3c       ??_C@_09DKMF@?4month?5?$DN?5?$AA@ 5f733b3c     dbrfx.obj
 0002:00002b48       ??_C@_08DFNB@?4year?5?$DN?5?$AA@ 5f733b48     dbrfx.obj
 0002:00002b54       ??_C@_1HA@GLOK@?$AAW?$AAa?$AAr?$AAn?$AAi?$AAn?$AAg?$AA?3?$AA?5?$AAT?$AAI?$AAM?$AAE?$AAS?$AAT?$AAA?$AAM?$AAP?$AA_?$AAS@ 5f733b54     dbrfx.obj
 0002:00002bc4       ??_C@_1GI@EJOD@?$AAW?$AAa?$AAr?$AAn?$AAi?$AAn?$AAg?$AA?3?$AA?5?$AAC?$AAO?$AAl?$AAe?$AAD?$AAa?$AAt?$AAe?$AAT?$AAi?$AAm@ 5f733bc4     dbrfx.obj
 0002:00002c2c       ??_C@_1BI@HDAA@?$AAS?$AAt?$AAa?$AAt?$AAe?$AA?3?$AA0?$AA1?$AA0?$AA0?$AA4?$AA?$AA@ 5f733c2c     dbrfx.obj
 0002:00002c48       ?classCRecordView@CRecordView@@2UCRuntimeClass@@B 5f733c48     dbview.obj
 0002:00002c60       ??_C@_0M@EAFL@CRecordView?$AA@ 5f733c60     dbview.obj
 0002:00002c70       ?messageMap@CRecordView@@1UAFX_MSGMAP@@B 5f733c70     dbview.obj
 0002:00002c78       ?_messageEntries@CRecordView@@0QBUAFX_MSGMAP_ENTRY@@B 5f733c78     dbview.obj
 0002:00002d54       ??_7CRecordView@@6B@       5f733d54     dbview.obj
 0002:00002e6c       ??_C@_1EI@FFBM@?$AAW?$AAa?$AAr?$AAn?$AAi?$AAn?$AAg?$AA?3?$AA?5?$AAn?$AAo?$AA?5?$AAl?$AAi?$AAs?$AAt?$AAb?$AAo?$AAx?$AA?5@ 5f733e6c     dbview.obj
 0002:00002eb4       ??_C@_1EK@OEMJ@?$AAW?$AAa?$AAr?$AAn?$AAi?$AAn?$AAg?$AA?3?$AA?5?$AAn?$AAo?$AA?5?$AAc?$AAo?$AAm?$AAb?$AAo?$AAb?$AAo?$AAx@ 5f733eb4     dbview.obj
 0002:00002f00       ??_C@_1HA@DPGA@?$AAW?$AAa?$AAr?$AAn?$AAi?$AAn?$AAg?$AA?3?$AA?5?$AAd?$AAi?$AAa?$AAl?$AAo?$AAg?$AA?5?$AAd?$AAa?$AAt?$AAa@ 5f733f00     dbview.obj
 0002:00002f70       ??_C@_1HE@NOFM@?$AAW?$AAa?$AAr?$AAn?$AAi?$AAn?$AAg?$AA?3?$AA?5?$AAf?$AAi?$AAe?$AAl?$AAd?$AA?5?$AAN?$AAU?$AAL?$AAL?$AA?5@ 5f733f70     dbview.obj
 0002:00002fe4       ??_C@_1IA@HLN@?$AAW?$AAa?$AAr?$AAn?$AAi?$AAn?$AAg?$AA?3?$AA?5?$AAc?$AAh?$AAe?$AAc?$AAk?$AAb?$AAo?$AAx?$AA?5?$AAv?$AAa@ 5f733fe4     dbview.obj
 0002:00003064       ??_C@_0BE@JDG@?6m_bOnLastRecord?5?$DN?5?$AA@ 5f734064     dbview.obj
 0002:00003078       ??_C@_0BE@GCEL@m_bOnFirstRecord?5?$DN?5?$AA@ 5f734078     dbview.obj
 0002:000030a0       ??_C@_1FK@HFKA@?$AAW?$AAa?$AAr?$AAn?$AAi?$AAn?$AAg?$AA?3?$AA?5?$AAf?$AAl?$AAo?$AAa?$AAt?$AA?5?$AAc?$AAo?$AAn?$AAv?$AAe@ 5f7340a0     dbflt.obj
 0002:000030fc       ??_C@_1FM@EACM@?$AAW?$AAa?$AAr?$AAn?$AAi?$AAn?$AAg?$AA?3?$AA?5?$AAd?$AAo?$AAu?$AAb?$AAl?$AAe?$AA?5?$AAc?$AAo?$AAn?$AAv@ 5f7340fc     dbflt.obj
 0002:00003158       ?classCLongBinary@CLongBinary@@2UCRuntimeClass@@B 5f734158     dblong.obj
 0002:00003170       ??_C@_0M@DJA@CLongBinary?$AA@ 5f734170     dblong.obj
 0002:00003180       ??_7CLongBinary@@6B@       5f734180     dblong.obj
 0002:00003194       ??_C@_0BD@HHCG@?6m_dwDataLength?5?$DN?5?$AA@ 5f734194     dblong.obj
 0002:000031a8       ??_C@_0L@DGJD@m_hData?5?$DN?5?$AA@ 5f7341a8     dblong.obj
 0002:000031b8       ??_7CDBVariant@@6B@        5f7341b8     dbvar.obj
 0002:000031c0       ?classCDaoRecordset@CDaoRecordset@@2UCRuntimeClass@@B 5f7341c0     daocore.obj
 0002:000031d8       ??_C@_0O@JOIL@CDaoRecordset?$AA@ 5f7341d8     daocore.obj
 0002:000031e8       ?classCDaoQueryDef@CDaoQueryDef@@2UCRuntimeClass@@B 5f7341e8     daocore.obj
 0002:00003200       ??_C@_0N@NGH@CDaoQueryDef?$AA@ 5f734200     daocore.obj
 0002:00003210       ?classCDaoTableDef@CDaoTableDef@@2UCRuntimeClass@@B 5f734210     daocore.obj
 0002:00003228       ??_C@_0N@PHMG@CDaoTableDef?$AA@ 5f734228     daocore.obj
 0002:00003238       ?classCDaoDatabase@CDaoDatabase@@2UCRuntimeClass@@B 5f734238     daocore.obj
 0002:00003250       ??_C@_0N@DDLP@CDaoDatabase?$AA@ 5f734250     daocore.obj
 0002:00003260       ?classCDaoWorkspace@CDaoWorkspace@@2UCRuntimeClass@@B 5f734260     daocore.obj
 0002:00003278       ??_C@_0O@IEJG@CDaoWorkspace?$AA@ 5f734278     daocore.obj
 0002:00003288       ?classCDaoException@CDaoException@@2UCRuntimeClass@@B 5f734288     daocore.obj
 0002:000032a0       ??_C@_0O@OIMH@CDaoException?$AA@ 5f7342a0     daocore.obj
 0002:000032b0       ?_afxTable2@@3QBGB         5f7342b0     daocore.obj
 0002:000032c0       ?_afxTransform2@@3QBGB     5f7342c0     daocore.obj
 0002:000032d8       ?_afxOrderBy2@@3QBGB       5f7342d8     daocore.obj
 0002:000032f0       ?_afxWhere2@@3QBGB         5f7342f0     daocore.obj
 0002:00003300       ?_afxFrom2@@3QBGB          5f734300     daocore.obj
 0002:00003310       ?_afxSelect2@@3QBGB        5f734310     daocore.obj
 0002:00003320       ?_afxParameters2@@3QBGB    5f734320     daocore.obj
 0002:0000333c       ??_7_AFX_DAO_STATE@@6B@    5f73433c     daocore.obj
 0002:00003340       ??_C@_1BM@FCKC@?$AA?6?$AA?7?$AAs?$AAc?$AAo?$AAd?$AAe?$AA?5?$AA?$DN?$AA?5?$AA?$CF?$AAX?$AA?6?$AA?$AA@ 5f734340     daocore.obj
 0002:0000335c       ??_C@_1DC@ENFN@?$AA?6?$AA?7?$AAI?$AAn?$AA?5?$AAf?$AAi?$AAl?$AAe?$AA?5?$AA?$CF?$AAh?$AAs?$AA?5?$AAo?$AAn?$AA?5?$AAl?$AAi?$AAn@ 5f73435c     daocore.obj
 0002:00003390       ??_C@_1M@LOF@?$AA?6?$AA?7?$AA?$CF?$AAh?$AAs?$AA?$AA@ 5f734390     daocore.obj
 0002:0000339c       ??_C@_1CE@CGEC@?$AA?6?$AAD?$AAA?$AAO?$AA?5?$AAC?$AAa?$AAl?$AAl?$AA?5?$AAF?$AAa?$AAi?$AAl?$AAe?$AAd?$AA?4?$AA?$AA@ 5f73439c     daocore.obj
 0002:000033c0       ??_C@_1BI@OIDH@?$AAs?$AAc?$AAo?$AAd?$AAe?$AA?5?$AA?$DN?$AA?5?$AA?$CF?$AAX?$AA?6?$AA?$AA@ 5f7343c0     daocore.obj
 0002:000033d8       ??_C@_1DC@NDDC@?$AA?6?$AAI?$AAn?$AA?5?$AAf?$AAi?$AAl?$AAe?$AA?5?$AA?$CF?$AAh?$AAs?$AA?5?$AAo?$AAn?$AA?5?$AAl?$AAi?$AAn?$AAe@ 5f7343d8     daocore.obj
 0002:0000340c       ??_C@_19MMFM@?$AA?6?$AA?$CF?$AAh?$AAs?$AA?$AA@ 5f73440c     daocore.obj
 0002:00003418       ??_C@_1CI@BBLE@?$AA?6?$AAD?$AAA?$AAO?$AA?5?$AAC?$AAa?$AAl?$AAl?$AA?5?$AAF?$AAa?$AAi?$AAl?$AAe?$AAd?$AA?4?$AA?6?$AA?7?$AA?$AA@ 5f734418     daocore.obj
 0002:00003440       ??_C@_0BD@JMBE@?6m_lHelpContext?5?$DN?5?$AA@ 5f734440     daocore.obj
 0002:00003454       ??_C@_0BC@FOHM@?6m_strHelpFile?5?$DN?5?$AA@ 5f734454     daocore.obj
 0002:00003468       ??_C@_0BF@JHNL@?6m_strDescription?5?$DN?5?$AA@ 5f734468     daocore.obj
 0002:00003480       ??_C@_0BA@HMPD@?6m_strSource?5?$DN?5?$AA@ 5f734480     daocore.obj
 0002:00003490       ??_C@_0BB@CCFD@?6m_lErrorCode?5?$DN?5?$AA@ 5f734490     daocore.obj
 0002:000034a4       ??_C@_0BE@OGG@a?5CDaoErrorInfo?5at?5?$AA@ 5f7344a4     daocore.obj
 0002:000034b8       ??_C@_0BJ@HLFP@?6b?5?$DN?5m_bIsolateODBCTrans?$AA@ 5f7344b8     daocore.obj
 0002:000034d4       ??_C@_0BC@HDK@?6m_strUserName?5?$DN?5?$AA@ 5f7344d4     daocore.obj
 0002:000034e8       ??_C@_0O@FEGP@?6m_strName?5?$DN?5?$AA@ 5f7344e8     daocore.obj
 0002:000034f8       ??_C@_0BI@EJIL@a?5CDaoWorkspaceInfo?5at?5?$AA@ 5f7344f8     daocore.obj
 0002:00003510       ??_C@_0BE@JLEN@?6m_nQueryTimeout?5?$DN?5?$AA@ 5f734510     daocore.obj
 0002:00003524       ??_C@_0BG@ILBM@?6m_lCollatingOrder?5?$DN?5?$AA@ 5f734524     daocore.obj
 0002:0000353c       ??_C@_0BB@LEGM@?6m_strVersion?5?$DN?5?$AA@ 5f73453c     daocore.obj
 0002:00003550       ??_C@_0BH@FIEC@a?5CDaoDatabaseInfo?5at?5?$AA@ 5f734550     daocore.obj
 0002:00003568       ??_C@_0BD@FJAC@?6m_lRecordCount?5?$DN?5?$AA@ 5f734568     daocore.obj
 0002:0000357c       ??_C@_0BI@JMNH@?6m_strValidationText?5?$DN?5?$AA@ 5f73457c     daocore.obj
 0002:00003594       ??_C@_0BI@NDBL@?6m_strValidationRule?5?$DN?5?$AA@ 5f734594     daocore.obj
 0002:000035ac       ??_C@_0BG@FOBO@?6m_strSrcTableName?5?$DN?5?$AA@ 5f7345ac     daocore.obj
 0002:000035c4       ??_C@_0BG@PCL@?6m_dateLastUpdated?5?$DN?5?$AA@ 5f7345c4     daocore.obj
 0002:000035dc       ??_C@_0BG@FOFB@?6m_dateDateCreated?5?$DN?5?$AA@ 5f7345dc     daocore.obj
 0002:000035f4       ??_C@_0BC@KBNC@?6m_lAttributes?5?$DN?5?$AA@ 5f7345f4     daocore.obj
 0002:00003608       ??_C@_0BH@JFIA@a?5CDaoTableDefInfo?5at?5?$AA@ 5f734608     daocore.obj
 0002:00003620       ??_C@_0BG@MHMB@?6m_strDefaultValue?5?$DN?5?$AA@ 5f734620     daocore.obj
 0002:00003638       ??_C@_0BF@HCFN@?6m_strSourceTable?5?$DN?5?$AA@ 5f734638     daocore.obj
 0002:00003650       ??_C@_0BF@NJHG@?6m_strSourceField?5?$DN?5?$AA@ 5f734650     daocore.obj
 0002:00003668       ??_C@_0BF@KILJ@?6m_strForeignName?5?$DN?5?$AA@ 5f734668     daocore.obj
 0002:00003680       ??_C@_0BH@BCFG@?6m_bAllowZeroLength?5?$DN?5?$AA@ 5f734680     daocore.obj
 0002:00003698       ??_C@_0BA@OOHL@?6m_bRequired?5?$DN?5?$AA@ 5f734698     daocore.obj
 0002:000036a8       ??_C@_0BH@IMAL@?6m_nOrdinalPosition?5?$DN?5?$AA@ 5f7346a8     daocore.obj
 0002:000036c0       ??_C@_0M@EOEG@?6m_lSize?5?$DN?5?$AA@ 5f7346c0     daocore.obj
 0002:000036cc       ??_C@_0M@MJB@?6m_nType?5?$DN?5?$AA@ 5f7346cc     daocore.obj
 0002:000036d8       ??_C@_0BE@PODE@a?5CDaoFieldInfo?5at?5?$AA@ 5f7346d8     daocore.obj
 0002:000036ec       ??_C@_0BC@ILAA@?6m_bDescending?5?$DN?5?$AA@ 5f7346ec     daocore.obj
 0002:00003700       ??_C@_0BK@KCFC@?5a?5CDaoIndexFieldInfo?5at?5?$AA@ 5f734700     daocore.obj
 0002:00003720       ??_7CDaoIndexInfo@@6B@     5f734720     daocore.obj
 0002:00003728       ??_C@_0BF@LIJD@?6m_lDistinctCount?5?$DN?5?$AA@ 5f734728     daocore.obj
 0002:00003740       ??_C@_0P@DLHL@?6m_bForeign?5?$DN?5?$AA@ 5f734740     daocore.obj
 0002:00003750       ??_C@_0BD@MAED@?6m_bIgnoreNulls?5?$DN?5?$AA@ 5f734750     daocore.obj
 0002:00003764       ??_C@_0BB@FFL@?6m_bClustered?5?$DN?5?$AA@ 5f734764     daocore.obj
 0002:00003778       ??_C@_0O@NMC@?6m_bUnique?5?$DN?5?$AA@ 5f734778     daocore.obj
 0002:00003788       ??_C@_0P@FFEB@?6m_bPrimary?5?$DN?5?$AA@ 5f734788     daocore.obj
 0002:00003798       ??_C@_0BE@OGHD@a?5CDaoIndexInfo?5at?5?$AA@ 5f734798     daocore.obj
 0002:000037ac       ??_C@_0BN@BEAM@?5a?5CDaoRelationFieldInfo?5at?5?$AA@ 5f7347ac     daocore.obj
 0002:000037d0       ??_7CDaoRelationInfo@@6B@  5f7347d0     daocore.obj
 0002:000037d8       ??_C@_0BG@NBH@?6m_strForeignTable?5?$DN?5?$AA@ 5f7347d8     daocore.obj
 0002:000037f0       ??_C@_0P@CHOL@?6m_strTable?5?$DN?5?$AA@ 5f7347f0     daocore.obj
 0002:00003800       ??_C@_0BH@ICPE@a?5CDaoRelationInfo?5at?5?$AA@ 5f734800     daocore.obj
 0002:00003818       ??_C@_0BD@BKGA@?6m_nODBCTimeout?5?$DN?5?$AA@ 5f734818     daocore.obj
 0002:0000382c       ??_C@_0BG@JDEE@?6m_bReturnsRecords?5?$DN?5?$AA@ 5f73482c     daocore.obj
 0002:00003844       ??_C@_0BC@DDHJ@?6m_dateCreated?5?$DN?5?$AA@ 5f734844     daocore.obj
 0002:00003858       ??_C@_0BH@OPB@a?5CDaoQueryDefInfo?5at?5?$AA@ 5f734858     daocore.obj
 0002:00003870       ??_C@_0P@MIHC@?6m_varValue?5?$DN?5?$AA@ 5f734870     daocore.obj
 0002:00003880       ??_C@_0BI@NAFD@a?5CDaoParameterInfo?5at?5?$AA@ 5f734880     daocore.obj
 0002:0000389c       ??_7CDaoException@@6B@     5f73489c     daocore.obj
 0002:000038b8       ??_C@_0CC@NFIM@m_pDAOErrors?9?$DOget_Count?$CI?$CGnErrors@ 5f7348b8     daocore.obj
 0002:000038dc       ??_C@_0EB@MBDI@m_pDAOErrors?9?$DOget_Item?$CI?5COleVari@ 5f7348dc     daocore.obj
 0002:00003920       ??_C@_0DG@CEPE@pDaoState?9?$DOm_pDAODBEngine?9?$DOget_E@ 5f734920     daocore.obj
 0002:00003958       ??_C@_0DN@LLAK@m_pDAOError?9?$DOget_HelpContext?$CI?5?$CGm@ 5f734958     daocore.obj
 0002:00003998       ??_C@_0CJ@LALL@m_pDAOError?9?$DOget_HelpFile?$CI?$CGV_BST@ 5f734998     daocore.obj
 0002:000039c4       ??_C@_0CM@BAFD@m_pDAOError?9?$DOget_Description?$CI?$CGV_@ 5f7349c4     daocore.obj
 0002:000039f0       ??_C@_0CH@NNNO@m_pDAOError?9?$DOget_Source?$CI?$CGV_BSTR?$CI@ 5f7349f0     daocore.obj
 0002:00003a18       ??_C@_0DG@GHAH@m_pDAOError?9?$DOget_Number?$CI?5?$CGm_pErr@ 5f734a18     daocore.obj
 0002:00003a54       ??_7CDaoErrorInfo@@6B@     5f734a54     daocore.obj
 0002:00003a58       ??_C@_1CE@BPEH@?$AAD?$AAe?$AAs?$AAc?$AAr?$AAi?$AAp?$AAt?$AAi?$AAo?$AAn?$AA?5?$AA?$DN?$AA?5?$AA?$CF?$AAs?$AA?6?$AA?$AA@ 5f734a58     daocore.obj
 0002:00003a7c       ??_C@_1BK@LBAO@?$AAS?$AAo?$AAu?$AAr?$AAc?$AAe?$AA?5?$AA?$DN?$AA?5?$AA?$CF?$AAs?$AA?6?$AA?$AA@ 5f734a7c     daocore.obj
 0002:00003a98       ??_C@_1CE@GONH@?$AA?6?$AAE?$AAr?$AAr?$AAo?$AAr?$AA?5?$AAC?$AAo?$AAd?$AAe?$AA?5?$AA?$DN?$AA?5?$AA?$CF?$AAd?$AA?6?$AA?$AA@ 5f734a98     daocore.obj
 0002:00003ac0       ??_7CDaoWorkspace@@6B@     5f734ac0     daocore.obj
 0002:00003ae8       ??_C@_0IA@IMA@pDaoState?9?$DOm_pDAODBEngine?9?$DO_30_C@ 5f734ae8     daocore.obj
 0002:00003b68       ??_C@_0CI@OLEJ@pDAOWorkspaces?9?$DOAppend?$CIm_pDAOWor@ 5f734b68     daocore.obj
 0002:00003b90       ??_C@_0DL@KMOM@pDaoState?9?$DOm_pDAODBEngine?9?$DOget_W@ 5f734b90     daocore.obj
 0002:00003bcc       ??_C@_0DC@BHKN@m_pDAOWorkspaces?9?$DOget_Item?$CIvar?0?5@ 5f734bcc     daocore.obj
 0002:00003c00       ??_C@_0DO@NCLP@pDaoState?9?$DOm_pDAODBEngine?9?$DOget_W@ 5f734c00     daocore.obj
 0002:00003c40       ??_C@_0BJ@BAIF@m_pDAOWorkspace?9?$DOClose?$CI?$CJ?$AA@ 5f734c40     daocore.obj
 0002:00003c5c       ??_C@_0DG@EKI@pDaoState?9?$DOm_pDAODBEngine?9?$DOget_V@ 5f734c5c     daocore.obj
 0002:00003c94       ??_C@_0DG@POMJ@pDaoState?9?$DOm_pDAODBEngine?9?$DOget_I@ 5f734c94     daocore.obj
 0002:00003ccc       ??_C@_0DF@FAOI@pDaoState?9?$DOm_pDAODBEngine?9?$DOput_I@ 5f734ccc     daocore.obj
 0002:00003d04       ??_C@_0DJ@GIII@pDaoState?9?$DOm_pDAODBEngine?9?$DOput_D@ 5f734d04     daocore.obj
 0002:00003d40       ??_C@_0DO@ONCK@pDaoState?9?$DOm_pDAODBEngine?9?$DOput_D@ 5f734d40     daocore.obj
 0002:00003d80       ??_C@_0DH@FIK@pDaoState?9?$DOm_pDAODBEngine?9?$DOget_L@ 5f734d80     daocore.obj
 0002:00003db8       ??_C@_0DG@FCKN@pDaoState?9?$DOm_pDAODBEngine?9?$DOput_L@ 5f734db8     daocore.obj
 0002:00003df0       ??_C@_0CJ@PIID@m_pDAOWorkspace?9?$DOget_Name?$CI?$CGV_BST@ 5f734df0     daocore.obj
 0002:00003e1c       ??_C@_0CN@LNMJ@m_pDAOWorkspace?9?$DOget_UserName?$CI?$CGV@ 5f734e1c     daocore.obj
 0002:00003e4c       ??_C@_0GC@MAIK@m_pDAOWorkspace?9?$DOput_IsolateODBC@ 5f734e4c     daocore.obj
 0002:00003eb0       ??_C@_0DK@BNMM@m_pDAOWorkspace?9?$DOget_IsolateODBC@ 5f734eb0     daocore.obj
 0002:00003eec       ??_C@_0PC@HCAP@pDaoState?9?$DOm_pDAODBEngine?9?$DOCompa@ 5f734eec     daocore.obj
 0002:00003fe0       ??_C@_0DN@CKIJ@pDaoState?9?$DOm_pDAODBEngine?9?$DORepai@ 5f734fe0     daocore.obj
 0002:00004020       ??_C@_0DN@BCJE@pDaoState?9?$DOm_pDAODBEngine?9?$DOIdle?$CI@ 5f735020     daocore.obj
 0002:00004060       ??_C@_0CG@MKCN@m_pDAOWorkspaces?9?$DOget_Count?$CI?$CGnFi@ 5f735060     daocore.obj
 0002:00004088       ??_C@_0EH@MIPG@m_pDAOWorkspaces?9?$DOget_Item?$CI?5COle@ 5f735088     daocore.obj
 0002:000040d0       ??_C@_0EN@CDCO@m_pDAOWorkspaces?9?$DOget_Item?$CI?5COle@ 5f7350d0     daocore.obj
 0002:00004120       ??_C@_0CF@NKKO@m_pDAODatabases?9?$DOget_Count?$CI?$CGnFie@ 5f735120     daocore.obj
 0002:00004148       ??_C@_0EF@MAIH@m_pDAODatabases?9?$DOget_Item?$CI?5COleV@ 5f735148     daocore.obj
 0002:00004190       ??_C@_0EL@BNEE@m_pDAODatabases?9?$DOget_Item?$CI?5COleV@ 5f735190     daocore.obj
 0002:000041dc       ??_C@_0BO@IBKO@m_pDAOWorkspace?9?$DOBeginTrans?$CI?$CJ?$AA@ 5f7351dc     daocore.obj
 0002:000041fc       ??_C@_0BO@ONLB@?$CIm_pDAOWorkspace?9?$DO?$CKpMethod?$CJ?$CI?$CJ?$AA@ 5f7351fc     daocore.obj
 0002:0000421c       ??_C@_0CA@PBAE@m_pDAOWorkspace?9?$DOCommitTrans?$CI0?$CJ?$AA@ 5f73521c     daocore.obj
 0002:0000423c       ??_C@_0BM@BBEN@m_pDAOWorkspace?9?$DORollback?$CI?$CJ?$AA@ 5f73523c     daocore.obj
 0002:00004258       ??_C@_0CM@PHDL@pDAOWorkspace?9?$DOget_IsolateODBCTr@ 5f735258     daocore.obj
 0002:00004284       ??_C@_0CL@LFDC@pDAOWorkspace?9?$DOget_UserName?$CI?$CGV_B@ 5f735284     daocore.obj
 0002:000042b0       ??_C@_0CH@NIA@pDAOWorkspace?9?$DOget_Name?$CI?$CGV_BSTR?$CI@ 5f7352b0     daocore.obj
 0002:000042d8       ??_C@_0DB@FMO@m_pDAOWorkspace?9?$DOget_Databases?$CI?$CG@ 5f7352d8     daocore.obj
 0002:0000430c       ??_C@_0CK@GLDA@pDAODatabase?9?$DOget_Connect?$CI?5?$CGV_BS@ 5f73530c     daocore.obj
 0002:00004338       ??_C@_0DJ@LMDF@pDAODatabase?9?$DOget_QueryTimeout?$CI?5@ 5f735338     daocore.obj
 0002:00004374       ??_C@_0DN@CAFO@pDAODatabase?9?$DOget_CollatingOrder@ 5f735374     daocore.obj
 0002:000043b4       ??_C@_0CK@LGL@pDAODatabase?9?$DOget_Version?$CI?5?$CGV_BS@ 5f7353b4     daocore.obj
 0002:000043e0       ??_C@_0CH@GLGK@pDAODatabase?9?$DOget_Transactions?$CI?$CG@ 5f7353e0     daocore.obj
 0002:00004408       ??_C@_0CE@GDMB@pDAODatabase?9?$DOget_Updatable?$CI?$CGnBo@ 5f735408     daocore.obj
 0002:0000442c       ??_C@_0CG@GEI@pDAODatabase?9?$DOget_Name?$CI?$CGV_BSTR?$CI?$CG@ 5f73542c     daocore.obj
 0002:00004454       ??_C@_0O@KPOJ@?6m_nStatus?5?$DN?5?$AA@ 5f735454     daocore.obj
 0002:00004464       ??_C@_0L@OLPD@?6m_bNew?5?$DN?5?$AA@ 5f735464     daocore.obj
 0002:00004470       ??_C@_0L@FNFF@m_bOpen?5?$DN?5?$AA@ 5f735470     daocore.obj
 0002:00004480       ??_7CDaoDatabase@@6B@      5f735480     daocore.obj
 0002:000044a4       ??_C@_0IC@FKK@m_pWorkspace?9?$DOm_pDAOWorkspace?9?$DOC@ 5f7354a4     daocore.obj
 0002:00004528       ??_C@_0LP@CIKN@m_pWorkspace?9?$DOm_pDAOWorkspace?9?$DOO@ 5f735528     daocore.obj
 0002:000045e8       ??_C@_0BI@NBCE@m_pDAODatabase?9?$DOClose?$CI?$CJ?$AA@ 5f7355e8     daocore.obj
 0002:00004600       ??_C@_0CL@ELFI@m_pDAODatabase?9?$DOget_Updatable?$CI?$CGn@ 5f735600     daocore.obj
 0002:0000462c       ??_C@_0DB@POJO@m_pDAODatabase?9?$DOget_Transactions@ 5f73562c     daocore.obj
 0002:00004660       ??_C@_0CI@FCO@m_pDAODatabase?9?$DOget_Name?$CI?$CGV_BSTR@ 5f735660     daocore.obj
 0002:00004688       ??_C@_0CL@OIPD@m_pDAODatabase?9?$DOget_Connect?$CI?$CGV_B@ 5f735688     daocore.obj
 0002:000046b4       ??_C@_0CL@LDKH@m_pDAODatabase?9?$DOget_Version?$CI?$CGV_B@ 5f7356b4     daocore.obj
 0002:000046e0       ??_C@_0DB@NKM@m_pDAODatabase?9?$DOget_QueryTimeout@ 5f7356e0     daocore.obj
 0002:00004714       ??_C@_0CL@CMOO@m_pDAODatabase?9?$DOput_QueryTimeout@ 5f735714     daocore.obj
 0002:00004740       ??_C@_0DH@EED@m_pDAODatabase?9?$DOget_RecordsAffec@ 5f735740     daocore.obj
 0002:00004778       ??_C@_0CG@DPNF@m_pDAOTableDefs?9?$DODelete?$CIV_BSTR?$CI?$CG@ 5f735778     daocore.obj
 0002:000047a0       ??_C@_0CG@PEFD@m_pDAOQueryDefs?9?$DODelete?$CIV_BSTR?$CI?$CG@ 5f7357a0     daocore.obj
 0002:000047cc       ??_7CDaoRelationFieldInfo@@6B@ 5f7357cc     daocore.obj
 0002:000047d0       ??_C@_0CG@KOHE@m_pDAORelations?9?$DOAppend?$CIpDAORela@ 5f7357d0     daocore.obj
 0002:000047f8       ??_C@_0BO@PKCL@pDAOFields?9?$DOAppend?$CIpDAOField?$CJ?$AA@ 5f7357f8     daocore.obj
 0002:00004818       ??_C@_0CJ@GPBE@pDAOField?9?$DOput_ForeignName?$CIV_BST@ 5f735818     daocore.obj
 0002:00004844       ??_C@_0JB@FHMF@pDAORelation?9?$DOCreateField?$CI?5COleV@ 5f735844     daocore.obj
 0002:000048d8       ??_C@_0CG@INKG@pDAORelation?9?$DOget_Fields?$CI?$CGpDAOFi@ 5f7358d8     daocore.obj
 0002:00004900       ??_C@_0NK@LJKP@m_pDAODatabase?9?$DOCreateRelation?$CI?5@ 5f735900     daocore.obj
 0002:000049dc       ??_C@_0CG@BJFH@m_pDAORelations?9?$DODelete?$CIV_BSTR?$CI?$CG@ 5f7359dc     daocore.obj
 0002:00004a04       ??_C@_0EE@KEMK@m_pDAODatabase?9?$DOExecute?$CI?5V_BSTR?$CI@ 5f735a04     daocore.obj
 0002:00004a48       ??_C@_0CF@JLMN@m_pDAOTableDefs?9?$DOget_Count?$CI?$CGnTab@ 5f735a48     daocore.obj
 0002:00004a70       ??_C@_0EF@FBLA@m_pDAOTableDefs?9?$DOget_Item?$CI?5COleV@ 5f735a70     daocore.obj
 0002:00004ab8       ??_C@_0EL@KPGC@m_pDAOTableDefs?9?$DOget_Item?$CI?5COleV@ 5f735ab8     daocore.obj
 0002:00004b04       ??_C@_0CI@LDJE@m_pDAORelations?9?$DOget_Count?$CI?$CGnRel@ 5f735b04     daocore.obj
 0002:00004b2c       ??_C@_0EF@IIIA@m_pDAORelations?9?$DOget_Item?$CI?5COleV@ 5f735b2c     daocore.obj
 0002:00004b74       ??_C@_0EL@IHJB@m_pDAORelations?9?$DOget_Item?$CI?5COleV@ 5f735b74     daocore.obj
 0002:00004bc0       ??_C@_0CI@MEAB@m_pDAOQueryDefs?9?$DOget_Count?$CI?$CGnQue@ 5f735bc0     daocore.obj
 0002:00004be8       ??_C@_0EF@NBOE@m_pDAOQueryDefs?9?$DOget_Item?$CI?5COleV@ 5f735be8     daocore.obj
 0002:00004c30       ??_C@_0EL@IINM@m_pDAOQueryDefs?9?$DOget_Item?$CI?5COleV@ 5f735c30     daocore.obj
 0002:00004c7c       ??_C@_0DA@GLPP@m_pDAODatabase?9?$DOget_TableDefs?$CI?$CGm@ 5f735c7c     daocore.obj
 0002:00004cac       ??_C@_0DN@PBMP@pDAOTableDef?9?$DOget_RecordCount?$CI?5?$CG@ 5f735cac     daocore.obj
 0002:00004cec       ??_C@_0DB@KOFA@pDAOTableDef?9?$DOget_ValidationText@ 5f735cec     daocore.obj
 0002:00004d20       ??_C@_0DB@HJKE@pDAOTableDef?9?$DOget_ValidationRule@ 5f735d20     daocore.obj
 0002:00004d54       ??_C@_0CK@LEHN@pDAOTableDef?9?$DOget_Connect?$CI?5?$CGV_BS@ 5f735d54     daocore.obj
 0002:00004d80       ??_C@_0DC@BFFJ@pDAOTableDef?9?$DOget_SourceTableNam@ 5f735d80     daocore.obj
 0002:00004db4       ??_C@_0CE@FNDA@pDAOTableDef?9?$DOget_LastUpdated?$CI?$CGv@ 5f735db4     daocore.obj
 0002:00004dd8       ??_C@_0CE@NEPA@pDAOTableDef?9?$DOget_DateCreated?$CI?$CGv@ 5f735dd8     daocore.obj
 0002:00004dfc       ??_C@_0DL@DLNJ@pDAOTableDef?9?$DOget_Attributes?$CI?5?$CGt@ 5f735dfc     daocore.obj
 0002:00004e38       ??_C@_0CE@GAKL@pDAOTableDef?9?$DOget_Updatable?$CI?$CGnBo@ 5f735e38     daocore.obj
 0002:00004e5c       ??_C@_0CG@GGLM@pDAOTableDef?9?$DOget_Name?$CI?$CGV_BSTR?$CI?$CG@ 5f735e5c     daocore.obj
 0002:00004e84       ??_C@_0DA@JLIC@m_pDAODatabase?9?$DOget_Relations?$CI?$CGm@ 5f735e84     daocore.obj
 0002:00004eb4       ??_C@_0CK@LAFA@pDAOField?9?$DOget_ForeignName?$CI?$CGV_BS@ 5f735eb4     daocore.obj
 0002:00004ee0       ??_C@_0CD@BJOA@pDAOField?9?$DOget_Name?$CI?$CGV_BSTR?$CI?$CGvar@ 5f735ee0     daocore.obj
 0002:00004f04       ??_C@_0DN@MJFF@pDAOFields?9?$DOget_Item?$CI?5COleVarian@ 5f735f04     daocore.obj
 0002:00004f44       ??_C@_0BP@FFPK@pDAOFields?9?$DOget_Count?$CI?$CGnCount?$CJ?$AA@ 5f735f44     daocore.obj
 0002:00004f64       ??_C@_0DG@DMNE@pDAORelation?9?$DOget_Attributes?$CI?5?$CGr@ 5f735f64     daocore.obj
 0002:00004f9c       ??_C@_0CP@PIMH@pDAORelation?9?$DOget_ForeignTable?$CI?5@ 5f735f9c     daocore.obj
 0002:00004fcc       ??_C@_0CH@LDAN@pDAORelation?9?$DOget_Table?$CI?$CGV_BSTR?$CI@ 5f735fcc     daocore.obj
 0002:00004ff4       ??_C@_0CG@NDBG@pDAORelation?9?$DOget_Name?$CI?$CGV_BSTR?$CI?$CG@ 5f735ff4     daocore.obj
 0002:0000501c       ??_C@_0DA@BPAN@m_pDAODatabase?9?$DOget_QueryDefs?$CI?$CGm@ 5f73601c     daocore.obj
 0002:0000504c       ??_C@_0DE@DPOF@pDAOQueryDef?9?$DOget_Connect?$CI?$CGV_BST@ 5f73604c     daocore.obj
 0002:00005080       ??_C@_0CF@HFEL@pDAOQueryDef?9?$DOget_SQL?$CI?$CGV_BSTR?$CI?$CGv@ 5f736080     daocore.obj
 0002:000050a8       ??_C@_0CJ@KFGF@pDAOQueryDef?9?$DOget_ReturnsRecords@ 5f7360a8     daocore.obj
 0002:000050d4       ??_C@_0CE@JGLG@pDAOQueryDef?9?$DOget_LastUpdated?$CI?$CGv@ 5f7360d4     daocore.obj
 0002:000050f8       ??_C@_0CE@BPHG@pDAOQueryDef?9?$DOget_DateCreated?$CI?$CGv@ 5f7360f8     daocore.obj
 0002:0000511c       ??_C@_0CE@KLCN@pDAOQueryDef?9?$DOget_Updatable?$CI?$CGnBo@ 5f73611c     daocore.obj
 0002:00005140       ??_C@_0CO@FAJF@pDAOQueryDef?9?$DOget_Type?$CI?$CGquerydef@ 5f736140     daocore.obj
 0002:00005170       ??_C@_0CG@DIGJ@pDAOQueryDef?9?$DOget_Name?$CI?$CGV_BSTR?$CI?$CG@ 5f736170     daocore.obj
 0002:0000519c       ??_7CDaoTableDef@@6B@      5f73619c     daocore.obj
 0002:000051c4       ??_C@_0MC@IBMF@m_pDatabase?9?$DOm_pDAODatabase?9?$DOCre@ 5f7361c4     daocore.obj
 0002:00005288       ??_C@_0CG@KMEO@pDAOTableDefs?9?$DOAppend?$CIm_pDAOTabl@ 5f736288     daocore.obj
 0002:000052b0       ??_C@_0DM@GNOH@m_pDatabase?9?$DOm_pDAODatabase?9?$DOget@ 5f7362b0     daocore.obj
 0002:000052ec       ??_C@_0EK@DHEO@pDAOTableDefs?9?$DOget_Item?$CI?5COleVar@ 5f7362ec     daocore.obj
 0002:00005338       ??_C@_0CL@GMF@m_pDAOTableDef?9?$DOget_Updatable?$CI?$CGn@ 5f736338     daocore.obj
 0002:00005364       ??_C@_0CH@LFFO@m_pDAOTableDef?9?$DOput_Name?$CIV_BSTR?$CI@ 5f736364     daocore.obj
 0002:0000538c       ??_C@_0CI@GFNK@m_pDAOTableDef?9?$DOget_Name?$CI?$CGV_BSTR@ 5f73638c     daocore.obj
 0002:000053b4       ??_C@_0DD@FHOC@m_pDAOTableDef?9?$DOput_SourceTableN@ 5f7363b4     daocore.obj
 0002:000053e8       ??_C@_0DE@CBJH@m_pDAOTableDef?9?$DOget_SourceTableN@ 5f7363e8     daocore.obj
 0002:0000541c       ??_C@_0CK@PHKK@m_pDAOTableDef?9?$DOput_Connect?$CIV_BS@ 5f73641c     daocore.obj
 0002:00005448       ??_C@_0CL@KFGO@m_pDAOTableDef?9?$DOget_Connect?$CI?$CGV_B@ 5f736448     daocore.obj
 0002:00005474       ??_C@_0CM@DGAH@m_pDAOTableDef?9?$DOput_Attributes?$CIl@ 5f736474     daocore.obj
 0002:000054a0       ??_C@_0CN@EPFM@m_pDAOTableDef?9?$DOget_Attributes?$CI?$CG@ 5f7364a0     daocore.obj
 0002:000054d0       ??_C@_0CK@CKHH@m_pDAOTableDef?9?$DOget_DateCreated?$CI@ 5f7364d0     daocore.obj
 0002:000054fc       ??_C@_0CK@ODEK@m_pDAOTableDef?9?$DOget_LastUpdated?$CI@ 5f7364fc     daocore.obj
 0002:00005528       ??_C@_0DC@EKFC@m_pDAOTableDef?9?$DOput_ValidationRu@ 5f736528     daocore.obj
 0002:0000555c       ??_C@_0DD@LHDC@m_pDAOTableDef?9?$DOget_ValidationRu@ 5f73655c     daocore.obj
 0002:00005590       ??_C@_0DC@LOBP@m_pDAOTableDef?9?$DOput_ValidationTe@ 5f736590     daocore.obj
 0002:000055c4       ??_C@_0DD@GAMG@m_pDAOTableDef?9?$DOget_ValidationTe@ 5f7365c4     daocore.obj
 0002:000055f8       ??_C@_0CP@NCFA@m_pDAOTableDef?9?$DOget_RecordCount?$CI@ 5f7365f8     daocore.obj
 0002:0000562c       ??_7CDaoFieldInfo@@6B@     5f73662c     daocore.obj
 0002:00005630       ??_C@_0CA@KBPE@m_pDAOFields?9?$DOAppend?$CIpDAOField?$CJ?$AA@ 5f736630     daocore.obj
 0002:00005650       ??_C@_0JF@NDIH@m_pDAOTableDef?9?$DOCreateField?$CI?5COl@ 5f736650     daocore.obj
 0002:000056e8       ??_C@_0CD@MPAH@m_pDAOFields?9?$DODelete?$CIV_BSTR?$CI?$CGvar@ 5f7366e8     daocore.obj
 0002:0000570c       ??_C@_0CB@GDE@m_pDAOIndexes?9?$DOAppend?$CIpDAOIndex?$CJ@ 5f73670c     daocore.obj
 0002:00005730       ??_C@_0FF@LAGC@m_pDAOTableDef?9?$DOCreateIndex?$CI?5COl@ 5f736730     daocore.obj
 0002:00005788       ??_C@_0CE@GGDB@m_pDAOIndexes?9?$DODelete?$CIV_BSTR?$CI?$CGva@ 5f736788     daocore.obj
 0002:000057ac       ??_C@_0CC@GCCM@m_pDAOFields?9?$DOget_Count?$CI?$CGnFields@ 5f7367ac     daocore.obj
 0002:000057d0       ??_C@_0DP@FPAO@m_pDAOFields?9?$DOget_Item?$CI?5COleVari@ 5f7367d0     daocore.obj
 0002:00005810       ??_C@_0EF@MHNO@m_pDAOFields?9?$DOget_Item?$CI?5COleVari@ 5f736810     daocore.obj
 0002:00005858       ??_C@_0CE@LMII@m_pDAOIndexes?9?$DOget_Count?$CI?$CGnIndex@ 5f736858     daocore.obj
 0002:0000587c       ??_C@_0EA@IAJA@m_pDAOIndexes?9?$DOget_Item?$CI?5COleVar@ 5f73687c     daocore.obj
 0002:000058bc       ??_C@_0EG@GOCN@m_pDAOIndexes?9?$DOget_Item?$CI?5COleVar@ 5f7368bc     daocore.obj
 0002:00005904       ??_C@_0BO@KAIF@m_pDAOTableDef?9?$DORefreshLink?$CI?$CJ?$AA@ 5f736904     daocore.obj
 0002:00005924       ??_C@_0CK@MDGM@m_pDAOTableDef?9?$DOget_Fields?$CI?$CGm_pD@ 5f736924     daocore.obj
 0002:00005950       ??_C@_0CM@GLNB@m_pDAOTableDef?9?$DOget_Indexes?$CI?$CGm_p@ 5f736950     daocore.obj
 0002:00005980       ??_7CDaoQueryDef@@6B@      5f736980     daocore.obj
 0002:000059bc       ??_C@_0GI@HNGJ@m_pDatabase?9?$DOm_pDAODatabase?9?$DOCre@ 5f7369bc     daocore.obj
 0002:00005a24       ??_C@_0HN@FLN@m_pDatabase?9?$DOm_pDAODatabase?9?$DOCre@ 5f736a24     daocore.obj
 0002:00005aa4       ??_C@_0CG@FLGB@pDAOQueryDefs?9?$DOAppend?$CIm_pDAOQuer@ 5f736aa4     daocore.obj
 0002:00005acc       ??_C@_0DM@IIMB@m_pDatabase?9?$DOm_pDAODatabase?9?$DOget@ 5f736acc     daocore.obj
 0002:00005b08       ??_C@_0EO@KMBN@m_pDatabase?9?$DOm_pDAODatabase?9?$DOOpe@ 5f736b08     daocore.obj
 0002:00005b58       ??_C@_0HC@LEBM@m_pDatabase?9?$DOm_pDAODatabase?9?$DOCre@ 5f736b58     daocore.obj
 0002:00005bcc       ??_C@_0BI@GPHC@m_pDAOQueryDef?9?$DOClose?$CI?$CJ?$AA@ 5f736bcc     daocore.obj
 0002:00005be4       ??_C@_0CL@HEGE@m_pDAOQueryDef?9?$DOget_Updatable?$CI?$CGn@ 5f736be4     daocore.obj
 0002:00005c10       ??_C@_0CI@DLAP@m_pDAOQueryDef?9?$DOget_Name?$CI?$CGV_BSTR@ 5f736c10     daocore.obj
 0002:00005c38       ??_C@_0CH@GAJF@m_pDAOQueryDef?9?$DOput_Name?$CIV_BSTR?$CI@ 5f736c38     daocore.obj
 0002:00005c60       ??_C@_0CH@BDHB@m_pDAOQueryDef?9?$DOget_SQL?$CI?$CGV_BSTR?$CI@ 5f736c60     daocore.obj
 0002:00005c88       ??_C@_0CG@HMBA@m_pDAOQueryDef?9?$DOput_SQL?$CIV_BSTR?$CI?$CG@ 5f736c88     daocore.obj
 0002:00005cb0       ??_C@_0CB@IFD@m_pDAOQueryDef?9?$DOget_Type?$CI?$CGnType?$CJ@ 5f736cb0     daocore.obj
 0002:00005cd4       ??_C@_0CK@ILJJ@m_pDAOQueryDef?9?$DOget_DateCreated?$CI@ 5f736cd4     daocore.obj
 0002:00005d00       ??_C@_0CK@ECKE@m_pDAOQueryDef?9?$DOget_LastUpdated?$CI@ 5f736d00     daocore.obj
 0002:00005d2c       ??_C@_0CL@NHMP@m_pDAOQueryDef?9?$DOget_Connect?$CI?$CGV_B@ 5f736d2c     daocore.obj
 0002:00005d58       ??_C@_0CK@FGEE@m_pDAOQueryDef?9?$DOput_Connect?$CIV_BS@ 5f736d58     daocore.obj
 0002:00005d84       ??_C@_0CL@ODLC@m_pDAOQueryDef?9?$DOget_ODBCTimeout?$CI@ 5f736d84     daocore.obj
 0002:00005db0       ??_C@_0CO@EFO@m_pDAOQueryDef?9?$DOput_ODBCTimeout?$CI@ 5f736db0     daocore.obj
 0002:00005de0       ??_C@_0DF@JBJO@m_pDAOQueryDef?9?$DOget_ReturnsRecor@ 5f736de0     daocore.obj
 0002:00005e18       ??_C@_0FN@IFJL@m_pDAOQueryDef?9?$DOput_ReturnsRecor@ 5f736e18     daocore.obj
 0002:00005e78       ??_C@_0DH@IBAL@m_pDAOQueryDef?9?$DOget_RecordsAffec@ 5f736e78     daocore.obj
 0002:00005eb0       ??_C@_0DF@FIBD@m_pDAOQueryDef?9?$DOExecute?$CICOleVari@ 5f736eb0     daocore.obj
 0002:00005ee8       ??_C@_0BP@JAF@pDAOParameter?9?$DOget_Value?$CI?$CGvar?$CJ?$AA@ 5f736ee8     daocore.obj
 0002:00005f08       ??_C@_0EN@DKKA@m_pDAOParameters?9?$DOget_Item?$CI?5COle@ 5f736f08     daocore.obj
 0002:00005f58       ??_C@_0EH@EAEJ@m_pDAOParameters?9?$DOget_Item?$CI?5COle@ 5f736f58     daocore.obj
 0002:00005fa0       ??_C@_0CD@KIO@pDAOParameter?9?$DOput_Value?$CIvarValu@ 5f736fa0     daocore.obj
 0002:00005fc4       ??_C@_0CK@MAHP@m_pDAOParameters?9?$DOget_Count?$CI?$CGnPa@ 5f736fc4     daocore.obj
 0002:00005ff0       ??_C@_0CK@GCIC@m_pDAOQueryDef?9?$DOget_Fields?$CI?$CGm_pD@ 5f736ff0     daocore.obj
 0002:0000601c       ??_C@_0DC@LDGL@m_pDAOQueryDef?9?$DOget_Parameters?$CI?$CG@ 5f73701c     daocore.obj
 0002:00006050       ??_C@_0DB@JEPD@pDAOParameter?9?$DOget_Value?$CI?5?$CGparam@ 5f737050     daocore.obj
 0002:00006084       ??_C@_0CN@IAMG@pDAOParameter?9?$DOget_Type?$CI?5?$CGparami@ 5f737084     daocore.obj
 0002:000060b4       ??_C@_0CH@MNLB@pDAOParameter?9?$DOget_Name?$CI?$CGV_BSTR?$CI@ 5f7370b4     daocore.obj
 0002:000060e0       ??_7CDaoRecordset@@6B@     5f7370e0     daocore.obj
 0002:00006160       ??_C@_0IB@OLCO@m_pQueryDef?9?$DOm_pDAOQueryDef?9?$DO_30@ 5f737160     daocore.obj
 0002:000061e4       ??_C@_0HN@DBDN@m_pTableDef?9?$DOm_pDAOTableDef?9?$DOOpe@ 5f7371e4     daocore.obj
 0002:00006264       ??_C@_0BJ@NGAG@m_pDAORecordset?9?$DOClose?$CI?$CJ?$AA@ 5f737264     daocore.obj
 0002:00006280       ??_C@_0CO@ENEN@m_pDAORecordset?9?$DORequery?$CI_afxOpt@ 5f737280     daocore.obj
 0002:000062b0       ??_C@_0CC@EHJO@m_pDAORecordset?9?$DORequery?$CIvarDisp@ 5f7372b0     daocore.obj
 0002:000062d4       ??_C@_0CA@OPCI@m_pDAORecordset?9?$DOget_BOF?$CI?$CGnBOF?$CJ?$AA@ 5f7372d4     daocore.obj
 0002:000062f4       ??_C@_0CA@LKNJ@m_pDAORecordset?9?$DOget_EOF?$CI?$CGnEOF?$CJ?$AA@ 5f7372f4     daocore.obj
 0002:00006314       ??_C@_0CM@BOKG@m_pDAORecordset?9?$DOget_Updatable?$CI?$CG@ 5f737314     daocore.obj
 0002:00006340       ??_C@_0DA@PJGA@m_pDAORecordset?9?$DOget_Restartable@ 5f737340     daocore.obj
 0002:00006370       ??_C@_0DC@DHEI@m_pDAORecordset?9?$DOget_Transaction@ 5f737370     daocore.obj
 0002:000063a4       ??_C@_0DC@BDFH@m_pDAORecordset?9?$DOget_Bookmarkabl@ 5f7373a4     daocore.obj
 0002:000063d8       ??_C@_0CJ@DDPM@m_pDAORecordset?9?$DOget_Name?$CI?$CGV_BST@ 5f7373d8     daocore.obj
 0002:00006404       ??_C@_0CC@NAA@m_pDAORecordset?9?$DOget_Type?$CI?$CGnType@ 5f737404     daocore.obj
 0002:00006428       ??_C@_0CK@OCGL@m_pDAORecordset?9?$DOget_EditMode?$CI?$CGn@ 5f737428     daocore.obj
 0002:00006454       ??_C@_0CL@EJNE@m_pDAORecordset?9?$DOget_DateCreated@ 5f737454     daocore.obj
 0002:00006480       ??_C@_0CL@IAOJ@m_pDAORecordset?9?$DOget_LastUpdated@ 5f737480     daocore.obj
 0002:000064ac       ??_C@_0CP@EDLK@m_pDAORecordset?9?$DOget_LastModifie@ 5f7374ac     daocore.obj
 0002:000064dc       ??_C@_0DD@KGH@m_pDAORecordset?9?$DOget_ValidationR@ 5f7374dc     daocore.obj
 0002:00006510       ??_C@_0DD@POCK@m_pDAORecordset?9?$DOget_ValidationT@ 5f737510     daocore.obj
 0002:00006544       ??_C@_0CK@NNM@m_pDAORecordset?9?$DOget_Index?$CI?$CGV_BS@ 5f737544     daocore.obj
 0002:00006570       ??_C@_0CJ@CEAC@m_pDAORecordset?9?$DOput_Index?$CIV_BST@ 5f737570     daocore.obj
 0002:0000659c       ??_C@_0DA@CFBI@m_pDAORecordset?9?$DOget_RecordCount@ 5f73759c     daocore.obj
 0002:000065cc       ??_C@_0CL@BMFG@m_pDAORecordset?9?$DOget_Bookmark?$CI?$CGv@ 5f7375cc     daocore.obj
 0002:000065f8       ??_C@_0DD@MOL@m_pDAORecordset?9?$DOput_Bookmark?$CI?$CGv@ 5f7375f8     daocore.obj
 0002:0000662c       ??_C@_0DC@GDMD@m_pDAORecordset?9?$DOget_AbsolutePos@ 5f73762c     daocore.obj
 0002:00006660       ??_C@_0DB@GLNO@m_pDAORecordset?9?$DOput_AbsolutePos@ 5f737660     daocore.obj
 0002:00006694       ??_C@_0DB@LIAP@m_pDAORecordset?9?$DOget_PercentPosi@ 5f737694     daocore.obj
 0002:000066c8       ??_C@_0DA@MHMB@m_pDAORecordset?9?$DOput_PercentPosi@ 5f7376c8     daocore.obj
 0002:000066f8       ??_C@_0CM@OLNL@m_pDAORecordset?9?$DOMove?$CIlRows?0?5COl@ 5f7376f8     daocore.obj
 0002:00006724       ??_C@_0CA@IGPM@m_pDAORecordset?9?$DO_30_MoveLast?$CI?$CJ?$AA@ 5f737724     daocore.obj
 0002:00006744       ??_C@_0BN@OKBK@m_pDAORecordset?9?$DOMoveFirst?$CI?$CJ?$AA@ 5f737744     daocore.obj
 0002:00006764       ??_C@_0CA@PGPJ@m_pDAORecordset?9?$DOMovePrevious?$CI?$CJ?$AA@ 5f737764     daocore.obj
 0002:00006784       ??_C@_0BM@KCOP@m_pDAORecordset?9?$DOMoveNext?$CI?$CJ?$AA@ 5f737784     daocore.obj
 0002:000067a0       ??_C@_0CI@BDFN@m_pDAORecordset?9?$DOFindLast?$CIV_BSTR@ 5f7377a0     daocore.obj
 0002:000067c8       ??_C@_0CJ@NOGD@m_pDAORecordset?9?$DOFindFirst?$CIV_BST@ 5f7377c8     daocore.obj
 0002:000067f4       ??_C@_0CM@CFIG@m_pDAORecordset?9?$DOFindPrevious?$CIV_@ 5f7377f4     daocore.obj
 0002:00006820       ??_C@_0CI@IEGA@m_pDAORecordset?9?$DOFindNext?$CIV_BSTR@ 5f737820     daocore.obj
 0002:00006848       ??_C@_0BKF@GBHJ@m_pDAORecordset?9?$DOSeek?$CIV_BSTR?$CI?$CGva@ 5f737848     daocore.obj
 0002:000069f0       ??_C@_0PE@MNIL@m_pDAORecordset?9?$DOSeek?$CIV_BSTR?$CI?$CGva@ 5f7379f0     daocore.obj
 0002:00006ae4       ??_C@_0CE@GKGD@m_pDAORecordset?9?$DO_30_CancelUpdat@ 5f737ae4     daocore.obj
 0002:00006b08       ??_C@_0FG@JILN@m_pDAORecordset?9?$DOput_LockEdits?$CI?5@ 5f737b08     daocore.obj
 0002:00006b60       ??_C@_0CM@FJGM@m_pDAORecordset?9?$DOget_LockEdits?$CI?$CG@ 5f737b60     daocore.obj
 0002:00006b8c       ??_C@_0DF@NEPL@m_pDAORecordset?9?$DOput_CacheStart?$CI@ 5f737b8c     daocore.obj
 0002:00006bc4       ??_C@_0CN@BBCI@m_pDAORecordset?9?$DOget_CacheStart?$CI@ 5f737bc4     daocore.obj
 0002:00006bf4       ??_C@_0CG@GPJG@m_pDAORecordset?9?$DOput_CacheSize?$CIl@ 5f737bf4     daocore.obj
 0002:00006c1c       ??_C@_0CH@FFJB@m_pDAORecordset?9?$DOget_CacheSize?$CI?$CG@ 5f737c1c     daocore.obj
 0002:00006c44       ??_C@_0JP@FOGE@m_pDAORecordset?9?$DOFillCache?$CI?5pSiz@ 5f737c44     daocore.obj
 0002:00006ce4       ??_C@_0BK@MEND@m_pDAORecordset?9?$DOAddNew?$CI?$CJ?$AA@ 5f737ce4     daocore.obj
 0002:00006d00       ??_C@_0BI@CNBL@m_pDAORecordset?9?$DOEdit?$CI?$CJ?$AA@ 5f737d00     daocore.obj
 0002:00006d18       ??_C@_0BO@JCIA@m_pDAORecordset?9?$DO_30_Update?$CI?$CJ?$AA@ 5f737d18     daocore.obj
 0002:00006d38       ??_C@_0BK@DPAI@m_pDAORecordset?9?$DODelete?$CI?$CJ?$AA@ 5f737d38     daocore.obj
 0002:00006d54       ??_C@_0EK@CMJC@m_pDAORecordset?9?$DOget_Collect?$CI?5CO@ 5f737d54     daocore.obj
 0002:00006da0       ??_C@_0EE@NBLG@m_pDAORecordset?9?$DOget_Collect?$CI?5CO@ 5f737da0     daocore.obj
 0002:00006de4       ??_C@_0EJ@FHEM@m_pDAORecordset?9?$DOput_Collect?$CI?5CO@ 5f737de4     daocore.obj
 0002:00006e30       ??_C@_0ED@ENAG@m_pDAORecordset?9?$DOput_Collect?$CI?5CO@ 5f737e30     daocore.obj
 0002:00006e74       ??_C@_0CL@KAMP@m_pDAORecordset?9?$DOget_Fields?$CI?$CGm_p@ 5f737e74     daocore.obj
 0002:00006ea0       ??_C@_0DJ@FHAD@m_pTableDef?9?$DOm_pDAOTableDef?9?$DOget@ 5f737ea0     daocore.obj
 0002:00006edc       ??_C@_13FDB@?$AA?$DL?$AA?$AA@ 5f737edc     daocore.obj
 0002:00006ee0       ??_C@_0FI@LEEG@m_pDAORecordset?9?$DOQueryInterface?$CI@ 5f737ee0     daocore.obj
 0002:00006f38       ??_C@_0CI@ILFL@m_pDAORecordset?9?$DOget_NoMatch?$CI?$CGnN@ 5f737f38     daocore.obj
 0002:00006f60       ??_C@_0CA@MLFB@?6m_bCheckCacheForDirtyFields?5?$DN?5?$AA@ 5f737f60     daocore.obj
 0002:00006f80       ??_C@_0BF@FEP@?6m_strRequerySort?5?$DN?5?$AA@ 5f737f80     daocore.obj
 0002:00006f98       ??_C@_0BH@NPKA@?6m_strRequeryFilter?5?$DN?5?$AA@ 5f737f98     daocore.obj
 0002:00006fb0       ??_C@_0BE@OAFC@?6m_strRequerySQL?5?$DN?5?$AA@ 5f737fb0     daocore.obj
 0002:00006fc4       ??_C@_0O@JOGM@?6m_strSort?5?$DN?5?$AA@ 5f737fc4     daocore.obj
 0002:00006fd4       ??_C@_0BA@ICBM@?6m_strFilter?5?$DN?5?$AA@ 5f737fd4     daocore.obj
 0002:00006fe4       ??_C@_0P@CAKJ@?6m_nOptions?5?$DN?5?$AA@ 5f737fe4     daocore.obj
 0002:00006ff4       ??_C@_0BD@FPPO@?6m_nDefaultType?5?$DN?5?$AA@ 5f737ff4     daocore.obj
 0002:00007008       ??_C@_0BA@DPMC@?6m_nOpenType?5?$DN?5?$AA@ 5f738008     daocore.obj
 0002:00007018       ??_C@_0M@NMDE@?6m_bOpen?5?$DN?5?$AA@ 5f738018     daocore.obj
 0002:00007024       ??_C@_0CN@LODG@pDAOField?9?$DOget_ValidationText?$CI?$CGV@ 5f738024     daocore.obj
 0002:00007054       ??_C@_0CN@EKHL@pDAOField?9?$DOget_ValidationRule?$CI?$CGV@ 5f738054     daocore.obj
 0002:00007084       ??_C@_0CK@NMNF@pDAOField?9?$DOget_SourceTable?$CI?$CGV_BS@ 5f738084     daocore.obj
 0002:000070b0       ??_C@_0CK@NMGJ@pDAOField?9?$DOget_SourceField?$CI?$CGV_BS@ 5f7380b0     daocore.obj
 0002:000070dc       ??_C@_0DN@PLFL@pDAOField?9?$DOget_CollatingOrder?$CI?5?$CG@ 5f7380dc     daocore.obj
 0002:0000711c       ??_C@_0CH@BDEE@pDAOField?9?$DOget_AllowZeroLength?$CI?$CG@ 5f73811c     daocore.obj
 0002:00007144       ??_C@_0CA@GJNH@pDAOField?9?$DOget_Required?$CI?$CGnBool?$CJ?$AA@ 5f738144     daocore.obj
 0002:00007164       ??_C@_0DP@GBEA@pDAOField?9?$DOget_OrdinalPosition?$CI?5@ 5f738164     daocore.obj
 0002:000071a4       ??_C@_0DE@DLJC@pDAOField?9?$DOget_Attributes?$CI?$CGfield@ 5f7381a4     daocore.obj
 0002:000071d8       ??_C@_0CI@DFJD@pDAOField?9?$DOget_Size?$CI?$CGfieldinfo?4m@ 5f7381d8     daocore.obj
 0002:00007200       ??_C@_0CI@LPDA@pDAOField?9?$DOget_Type?$CI?$CGfieldinfo?4m@ 5f738200     daocore.obj
 0002:00007228       ??_C@_0CM@OIHD@pDAOField?9?$DOput_ValidationText?$CIV_@ 5f738228     daocore.obj
 0002:00007254       ??_C@_0CM@KFNC@pDAOField?9?$DOput_ValidationRule?$CIV_@ 5f738254     daocore.obj
 0002:00007280       ??_C@_0CN@ECE@pDAOField?9?$DOput_AllowZeroLength?$CIA@ 5f738280     daocore.obj
 0002:000072b0       ??_C@_0CG@NDE@pDAOField?9?$DOput_Required?$CIAFX_DAO_@ 5f7382b0     daocore.obj
 0002:000072d8       ??_C@_0DO@LDPI@pDAOField?9?$DOput_OrdinalPosition?$CI?5@ 5f7382d8     daocore.obj
 0002:00007318       ??_C@_0DD@KMNM@pDAOField?9?$DOput_Attributes?$CIfieldi@ 5f738318     daocore.obj
 0002:0000734c       ??_C@_0CF@IAPF@?$CIpDAOField?9?$DO?$CKpMethod?$CJ?$CI?$CGV_BSTR?$CI?$CGv@ 5f73834c     daocore.obj
 0002:00007374       ??_C@_0CC@GCFC@pDAOField?9?$DOget_DefaultValue?$CI?$CGvar@ 5f738374     daocore.obj
 0002:00007398       ??_C@_0CE@DCCL@?$CIpDAOField?9?$DO?$CKpMethod?$CJ?$CIV_BSTR?$CI?$CGva@ 5f738398     daocore.obj
 0002:000073bc       ??_C@_0CB@DPPD@pDAOField?9?$DOput_DefaultValue?$CIvar?$CJ@ 5f7383bc     daocore.obj
 0002:000073e0       ??_C@_0DL@MFON@pDAOIndex?9?$DOget_DistinctCount?$CI?5?$CGi@ 5f7383e0     daocore.obj
 0002:0000741c       ??_C@_0BP@GBPC@pDAOIndex?9?$DOget_Foreign?$CI?$CGnBool?$CJ?$AA@ 5f73841c     daocore.obj
 0002:0000743c       ??_C@_0CA@LEOO@pDAOIndex?9?$DOget_Required?$CI?$CGnBool?$CJ?$AA@ 5f73843c     daocore.obj
 0002:0000745c       ??_C@_0CD@PNHL@pDAOIndex?9?$DOget_IgnoreNulls?$CI?$CGnBoo@ 5f73845c     daocore.obj
 0002:00007480       ??_C@_0CB@MCH@pDAOIndex?9?$DOget_Clustered?$CI?$CGnBool?$CJ@ 5f738480     daocore.obj
 0002:000074a4       ??_C@_0BO@HDBC@pDAOIndex?9?$DOget_Unique?$CI?$CGnBool?$CJ?$AA@ 5f7384a4     daocore.obj
 0002:000074c4       ??_C@_0BP@JAAH@pDAOIndex?9?$DOget_Primary?$CI?$CGnBool?$CJ?$AA@ 5f7384c4     daocore.obj
 0002:000074e4       ??_C@_0CD@MEGG@pDAOIndex?9?$DOget_Name?$CI?$CGV_BSTR?$CI?$CGvar@ 5f7384e4     daocore.obj
 0002:00007508       ??_C@_0CG@NMKH@pDAOIndex?9?$DOput_Required?$CIAFX_DAO_@ 5f738508     daocore.obj
 0002:00007530       ??_C@_0CJ@GEID@pDAOIndex?9?$DOput_IgnoreNulls?$CIAFX_D@ 5f738530     daocore.obj
 0002:0000755c       ??_C@_0CH@PIFK@pDAOIndex?9?$DOput_Clustered?$CIAFX_DAO@ 5f73855c     daocore.obj
 0002:00007584       ??_C@_0CE@PPGA@pDAOIndex?9?$DOput_Unique?$CIAFX_DAO_TR@ 5f738584     daocore.obj
 0002:000075a8       ??_C@_0CF@ONFI@pDAOIndex?9?$DOput_Primary?$CIAFX_DAO_T@ 5f7385a8     daocore.obj
 0002:000075d0       ??_C@_0EJ@HLNA@var?4pdispVal?9?$DOQueryInterface?$CI?5gu@ 5f7385d0     daocore.obj
 0002:0000761c       ??_C@_0BM@FLME@pDAOIndex?9?$DOget_Fields?$CI?$CGvar?$CJ?$AA@ 5f73861c     daocore.obj
 0002:00007638       ??_C@_0CI@GIHF@pDAOField?9?$DOget_Attributes?$CI?$CGlAttr@ 5f738638     daocore.obj
 0002:00007660       ??_C@_0DN@MHHF@var?4pdispVal?9?$DOQueryInterface?$CI?5gu@ 5f738660     daocore.obj
 0002:000076a0       ??_C@_0DF@CLB@pDAOIndexFields?9?$DOget_Item?$CICOleVa@ 5f7386a0     daocore.obj
 0002:000076d8       ??_C@_0CE@GNBF@pDAOIndexFields?9?$DOget_Count?$CI?$CGnCou@ 5f7386d8     daocore.obj
 0002:00007700       ??_7CDaoIndexFieldInfo@@6B@ 5f738700     daocore.obj
 0002:00007704       ??_C@_0CH@BPFN@pDAOField?9?$DOput_Attributes?$CIlAttri@ 5f738704     daocore.obj
 0002:0000772c       ??_C@_0JA@MEIF@pDAOIndex?9?$DOCreateField?$CI?5COleVari@ 5f73872c     daocore.obj
 0002:000077bc       ??_C@_1CO@HEDE@?$AAI?$AAC?$AAD?$AAA?$AAO?$AAR?$AAe?$AAc?$AAo?$AAr?$AAd?$AAs?$AAe?$AAt?$AA?4?$AAG?$AAe?$AAt?$AAR?$AAo@ 5f7387bc     daocore.obj
 0002:000077ec       ??_C@_0GH@DHEN@pCF2?9?$DOCreateInstanceLic?$CI?5NULL?0?5N@ 5f7387ec     daocore.obj
 0002:00007854       ??_C@_0GA@FMGC@?3?3CoGetClassObject?$CIclsidEngine?0?5@ 5f738854     daocore.obj
 0002:000078b4       ??_C@_1EK@JJKF@?$AAm?$AAj?$AAg?$AAc?$AAq?$AAc?$AAe?$AAj?$AAf?$AAc?$AAh?$AAc?$AAi?$AAj?$AAe?$AAc?$AAp?$AAd?$AAh?$AAc@ 5f7388b4     daocore.obj
 0002:00007900       ??_C@_1EK@JBEF@?$AAm?$AAb?$AAm?$AAa?$AAb?$AAp?$AAt?$AAe?$AAb?$AAk?$AAj?$AAc?$AAd?$AAl?$AAg?$AAt?$AAj?$AAm?$AAs?$AAk@ 5f738900     daocore.obj
 0002:0000794c       ??_C@_0BF@DC@?3?3CoInitialize?$CINULL?$CJ?$AA@ 5f73894c     daocore.obj
 0002:00007968       ?_afxDoublePseudoNull@@3NB 5f738968     daodfx.obj
 0002:00007970       ?_afxFloatPseudoNull@@3MB  5f738970     daodfx.obj
 0002:00007974       ??_C@_09CGOK@?5DateTime?$AA@ 5f738974     daodfx.obj
 0002:00007980       ??_C@_0M@BGKI@?5IEEEDouble?$AA@ 5f738980     daodfx.obj
 0002:0000798c       ??_C@_0M@GOBO@?5IEEESingle?$AA@ 5f73898c     daodfx.obj
 0002:00007998       ??_C@_09GDCP@?5Currency?$AA@ 5f738998     daodfx.obj
 0002:000079a4       ??_C@_05BJMF@?5Long?$AA@   5f7389a4     daodfx.obj
 0002:000079ac       ??_C@_06KOJB@?5Short?$AA@  5f7389ac     daodfx.obj
 0002:000079b4       ??_C@_05IGCC@?5Byte?$AA@   5f7389b4     daodfx.obj
 0002:000079bc       ??_C@_04KDMA@?5Bit?$AA@    5f7389bc     daodfx.obj
 0002:000079c4       ??_C@_0M@MOAI@?5LongBinary?$AA@ 5f7389c4     daodfx.obj
 0002:000079d0       ??_C@_05BJHD@?5Text?$AA@   5f7389d0     daodfx.obj
 0002:000079d8       ??_C@_01KMAE@?0?$AA@       5f7389d8     daodfx.obj
 0002:000079e0       ?messageMap@CDaoRecordView@@1UAFX_MSGMAP@@B 5f7389e0     daoview.obj
 0002:000079e8       ?_messageEntries@CDaoRecordView@@0QBUAFX_MSGMAP_ENTRY@@B 5f7389e8     daoview.obj
 0002:00007ac0       ?classCDaoRecordView@CDaoRecordView@@2UCRuntimeClass@@B 5f738ac0     daoview.obj
 0002:00007ad8       ??_C@_0P@KPJP@CDaoRecordView?$AA@ 5f738ad8     daoview.obj
 0002:00007aec       ??_7CDaoRecordView@@6B@    5f738aec     daoview.obj
 0002:00007c04       ??_C@_1GG@NJGF@?$AAW?$AAa?$AAr?$AAn?$AAi?$AAn?$AAg?$AA?3?$AA?5?$AAc?$AAa?$AAn?$AA?8?$AAt?$AA?5?$AAs?$AAe?$AAt?$AA?5?$AAc@ 5f738c04     daoview.obj
 0002:00007c6c       ??_C@_1GG@MNDJ@?$AAW?$AAa?$AAr?$AAn?$AAi?$AAn?$AAg?$AA?3?$AA?5?$AAc?$AAa?$AAn?$AA?8?$AAt?$AA?5?$AAs?$AAe?$AAt?$AA?5?$AAf@ 5f738c6c     daoview.obj
 0002:00007cd4       ??_C@_0BE@CLIM@m_varBookmarkLast?5?$DN?$AA@ 5f738cd4     daoview.obj
 0002:00007ce8       ??_C@_0BF@EDLD@m_varBookmarkFirst?5?$DN?$AA@ 5f738ce8     daoview.obj
 0002:00007d00       ??_C@_0BH@FBNH@m_varBookmarkCurrent?5?$DN?$AA@ 5f738d00     daoview.obj
 0002:00007d18       ??_C@_0M@LNMN@m_nStatus?5?$DN?$AA@ 5f738d18     daoview.obj
 0002:00007d28       ?classCOleDBRecordView@COleDBRecordView@@2UCRuntimeClass@@B 5f738d28     viewoled.obj
 0002:00007d40       ??_C@_0BB@HKOA@COleDBRecordView?$AA@ 5f738d40     viewoled.obj
 0002:00007d58       ?messageMap@COleDBRecordView@@1UAFX_MSGMAP@@B 5f738d58     viewoled.obj
 0002:00007d60       ?_messageEntries@COleDBRecordView@@0QBUAFX_MSGMAP_ENTRY@@B 5f738d60     viewoled.obj
 0002:00007e38       ??_C@_1EC@DLJM@?$AAG?$AAe?$AAt?$AAD?$AAa?$AAt?$AAa?$AA?5?$AAf?$AAa?$AAi?$AAl?$AAe?$AAd?$AA?5?$AA?9?$AA?5?$AAH?$AAR?$AAE@ 5f738e38     viewoled.obj
 0002:00007e7c       ??_C@_0BB@OJDA@m_pAccessor?5?$CB?$DN?50?$AA@ 5f738e7c     viewoled.obj
 0002:00007e90       ??_C@_0CI@GKMH@E?3?28168?2vc98?2mfc?2atl?2include?2atl@ 5f738e90     viewoled.obj
 0002:00007eb8       ??_C@_0BA@EFBK@m_spRowset?5?$CB?$DN?50?$AA@ 5f738eb8     viewoled.obj
 0002:00007ec8       ??_C@_1M@JIAP@?$AAA?$AAT?$AAL?$AA?3?$AA?5?$AA?$AA@ 5f738ec8     viewoled.obj
 0002:00007ed4       ??_C@_09PLJB@atlbase?4h?$AA@ 5f738ed4     viewoled.obj
 0002:00007ee0       ??_C@_0BI@CIAH@nBuf?5?$DM?5sizeof?$CIszBuffer?$CJ?$AA@ 5f738ee0     viewoled.obj
 0002:00007ef8       ??_C@_1FO@OKAP@?$AAG?$AAe?$AAt?$AAD?$AAa?$AAt?$AAa?$AA?5?$AAf?$AAr?$AAo?$AAm?$AA?5?$AAM?$AAo?$AAv?$AAe?$AAL?$AAa?$AAs@ 5f738ef8     viewoled.obj
 0002:00007f58       ??_C@_0BF@GPJA@m_pAccessorInfo?5?$CB?$DN?50?$AA@ 5f738f58     viewoled.obj
 0002:00007f70       ??_C@_0BJ@NICA@nAccessor?5?$DM?5m_nAccessors?$AA@ 5f738f70     viewoled.obj
 0002:00007f8c       ??_C@_0M@DLL@m_hRow?5?$CB?$DN?50?$AA@ 5f738f8c     viewoled.obj
 0002:00007f98       ??_C@_0BH@DLBO@nAccessor?$DMm_nAccessors?$AA@ 5f738f98     viewoled.obj
 0002:00007fb0       ??_C@_04GBK@p?$CB?$DN0?$AA@ 5f738fb0     viewoled.obj
 0002:00007fe8       ??_7type_info@@6B@         5f738fe8     msvcrtd:ti_inst.obj
 0002:00007fec       ??_C@_08JKC@crtdll?4c?$AA@ 5f738fec     msvcrtd:crtdll.obj
 0002:00007ff8       _IID_IClassFactory2        5f738ff8     uuid:ocidl_i_guid4.obj
 0002:00008008       _LIBID_CJETSQLHELP         5f739008     daouuid:daouuid.obj
 0002:00008018       _LIBID_CDAO                5f739018     daouuid:daouuid.obj
 0002:00008028       _LIBID_CDAO25              5f739028     daouuid:daouuid.obj
 0002:00008038       _BETA_LIBID_CDAO           5f739038     daouuid:daouuid.obj
 0002:00008048       _BETA_LIBID_CDAO25         5f739048     daouuid:daouuid.obj
 0002:00008058       _IID_IDAOStdObject         5f739058     daouuid:daouuid.obj
 0002:00008068       _IID_IDAOStdCollection     5f739068     daouuid:daouuid.obj
 0002:00008078       _CLSID_CDAODBEngine        5f739078     daouuid:daouuid.obj
 0002:00008088       _CLSID_CDAOPrivDBEngine    5f739088     daouuid:daouuid.obj
 0002:00008098       _CLSID_CDAOConnection      5f739098     daouuid:daouuid.obj
 0002:000080a8       _CLSID_CDAOTableDef        5f7390a8     daouuid:daouuid.obj
 0002:000080b8       _CLSID_CDAOField           5f7390b8     daouuid:daouuid.obj
 0002:000080c8       _CLSID_CDAOIndex           5f7390c8     daouuid:daouuid.obj
 0002:000080d8       _CLSID_CDAOGroup           5f7390d8     daouuid:daouuid.obj
 0002:000080e8       _CLSID_CDAOUser            5f7390e8     daouuid:daouuid.obj
 0002:000080f8       _CLSID_CDAOQueryDef        5f7390f8     daouuid:daouuid.obj
 0002:00008108       _CLSID_CDAORelation        5f739108     daouuid:daouuid.obj
 0002:00008118       _CLSID35_CDAODBEngine      5f739118     daouuid:daouuid.obj
 0002:00008128       _CLSID35_CDAOPrivDBEngine  5f739128     daouuid:daouuid.obj
 0002:00008138       _CLSID35_CDAOConnection    5f739138     daouuid:daouuid.obj
 0002:00008148       _CLSID35_CDAOTableDef      5f739148     daouuid:daouuid.obj
 0002:00008158       _CLSID35_CDAOField         5f739158     daouuid:daouuid.obj
 0002:00008168       _CLSID35_CDAOIndex         5f739168     daouuid:daouuid.obj
 0002:00008178       _CLSID35_CDAOGroup         5f739178     daouuid:daouuid.obj
 0002:00008188       _CLSID35_CDAOUser          5f739188     daouuid:daouuid.obj
 0002:00008198       _CLSID35_CDAOQueryDef      5f739198     daouuid:daouuid.obj
 0002:000081a8       _CLSID35_CDAORelation      5f7391a8     daouuid:daouuid.obj
 0002:000081b8       _IID_IDAODBEngine          5f7391b8     daouuid:daouuid.obj
 0002:000081c8       _IID_IDAODBEngineW         5f7391c8     daouuid:daouuid.obj
 0002:000081d8       _IID_IDAOError             5f7391d8     daouuid:daouuid.obj
 0002:000081e8       _IID_IDAOErrorW            5f7391e8     daouuid:daouuid.obj
 0002:000081f8       _IID_IDAOErrors            5f7391f8     daouuid:daouuid.obj
 0002:00008208       _IID_IDAOErrorsW           5f739208     daouuid:daouuid.obj
 0002:00008218       _IID_IDAOProperty          5f739218     daouuid:daouuid.obj
 0002:00008228       _IID_IDAOPropertyW         5f739228     daouuid:daouuid.obj
 0002:00008238       _IID_IDAOProperties        5f739238     daouuid:daouuid.obj
 0002:00008248       _IID_IDAOPropertiesW       5f739248     daouuid:daouuid.obj
 0002:00008258       _IID_IDAORecordset         5f739258     daouuid:daouuid.obj
 0002:00008268       _IID_IDAORecordsetW        5f739268     daouuid:daouuid.obj
 0002:00008278       _IID_IDAORecordsets        5f739278     daouuid:daouuid.obj
 0002:00008288       _IID_IDAORecordsetsW       5f739288     daouuid:daouuid.obj
 0002:00008298       _IID_ICDAORecordset        5f739298     daouuid:daouuid.obj
 0002:000082a8       _IID_IDAOWorkspace         5f7392a8     daouuid:daouuid.obj
 0002:000082b8       _IID_IDAOWorkspaceW        5f7392b8     daouuid:daouuid.obj
 0002:000082c8       _IID_IDAOWorkspaces        5f7392c8     daouuid:daouuid.obj
 0002:000082d8       _IID_IDAOWorkspacesW       5f7392d8     daouuid:daouuid.obj
 0002:000082e8       _IID_IDAOConnection        5f7392e8     daouuid:daouuid.obj
 0002:000082f8       _IID_IDAOConnectionW       5f7392f8     daouuid:daouuid.obj
 0002:00008308       _IID_IDAOConnections       5f739308     daouuid:daouuid.obj
 0002:00008318       _IID_IDAOConnectionsW      5f739318     daouuid:daouuid.obj
 0002:00008328       _IID_IDAOTableDef          5f739328     daouuid:daouuid.obj
 0002:00008338       _IID_IDAOTableDefW         5f739338     daouuid:daouuid.obj
 0002:00008348       _IID_IDAOTableDefs         5f739348     daouuid:daouuid.obj
 0002:00008358       _IID_IDAOTableDefsW        5f739358     daouuid:daouuid.obj
 0002:00008368       _IID_IDAOField             5f739368     daouuid:daouuid.obj
 0002:00008378       _IID_IDAOFieldW            5f739378     daouuid:daouuid.obj
 0002:00008388       _IID_IDAOFields            5f739388     daouuid:daouuid.obj
 0002:00008398       _IID_IDAOFieldsW           5f739398     daouuid:daouuid.obj
 0002:000083a8       _IID_IDAOIndex             5f7393a8     daouuid:daouuid.obj
 0002:000083b8       _IID_IDAOIndexW            5f7393b8     daouuid:daouuid.obj
 0002:000083c8       _IID_IDAOIndexes           5f7393c8     daouuid:daouuid.obj
 0002:000083d8       _IID_IDAOIndexesW          5f7393d8     daouuid:daouuid.obj
 0002:000083e8       _IID_IDAOIndexFields       5f7393e8     daouuid:daouuid.obj
 0002:000083f8       _IID_IDAOIndexFieldsW      5f7393f8     daouuid:daouuid.obj
 0002:00008408       _IID_IDAOGroup             5f739408     daouuid:daouuid.obj
 0002:00008418       _IID_IDAOGroupW            5f739418     daouuid:daouuid.obj
 0002:00008428       _IID_IDAOGroups            5f739428     daouuid:daouuid.obj
 0002:00008438       _IID_IDAOGroupsW           5f739438     daouuid:daouuid.obj
 0002:00008448       _IID_IDAOUser              5f739448     daouuid:daouuid.obj
 0002:00008458       _IID_IDAOUserW             5f739458     daouuid:daouuid.obj
 0002:00008468       _IID_IDAOUsers             5f739468     daouuid:daouuid.obj
 0002:00008478       _IID_IDAOUsersW            5f739478     daouuid:daouuid.obj
 0002:00008488       _IID_IDAODatabase          5f739488     daouuid:daouuid.obj
 0002:00008498       _IID_IDAODatabaseW         5f739498     daouuid:daouuid.obj
 0002:000084a8       _IID_IDAODatabases         5f7394a8     daouuid:daouuid.obj
 0002:000084b8       _IID_IDAODatabasesW        5f7394b8     daouuid:daouuid.obj
 0002:000084c8       _IID_IDAOQueryDef          5f7394c8     daouuid:daouuid.obj
 0002:000084d8       _IID_IDAOQueryDefW         5f7394d8     daouuid:daouuid.obj
 0002:000084e8       _IID_IDAOQueryDefs         5f7394e8     daouuid:daouuid.obj
 0002:000084f8       _IID_IDAOQueryDefsW        5f7394f8     daouuid:daouuid.obj
 0002:00008508       _IID_IDAOParameter         5f739508     daouuid:daouuid.obj
 0002:00008518       _IID_IDAOParameterW        5f739518     daouuid:daouuid.obj
 0002:00008528       _IID_IDAOParameters        5f739528     daouuid:daouuid.obj
 0002:00008538       _IID_IDAOParametersW       5f739538     daouuid:daouuid.obj
 0002:00008548       _IID_IDAORelation          5f739548     daouuid:daouuid.obj
 0002:00008558       _IID_IDAORelationW         5f739558     daouuid:daouuid.obj
 0002:00008568       _IID_IDAORelations         5f739568     daouuid:daouuid.obj
 0002:00008578       _IID_IDAORelationsW        5f739578     daouuid:daouuid.obj
 0002:00008588       _IID_IDAOContainer         5f739588     daouuid:daouuid.obj
 0002:00008598       _IID_IDAOContainerW        5f739598     daouuid:daouuid.obj
 0002:000085a8       _IID_IDAOContainers        5f7395a8     daouuid:daouuid.obj
 0002:000085b8       _IID_IDAOContainersW       5f7395b8     daouuid:daouuid.obj
 0002:000085c8       _IID_IDAODocument          5f7395c8     daouuid:daouuid.obj
 0002:000085d8       _IID_IDAODocumentW         5f7395d8     daouuid:daouuid.obj
 0002:000085e8       _IID_IDAODocuments         5f7395e8     daouuid:daouuid.obj
 0002:000085f8       _IID_IDAODocumentsW        5f7395f8     daouuid:daouuid.obj
 0002:00008608       _IID_IDAOCollection        5f739608     daouuid:daouuid.obj
 0002:00008618       _IID_IDAODynaCollection    5f739618     daouuid:daouuid.obj
 0002:00008628       _IID_IDAOQueryCP           5f739628     daouuid:daouuid.obj
 0002:00008638       _IID_IDAOQueryAS           5f739638     daouuid:daouuid.obj
 0002:00008648       _IID_ICDAOJETDBEngine      5f739648     daouuid:daouuid.obj
 0002:00008658       _IID_ICDAOJETError         5f739658     daouuid:daouuid.obj
 0002:00008668       _IID_ICDAOJETRecordset     5f739668     daouuid:daouuid.obj
 0002:00008678       _IID_ICDAOJETWorkspace     5f739678     daouuid:daouuid.obj
 0002:00008688       _IID_ICDAOJETField         5f739688     daouuid:daouuid.obj
 0002:00008698       _IID_ICDAOJETDatabase      5f739698     daouuid:daouuid.obj
 0002:000086a8       _IID_IDAOSnapshot          5f7396a8     daouuid:daouuid.obj
 0002:000086b8       _IID_IDAOTable             5f7396b8     daouuid:daouuid.obj
 0002:000086c8       _IID_IDAODynaset           5f7396c8     daouuid:daouuid.obj
 0002:000086d8       _IID_IDisconnect           5f7396d8     daouuid:daouuid.obj
 0002:000086e8       _IID_IDisconnectAll        5f7396e8     daouuid:daouuid.obj
 0002:000086f8       _IID_IDSCAdviseSink        5f7396f8     daouuid:daouuid.obj
 0002:00008708       _IID_IDSCConnectionPoint   5f739708     daouuid:daouuid.obj
 0002:00008718       _IID_IDBAdviseSink         5f739718     daouuid:daouuid.obj
 0002:00008728       _IID_IDBConnectionPoint    5f739728     daouuid:daouuid.obj
 0002:00008738       _LIBID30_CDAO              5f739738     daouuid:daouuid.obj
 0002:00008748       _LIBID30_CDAO25            5f739748     daouuid:daouuid.obj
 0002:00008758       _IID30_IDAOStdObject       5f739758     daouuid:daouuid.obj
 0002:00008768       _IID30_IDAOStdCollection   5f739768     daouuid:daouuid.obj
 0002:00008778       _CLSID30_CDAODBEngine      5f739778     daouuid:daouuid.obj
 0002:00008788       _IID30_IDAODBEngine        5f739788     daouuid:daouuid.obj
 0002:00008798       _IID30_IDAODBEngineW       5f739798     daouuid:daouuid.obj
 0002:000087a8       _IID30_ICDAOJETDBEngine    5f7397a8     daouuid:daouuid.obj
 0002:000087b8       _CLSID30_CDAOPrivDBEngine  5f7397b8     daouuid:daouuid.obj
 0002:000087c8       _IID30_IDAOError           5f7397c8     daouuid:daouuid.obj
 0002:000087d8       _IID30_IDAOErrorW          5f7397d8     daouuid:daouuid.obj
 0002:000087e8       _IID30_IDAOErrors          5f7397e8     daouuid:daouuid.obj
 0002:000087f8       _IID30_IDAOErrorsW         5f7397f8     daouuid:daouuid.obj
 0002:00008808       _IID30_ICDAOJETError       5f739808     daouuid:daouuid.obj
 0002:00008818       _IID30_IDAOProperty        5f739818     daouuid:daouuid.obj
 0002:00008828       _IID30_IDAOPropertyW       5f739828     daouuid:daouuid.obj
 0002:00008838       _IID30_IDAOProperties      5f739838     daouuid:daouuid.obj
 0002:00008848       _IID30_IDAOPropertiesW     5f739848     daouuid:daouuid.obj
 0002:00008858       _IID30_IDAORecordset       5f739858     daouuid:daouuid.obj
 0002:00008868       _IID30_IDAORecordsetW      5f739868     daouuid:daouuid.obj
 0002:00008878       _IID30_IDAORecordsets      5f739878     daouuid:daouuid.obj
 0002:00008888       _IID30_IDAORecordsetsW     5f739888     daouuid:daouuid.obj
 0002:00008898       _IID30_ICDAORecordset      5f739898     daouuid:daouuid.obj
 0002:000088a8       _IID30_ICDAOJETRecordset   5f7398a8     daouuid:daouuid.obj
 0002:000088b8       _IID30_IDAOSnapshot        5f7398b8     daouuid:daouuid.obj
 0002:000088c8       _IID30_IDAOTable           5f7398c8     daouuid:daouuid.obj
 0002:000088d8       _IID30_IDAODynaset         5f7398d8     daouuid:daouuid.obj
 0002:000088e8       _IID30_IDAOWorkspace       5f7398e8     daouuid:daouuid.obj
 0002:000088f8       _IID30_IDAOWorkspaceW      5f7398f8     daouuid:daouuid.obj
 0002:00008908       _IID30_IDAOWorkspaces      5f739908     daouuid:daouuid.obj
 0002:00008918       _IID30_IDAOWorkspacesW     5f739918     daouuid:daouuid.obj
 0002:00008928       _IID30_ICDAOJETWorkspace   5f739928     daouuid:daouuid.obj
 0002:00008938       _CLSID30_CDAOConnection    5f739938     daouuid:daouuid.obj
 0002:00008948       _IID30_IDAOConnection      5f739948     daouuid:daouuid.obj
 0002:00008958       _IID30_IDAOConnectionW     5f739958     daouuid:daouuid.obj
 0002:00008968       _IID30_IDAOConnections     5f739968     daouuid:daouuid.obj
 0002:00008978       _IID30_IDAOConnectionsW    5f739978     daouuid:daouuid.obj
 0002:00008988       _CLSID30_CDAOTableDef      5f739988     daouuid:daouuid.obj
 0002:00008998       _IID30_IDAOTableDef        5f739998     daouuid:daouuid.obj
 0002:000089a8       _IID30_IDAOTableDefW       5f7399a8     daouuid:daouuid.obj
 0002:000089b8       _IID30_IDAOTableDefs       5f7399b8     daouuid:daouuid.obj
 0002:000089c8       _IID30_IDAOTableDefsW      5f7399c8     daouuid:daouuid.obj
 0002:000089d8       _CLSID30_CDAOField         5f7399d8     daouuid:daouuid.obj
 0002:000089e8       _IID30_IDAOField           5f7399e8     daouuid:daouuid.obj
 0002:000089f8       _IID30_IDAOFieldW          5f7399f8     daouuid:daouuid.obj
 0002:00008a08       _IID30_IDAOFields          5f739a08     daouuid:daouuid.obj
 0002:00008a18       _IID30_IDAOFieldsW         5f739a18     daouuid:daouuid.obj
 0002:00008a28       _IID30_ICDAOJETField       5f739a28     daouuid:daouuid.obj
 0002:00008a38       _CLSID30_CDAOIndex         5f739a38     daouuid:daouuid.obj
 0002:00008a48       _IID30_IDAOIndex           5f739a48     daouuid:daouuid.obj
 0002:00008a58       _IID30_IDAOIndexW          5f739a58     daouuid:daouuid.obj
 0002:00008a68       _IID30_IDAOIndexes         5f739a68     daouuid:daouuid.obj
 0002:00008a78       _IID30_IDAOIndexesW        5f739a78     daouuid:daouuid.obj
 0002:00008a88       _IID30_IDAOIndexFields     5f739a88     daouuid:daouuid.obj
 0002:00008a98       _IID30_IDAOIndexFieldsW    5f739a98     daouuid:daouuid.obj
 0002:00008aa8       _CLSID30_CDAOGroup         5f739aa8     daouuid:daouuid.obj
 0002:00008ab8       _IID30_IDAOGroup           5f739ab8     daouuid:daouuid.obj
 0002:00008ac8       _IID30_IDAOGroupW          5f739ac8     daouuid:daouuid.obj
 0002:00008ad8       _IID30_IDAOGroups          5f739ad8     daouuid:daouuid.obj
 0002:00008ae8       _IID30_IDAOGroupsW         5f739ae8     daouuid:daouuid.obj
 0002:00008af8       _CLSID30_CDAOUser          5f739af8     daouuid:daouuid.obj
 0002:00008b08       _IID30_IDAOUser            5f739b08     daouuid:daouuid.obj
 0002:00008b18       _IID30_IDAOUserW           5f739b18     daouuid:daouuid.obj
 0002:00008b28       _IID30_IDAOUsers           5f739b28     daouuid:daouuid.obj
 0002:00008b38       _IID30_IDAOUsersW          5f739b38     daouuid:daouuid.obj
 0002:00008b48       _IID30_IDAODatabase        5f739b48     daouuid:daouuid.obj
 0002:00008b58       _IID30_IDAODatabaseW       5f739b58     daouuid:daouuid.obj
 0002:00008b68       _IID30_IDAODatabases       5f739b68     daouuid:daouuid.obj
 0002:00008b78       _IID30_IDAODatabasesW      5f739b78     daouuid:daouuid.obj
 0002:00008b88       _IID30_ICDAOJETDatabase    5f739b88     daouuid:daouuid.obj
 0002:00008b98       _CLSID30_CDAOQueryDef      5f739b98     daouuid:daouuid.obj
 0002:00008ba8       _IID30_IDAOQueryDef        5f739ba8     daouuid:daouuid.obj
 0002:00008bb8       _IID30_IDAOQueryDefW       5f739bb8     daouuid:daouuid.obj
 0002:00008bc8       _IID30_IDAOQueryDefs       5f739bc8     daouuid:daouuid.obj
 0002:00008bd8       _IID30_IDAOQueryDefsW      5f739bd8     daouuid:daouuid.obj
 0002:00008be8       _IID30_IDAOParameter       5f739be8     daouuid:daouuid.obj
 0002:00008bf8       _IID30_IDAOParameterW      5f739bf8     daouuid:daouuid.obj
 0002:00008c08       _IID30_IDAOParameters      5f739c08     daouuid:daouuid.obj
 0002:00008c18       _IID30_IDAOParametersW     5f739c18     daouuid:daouuid.obj
 0002:00008c28       _CLSID30_CDAORelation      5f739c28     daouuid:daouuid.obj
 0002:00008c38       _IID30_IDAORelation        5f739c38     daouuid:daouuid.obj
 0002:00008c48       _IID30_IDAORelationW       5f739c48     daouuid:daouuid.obj
 0002:00008c58       _IID30_IDAORelations       5f739c58     daouuid:daouuid.obj
 0002:00008c68       _IID30_IDAORelationsW      5f739c68     daouuid:daouuid.obj
 0002:00008c78       _IID30_IDAOContainer       5f739c78     daouuid:daouuid.obj
 0002:00008c88       _IID30_IDAOContainerW      5f739c88     daouuid:daouuid.obj
 0002:00008c98       _IID30_IDAOContainers      5f739c98     daouuid:daouuid.obj
 0002:00008ca8       _IID30_IDAOContainersW     5f739ca8     daouuid:daouuid.obj
 0002:00008cb8       _IID30_IDAODocument        5f739cb8     daouuid:daouuid.obj
 0002:00008cc8       _IID30_IDAODocumentW       5f739cc8     daouuid:daouuid.obj
 0002:00008cd8       _IID30_IDAODocuments       5f739cd8     daouuid:daouuid.obj
 0002:00008ce8       _IID30_IDAODocumentsW      5f739ce8     daouuid:daouuid.obj
 0002:00008cf8       _IID30_IDAOCollection      5f739cf8     daouuid:daouuid.obj
 0002:00008d08       _IID30_IDAODynaCollection  5f739d08     daouuid:daouuid.obj
 0002:00008d18       _IID30_IDAOQueryCP         5f739d18     daouuid:daouuid.obj
 0002:00008d28       _IID30_IDAOQueryAS         5f739d28     daouuid:daouuid.obj
 0002:00008d38       _IID30_IDisconnect         5f739d38     daouuid:daouuid.obj
 0002:00008d48       _IID30_IDisconnectAll      5f739d48     daouuid:daouuid.obj
 0002:00008d58       _IID30_IDSCAdviseSink      5f739d58     daouuid:daouuid.obj
 0002:00008d68       _IID30_IDSCConnectionPoint 5f739d68     daouuid:daouuid.obj
 0002:00008d78       _IID30_IDBAdviseSink       5f739d78     daouuid:daouuid.obj
 0002:00008d88       _IID30_IDBConnectionPoint  5f739d88     daouuid:daouuid.obj
 0002:00008da0       __sz_ole32                 5f739da0     ole32:ole32.dll
 0002:00008db0       __sz_OLEAUT32              5f739db0     oleaut32:OLEAUT32.dll
 0002:00008dc0       __sz_ODBC32                5f739dc0     odbc32:ODBC32.dll
 0002:00008dd0       ??_R1A@?0A@A@CObject@@8    5f739dd0     dbcore.obj
 0002:00008de8       ??_R1A@?0A@A@CException@@8 5f739de8     dbcore.obj
 0002:00008e00       ??_R1A@?0A@A@CDBException@@8 5f739e00     dbcore.obj
 0002:00008e18       ??_R2CDBException@@8       5f739e18     dbcore.obj
 0002:00008e28       ??_R3CDBException@@8       5f739e28     dbcore.obj
 0002:00008e38       ??_R4CDBException@@6B@     5f739e38     dbcore.obj
 0002:00008e50       ??_R1A@?0A@A@CDatabase@@8  5f739e50     dbcore.obj
 0002:00008e68       ??_R2CDatabase@@8          5f739e68     dbcore.obj
 0002:00008e78       ??_R3CDatabase@@8          5f739e78     dbcore.obj
 0002:00008e88       ??_R4CDatabase@@6B@        5f739e88     dbcore.obj
 0002:00008ea0       ??_R1A@?0A@A@CRecordset@@8 5f739ea0     dbcore.obj
 0002:00008eb8       ??_R2CRecordset@@8         5f739eb8     dbcore.obj
 0002:00008ec8       ??_R3CRecordset@@8         5f739ec8     dbcore.obj
 0002:00008ed8       ??_R4CRecordset@@6B@       5f739ed8     dbcore.obj
 0002:00008ef0       ??_R1A@?0A@A@CNoTrackObject@@8 5f739ef0     dbcore.obj
 0002:00008f08       ??_R1A@?0A@A@_AFX_DB_STATE@@8 5f739f08     dbcore.obj
 0002:00008f20       ??_R2_AFX_DB_STATE@@8      5f739f20     dbcore.obj
 0002:00008f30       ??_R3_AFX_DB_STATE@@8      5f739f30     dbcore.obj
 0002:00008f40       ??_R4_AFX_DB_STATE@@6B@    5f739f40     dbcore.obj
 0002:00008f54       ??_R2CNoTrackObject@@8     5f739f54     dbcore.obj
 0002:00008f60       ??_R3CNoTrackObject@@8     5f739f60     dbcore.obj
 0002:00008f70       ??_R4CNoTrackObject@@6B@   5f739f70     dbcore.obj
 0002:00008f88       ??_R1A@?0A@A@CCmdTarget@@8 5f739f88     dbview.obj
 0002:00008fa0       ??_R1A@?0A@A@CWnd@@8       5f739fa0     dbview.obj
 0002:00008fb8       ??_R1A@?0A@A@CView@@8      5f739fb8     dbview.obj
 0002:00008fd0       ??_R1A@?0A@A@CScrollView@@8 5f739fd0     dbview.obj
 0002:00008fe8       ??_R1A@?0A@A@CFormView@@8  5f739fe8     dbview.obj
 0002:00009000       ??_R1A@?0A@A@CRecordView@@8 5f73a000     dbview.obj
 0002:00009018       ??_R2CRecordView@@8        5f73a018     dbview.obj
 0002:00009038       ??_R3CRecordView@@8        5f73a038     dbview.obj
 0002:00009048       ??_R4CRecordView@@6B@      5f73a048     dbview.obj
 0002:00009060       ??_R1A@?0A@A@CLongBinary@@8 5f73a060     dblong.obj
 0002:00009078       ??_R2CLongBinary@@8        5f73a078     dblong.obj
 0002:00009088       ??_R3CLongBinary@@8        5f73a088     dblong.obj
 0002:00009098       ??_R4CLongBinary@@6B@      5f73a098     dblong.obj
 0002:000090b0       ??_R1A@?0A@A@CDBVariant@@8 5f73a0b0     dbvar.obj
 0002:000090c8       ??_R2CDBVariant@@8         5f73a0c8     dbvar.obj
 0002:000090d0       ??_R3CDBVariant@@8         5f73a0d0     dbvar.obj
 0002:000090e0       ??_R4CDBVariant@@6B@       5f73a0e0     dbvar.obj
 0002:000090f8       ??_R1A@?0A@A@_AFX_DAO_STATE@@8 5f73a0f8     daocore.obj
 0002:00009110       ??_R2_AFX_DAO_STATE@@8     5f73a110     daocore.obj
 0002:00009120       ??_R3_AFX_DAO_STATE@@8     5f73a120     daocore.obj
 0002:00009130       ??_R4_AFX_DAO_STATE@@6B@   5f73a130     daocore.obj
 0002:00009148       ??_R1A@?0A@A@CDaoIndexInfo@@8 5f73a148     daocore.obj
 0002:00009160       ??_R2CDaoIndexInfo@@8      5f73a160     daocore.obj
 0002:00009168       ??_R3CDaoIndexInfo@@8      5f73a168     daocore.obj
 0002:00009178       ??_R4CDaoIndexInfo@@6B@    5f73a178     daocore.obj
 0002:00009190       ??_R1A@?0A@A@CDaoRelationInfo@@8 5f73a190     daocore.obj
 0002:000091a8       ??_R2CDaoRelationInfo@@8   5f73a1a8     daocore.obj
 0002:000091b0       ??_R3CDaoRelationInfo@@8   5f73a1b0     daocore.obj
 0002:000091c0       ??_R4CDaoRelationInfo@@6B@ 5f73a1c0     daocore.obj
 0002:000091d8       ??_R1A@?0A@A@CDaoException@@8 5f73a1d8     daocore.obj
 0002:000091f0       ??_R2CDaoException@@8      5f73a1f0     daocore.obj
 0002:00009200       ??_R3CDaoException@@8      5f73a200     daocore.obj
 0002:00009210       ??_R4CDaoException@@6B@    5f73a210     daocore.obj
 0002:00009228       ??_R1A@?0A@A@CDaoErrorInfo@@8 5f73a228     daocore.obj
 0002:00009240       ??_R2CDaoErrorInfo@@8      5f73a240     daocore.obj
 0002:00009248       ??_R3CDaoErrorInfo@@8      5f73a248     daocore.obj
 0002:00009258       ??_R4CDaoErrorInfo@@6B@    5f73a258     daocore.obj
 0002:00009270       ??_R1A@?0A@A@CDaoWorkspace@@8 5f73a270     daocore.obj
 0002:00009288       ??_R2CDaoWorkspace@@8      5f73a288     daocore.obj
 0002:00009298       ??_R3CDaoWorkspace@@8      5f73a298     daocore.obj
 0002:000092a8       ??_R4CDaoWorkspace@@6B@    5f73a2a8     daocore.obj
 0002:000092c0       ??_R1A@?0A@A@CDaoDatabase@@8 5f73a2c0     daocore.obj
 0002:000092d8       ??_R2CDaoDatabase@@8       5f73a2d8     daocore.obj
 0002:000092e8       ??_R3CDaoDatabase@@8       5f73a2e8     daocore.obj
 0002:000092f8       ??_R4CDaoDatabase@@6B@     5f73a2f8     daocore.obj
 0002:00009310       ??_R1A@?0A@A@CDaoRelationFieldInfo@@8 5f73a310     daocore.obj
 0002:00009328       ??_R2CDaoRelationFieldInfo@@8 5f73a328     daocore.obj
 0002:00009330       ??_R3CDaoRelationFieldInfo@@8 5f73a330     daocore.obj
 0002:00009340       ??_R4CDaoRelationFieldInfo@@6B@ 5f73a340     daocore.obj
 0002:00009358       ??_R1A@?0A@A@CDaoTableDef@@8 5f73a358     daocore.obj
 0002:00009370       ??_R2CDaoTableDef@@8       5f73a370     daocore.obj
 0002:00009380       ??_R3CDaoTableDef@@8       5f73a380     daocore.obj
 0002:00009390       ??_R4CDaoTableDef@@6B@     5f73a390     daocore.obj
 0002:000093a8       ??_R1A@?0A@A@CDaoFieldInfo@@8 5f73a3a8     daocore.obj
 0002:000093c0       ??_R2CDaoFieldInfo@@8      5f73a3c0     daocore.obj
 0002:000093c8       ??_R3CDaoFieldInfo@@8      5f73a3c8     daocore.obj
 0002:000093d8       ??_R4CDaoFieldInfo@@6B@    5f73a3d8     daocore.obj
 0002:000093f0       ??_R1A@?0A@A@CDaoQueryDef@@8 5f73a3f0     daocore.obj
 0002:00009408       ??_R2CDaoQueryDef@@8       5f73a408     daocore.obj
 0002:00009418       ??_R3CDaoQueryDef@@8       5f73a418     daocore.obj
 0002:00009428       ??_R4CDaoQueryDef@@6B@     5f73a428     daocore.obj
 0002:00009440       ??_R1A@?0A@A@CDaoRecordset@@8 5f73a440     daocore.obj
 0002:00009458       ??_R2CDaoRecordset@@8      5f73a458     daocore.obj
 0002:00009468       ??_R3CDaoRecordset@@8      5f73a468     daocore.obj
 0002:00009478       ??_R4CDaoRecordset@@6B@    5f73a478     daocore.obj
 0002:00009490       ??_R1A@?0A@A@CDaoIndexFieldInfo@@8 5f73a490     daocore.obj
 0002:000094a8       ??_R2CDaoIndexFieldInfo@@8 5f73a4a8     daocore.obj
 0002:000094b0       ??_R3CDaoIndexFieldInfo@@8 5f73a4b0     daocore.obj
 0002:000094c0       ??_R4CDaoIndexFieldInfo@@6B@ 5f73a4c0     daocore.obj
 0002:000094d8       ??_R1A@?0A@A@CDaoRecordView@@8 5f73a4d8     daoview.obj
 0002:000094f0       ??_R2CDaoRecordView@@8     5f73a4f0     daoview.obj
 0002:00009510       ??_R3CDaoRecordView@@8     5f73a510     daoview.obj
 0002:00009520       ??_R4CDaoRecordView@@6B@   5f73a520     daoview.obj
 0002:00009538       ??_R1A@?0A@A@type_info@@8  5f73a538     msvcrtd:ti_inst.obj
 0002:00009550       ??_R2type_info@@8          5f73a550     msvcrtd:ti_inst.obj
 0002:00009558       ??_R3type_info@@8          5f73a558     msvcrtd:ti_inst.obj
 0002:00009568       ??_R4type_info@@6B@        5f73a568     msvcrtd:ti_inst.obj
 0002:000095f8       __CT??_R0PAX@84            5f73a5f8     dbcore.obj
 0002:00009618       __CT??_R0PAVCObject@@@84   5f73a618     dbcore.obj
 0002:00009638       __CT??_R0PAVCException@@@84 5f73a638     dbcore.obj
 0002:00009658       __CT??_R0PAVCDBException@@@84 5f73a658     dbcore.obj
 0002:00009678       __CTA4PAVCDBException@@    5f73a678     dbcore.obj
 0002:00009690       __TI4PAVCDBException@@     5f73a690     dbcore.obj
 0002:0000c448       __CT??_R0PAVCDaoException@@@84 5f73d448     daocore.obj
 0002:0000c468       __CTA4PAVCDaoException@@   5f73d468     daocore.obj
 0002:0000c480       __TI4PAVCDaoException@@    5f73d480     daocore.obj
 0002:0000c958       __DELAY_IMPORT_DESCRIPTOR_ole32 5f73d958     ole32:ole32.dll
 0002:0000c978       __DELAY_IMPORT_DESCRIPTOR_OLEAUT32 5f73d978     oleaut32:OLEAUT32.dll
 0002:0000c998       __DELAY_IMPORT_DESCRIPTOR_ODBC32 5f73d998     odbc32:ODBC32.dll
 0002:0000c9b8       __NULL_DELAY_IMPORT_DESCRIPTOR 5f73d9b8     ole32:ole32.dll
 0002:0000ca58       \177ODBC32_NULL_THUNK_DATA_DLN 5f73da58     odbc32:ODBC32.dll
 0002:0000ca60       \177OLEAUT32_NULL_THUNK_DATA_DLN 5f73da60     oleaut32:OLEAUT32.dll
 0002:0000ca70       \177ole32_NULL_THUNK_DATA_DLN 5f73da70     ole32:ole32.dll
 0002:0000cab0       \177ole32_NULL_THUNK_DATA_DLB 5f73dab0     ole32:ole32.dll
 0002:0000cac0       \177OLEAUT32_NULL_THUNK_DATA_DLB 5f73dac0     oleaut32:OLEAUT32.dll
 0002:0000cac8       \177ODBC32_NULL_THUNK_DATA_DLB 5f73dac8     odbc32:ODBC32.dll
 0002:0000cb48       __IMPORT_DESCRIPTOR_MFC42uD 5f73db48     MFC42UD:MFC42uD.DLL
 0002:0000cb5c       __IMPORT_DESCRIPTOR_MFCO42uD 5f73db5c     MFCO42UD:MFCO42uD.DLL
 0002:0000cb70       __IMPORT_DESCRIPTOR_MSVCRTD 5f73db70     msvcrtd:MSVCRTD.dll
 0002:0000cb84       __IMPORT_DESCRIPTOR_KERNEL32 5f73db84     kernel32:KERNEL32.dll
 0002:0000cb98       __IMPORT_DESCRIPTOR_USER32 5f73db98     user32:USER32.dll
 0002:0000cbac       __NULL_IMPORT_DESCRIPTOR   5f73dbac     MFC42UD:MFC42uD.DLL
 0003:00000000       ___xc_a                    5f73f000     msvcrtd:cinitexe.obj
 0003:00000008       ___xc_z                    5f73f008     msvcrtd:cinitexe.obj
 0003:0000000c       ___xi_a                    5f73f00c     msvcrtd:cinitexe.obj
 0003:00000010       ___xi_z                    5f73f010     msvcrtd:cinitexe.obj
 0003:0000002c       __pRawDllMain              5f73f02c     dlldb.obj
 0003:00000030       ?_afxForceVectorDelete_mfcd@@3P6AXXZA 5f73f030     dlldb.obj
 0003:00000038       ?GUID_ATLVer30@ATL@@3U_GUID@@A 5f73f038     dlldb.obj
 0003:00000060       ??_R0PAX@8                 5f73f060     dbcore.obj
 0003:00000070       ??_R0PAVCObject@@@8        5f73f070     dbcore.obj
 0003:00000088       ??_R0PAVCException@@@8     5f73f088     dbcore.obj
 0003:000000a8       ??_R0PAVCDBException@@@8   5f73f0a8     dbcore.obj
 0003:000000c8       ??_R0?AVCObject@@@8        5f73f0c8     dbcore.obj
 0003:000000e0       ??_R0?AVCException@@@8     5f73f0e0     dbcore.obj
 0003:00000100       ??_R0?AVCDBException@@@8   5f73f100     dbcore.obj
 0003:00000120       ??_R0?AVCDatabase@@@8      5f73f120     dbcore.obj
 0003:00000138       ??_R0?AVCRecordset@@@8     5f73f138     dbcore.obj
 0003:00000158       ??_R0?AVCNoTrackObject@@@8 5f73f158     dbcore.obj
 0003:00000178       ??_R0?AV_AFX_DB_STATE@@@8  5f73f178     dbcore.obj
 0003:000001c8       ??_R0?AVCCmdTarget@@@8     5f73f1c8     dbview.obj
 0003:000001e8       ??_R0?AVCWnd@@@8           5f73f1e8     dbview.obj
 0003:00000200       ??_R0?AVCView@@@8          5f73f200     dbview.obj
 0003:00000218       ??_R0?AVCScrollView@@@8    5f73f218     dbview.obj
 0003:00000238       ??_R0?AVCFormView@@@8      5f73f238     dbview.obj
 0003:00000250       ??_R0?AVCRecordView@@@8    5f73f250     dbview.obj
 0003:00000288       ??_R0?AVCLongBinary@@@8    5f73f288     dblong.obj
 0003:000002b0       ??_R0?AVCDBVariant@@@8     5f73f2b0     dbvar.obj
 0003:000002e8       ?_afxNullVariant@@3UtagVARIANT@@A 5f73f2e8     daocore.obj
 0003:000002f8       ?_afxOptionalVariant@@3UtagVARIANT@@A 5f73f2f8     daocore.obj
 0003:00000308       ??_R0?AV_AFX_DAO_STATE@@@8 5f73f308     daocore.obj
 0003:00000328       ??_R0?AUCDaoIndexInfo@@@8  5f73f328     daocore.obj
 0003:00000348       ??_R0?AUCDaoRelationInfo@@@8 5f73f348     daocore.obj
 0003:00000368       ??_R0?AVCDaoException@@@8  5f73f368     daocore.obj
 0003:00000388       ??_R0?AUCDaoErrorInfo@@@8  5f73f388     daocore.obj
 0003:000003a8       ??_R0PAVCDaoException@@@8  5f73f3a8     daocore.obj
 0003:000003c8       ??_R0?AVCDaoWorkspace@@@8  5f73f3c8     daocore.obj
 0003:000003e8       ??_R0?AVCDaoDatabase@@@8   5f73f3e8     daocore.obj
 0003:00000408       ??_R0?AUCDaoRelationFieldInfo@@@8 5f73f408     daocore.obj
 0003:00000430       ??_R0?AVCDaoTableDef@@@8   5f73f430     daocore.obj
 0003:00000450       ??_R0?AUCDaoFieldInfo@@@8  5f73f450     daocore.obj
 0003:00000470       ??_R0?AVCDaoQueryDef@@@8   5f73f470     daocore.obj
 0003:00000490       ??_R0?AVCDaoRecordset@@@8  5f73f490     daocore.obj
 0003:000004b0       ??_R0?AUCDaoIndexFieldInfo@@@8 5f73f4b0     daocore.obj
 0003:00000508       ??_R0?AVCDaoRecordView@@@8 5f73f508     daoview.obj
 0003:00000540       ??_R0?AVtype_info@@@8      5f73f540     msvcrtd:ti_inst.obj
 0003:00000560       __imp__SQLGetInfo@20       5f73f560     odbc32:ODBC32.dll
 0003:00000564       __imp__SQLSetConnectOption@12 5f73f564     odbc32:ODBC32.dll
 0003:00000568       __imp__SQLBindCol@24       5f73f568     odbc32:ODBC32.dll
 0003:0000056c       __imp__SQLParamData@8      5f73f56c     odbc32:ODBC32.dll
 0003:00000570       __imp__SQLBindParameter@40 5f73f570     odbc32:ODBC32.dll
 0003:00000574       __imp__SQLPutData@12       5f73f574     odbc32:ODBC32.dll
 0003:00000578       __imp__SQLError@32         5f73f578     odbc32:ODBC32.dll
 0003:0000057c       __imp__SQLFreeStmt@8       5f73f57c     odbc32:ODBC32.dll
 0003:00000580       __imp__SQLCancel@4         5f73f580     odbc32:ODBC32.dll
 0003:00000584       __imp__SQLMoreResults@4    5f73f584     odbc32:ODBC32.dll
 0003:00000588       __imp__SQLFetch@4          5f73f588     odbc32:ODBC32.dll
 0003:0000058c       __imp__SQLNumResultCols@8  5f73f58c     odbc32:ODBC32.dll
 0003:00000590       __imp__SQLExecDirect@12    5f73f590     odbc32:ODBC32.dll
 0003:00000594       __imp__SQLAllocStmt@8      5f73f594     odbc32:ODBC32.dll
 0003:00000598       __imp__SQLFreeConnect@4    5f73f598     odbc32:ODBC32.dll
 0003:0000059c       __imp__SQLDisconnect@4     5f73f59c     odbc32:ODBC32.dll
 0003:000005a0       __imp__SQLFreeEnv@4        5f73f5a0     odbc32:ODBC32.dll
 0003:000005a4       __imp__SQLSetStmtOption@12 5f73f5a4     odbc32:ODBC32.dll
 0003:000005a8       __imp__SQLRowCount@8       5f73f5a8     odbc32:ODBC32.dll
 0003:000005ac       __imp__SQLExecute@4        5f73f5ac     odbc32:ODBC32.dll
 0003:000005b0       __imp__SQLTransact@12      5f73f5b0     odbc32:ODBC32.dll
 0003:000005b4       __imp__SQLAllocConnect@8   5f73f5b4     odbc32:ODBC32.dll
 0003:000005b8       __imp__SQLAllocEnv@4       5f73f5b8     odbc32:ODBC32.dll
 0003:000005bc       __imp__SQLDriverConnect@32 5f73f5bc     odbc32:ODBC32.dll
 0003:000005c0       __imp__SQLGetData@24       5f73f5c0     odbc32:ODBC32.dll
 0003:000005c4       __imp__SQLSetPos@16        5f73f5c4     odbc32:ODBC32.dll
 0003:000005c8       __imp__SQLGetStmtOption@12 5f73f5c8     odbc32:ODBC32.dll
 0003:000005cc       __imp__SQLPrepare@12       5f73f5cc     odbc32:ODBC32.dll
 0003:000005d0       __imp__SQLGetFunctions@12  5f73f5d0     odbc32:ODBC32.dll
 0003:000005d4       __imp__SQLDescribeCol@36   5f73f5d4     odbc32:ODBC32.dll
 0003:000005d8       __imp__SQLExtendedFetch@20 5f73f5d8     odbc32:ODBC32.dll
 0003:000005dc       __imp__SQLGetCursorName@16 5f73f5dc     odbc32:ODBC32.dll
 0003:000005e0       \177ODBC32_NULL_THUNK_DATA_DLA 5f73f5e0     odbc32:ODBC32.dll
 0003:000005e4       __imp__SysFreeString@4     5f73f5e4     oleaut32:OLEAUT32.dll
 0003:000005e8       \177OLEAUT32_NULL_THUNK_DATA_DLA 5f73f5e8     oleaut32:OLEAUT32.dll
 0003:000005ec       __imp__CoUninitialize@0    5f73f5ec     ole32:ole32.dll
 0003:000005f0       __imp__CoGetClassObject@20 5f73f5f0     ole32:ole32.dll
 0003:000005f4       __imp__CoInitialize@4      5f73f5f4     ole32:ole32.dll
 0003:000005f8       \177ole32_NULL_THUNK_DATA_DLA 5f73f5f8     ole32:ole32.dll
 0003:00000600       ?ATL_CREATE_OBJECT@CComApartment@ATL@@2IA 5f73f600     dlldb.obj
 0003:00000608       ?m_libid@CComModule@ATL@@2U_GUID@@A 5f73f608     dlldb.obj
 0003:00000618       ?_pModule@ATL@@3PAVCComModule@1@A 5f73f618     dlldb.obj
 0003:00000634       ?_afxDbState@@3V?$CProcessLocal@V_AFX_DB_STATE@@@@A 5f73f634     dbcore.obj
 0003:00000638       ?bTraceSql@@3HA            5f73f638     dbcore.obj
 0003:00000640       __hmod__OLE32              5f73f640     ole32:ole32.dll
 0003:00000644       __hmod__OLEAUT32           5f73f644     oleaut32:OLEAUT32.dll
 0003:00000648       __hmod__ODBC32             5f73f648     odbc32:ODBC32.dll
 0003:0000064c       ___puiHead                 5f73f64c     delayimp:delayhlp.obj
 0003:00000650       ___pfnDliFailureHook       5f73f650     delayimp:delayhk1.obj
 0003:00000654       ___pfnDliNotifyHook        5f73f654     delayimp:delayhk2.obj
 0003:00000658       __adjust_fdiv              5f73f658     <common>
 0003:0000065c       ___onexitend               5f73f65c     <common>
 0003:00000660       ___onexitbegin             5f73f660     <common>

 entry point at        0001:0002c330

 Static symbols

 0001:0001673c       ?_AfxDetermineDaoVersion@@YAEXZ 5f71773c f   daocore.obj
 0001:0002cf4e       _$E376                     5f72df4e f   dbcore.obj
 0001:0002cf5d       _$E373                     5f72df5d f   dbcore.obj
 0001:0002cf62       _$E375                     5f72df62 f   dbcore.obj
 0001:0002cf74       _$E374                     5f72df74 f   dbcore.obj
 0001:0002d1e0       ?_AfxForceVectorDelete@@YAXXZ 5f72e1e0 f   dlldb.obj
 0001:0002c160       _$$$00001                  5f72d160 f   msvcrtd:chkstk.obj
 0001:0002c16c       probepages                 5f72d16c f   msvcrtd:chkstk.obj
 0001:0002c180       lastpage                   5f72d180 f   msvcrtd:chkstk.obj
 0001:0002c0c0       ?ArrayUnwindFilter@@YAHPAU_EXCEPTION_POINTERS@@@Z 5f72d0c0 f   msvcrtd:ehvecdtr.obj
 0001:0002ca2b       ?OverlayIAT@@YGXPAU_IMAGE_THUNK_DATA32@@PBU1@@Z 5f72da2b f   delayimp:delayhlp.obj

 105 bytes saved through ICF

